:020000040800F2
:1000000000A00020B1980108199901088981010810
:1000100019990108199901081999010800000000AF
:100020000000000000000000000000001999010815
:10003000199901080000000019990108B54F01083D
:1000400019990108199901081999010819990108C4
:100050001999010819990108EF260108F9260108E4
:10006000F7260108F5260108F32601088D7A000815
:100070007D7A00086D7A00085D7A00084D7A0008E4
:10008000397A0008257A0008199901081999010898
:10009000199901081999010819990108F12601080F
:1000A000A14C0108DD4C0108914C0108054D0108E7
:1000B000D14C0108C14C0108B14C01081999010843
:1000C0001999010819990108199901081999010844
:1000D0001999010861790008557900084B790008E1
:1000E000ED260108199901081999010819990108C3
:1000F0001999010819990108199901081999010814
:100100000000000000000000000000001999010834
:1001100019990108199901081999010819990108F3
:10012000117A0008FD790008E9790008D5790008FE
:10013000C1790008199901080000000000000000C2
:10014000199901081999010819990108000000007E
:10015000000000000000000000000000000000009F
:100160000000000000000000199901081999010819
:1001700019990108000000000000000000000000C4
:080180000000000019990108BC
:100188002DE9F04FA34BA44A2DED068B1A60A34B23
:10019800AFB000221A6009F0C3FD18B90AF018FAC6
:1001A80012F0ACFB09F0E0FD9D4A137843F001031F
:1001B80013709C4A9C4B116899424FF0000309D177
:1001C800136062B6994B1B6883F30888984B1B68C9
:1001D8009847FEE7974A984C4FF47001C2F8881088
:1001E8000C930D93236843F480332360236803F44E
:1001F80000330D930C9B01330C930D9B1BB90C9B87
:10020800B3F5A04FF2D1236813F4003318BF0123CC
:100218000D930D9B012B52D0DFF81882874BC8F83D
:100228000C30874F666A3E60636A43F0807363628E
:10023800636943F4FC032EAD636103238DF86A30D0
:1002480041F6FF7325F8503D4FF09040294607F0DE
:1002580089FB4FF6FF7329467A48ADF8683007F0F6
:1002680081FB2946784807F07DFB2946774807F047
:1002780079FB2946764807F075FB2946754807F04B
:1002880071FB28460DF04CFD734A1A9BB3FBF2F341
:10029800724A00211360381D10221BF0D9FF704AE2
:1002A800704B5360F02388F82330072100239360B4
:1002B800DFF8E0E111604FF0010C6B4928E06B4B6F
:1002C80012221A606368636063686360636843F45A
:1002D80080636360636823F47C136360636843F43A
:1002E800E8136360236843F0807323602268524BED
:1002F8009501FBD55A6822F003025A605A6842F009
:1003080002025A60636803F00C03082BFAD183E7F2
:1003180098023EF8135000F19040002245FA02F886
:1003280018F0010F18BF0CFA02F802F101021EBF03
:100338000860A1F804800C31102AEFD10133062B94
:10034800E6D14B4D4B4B95F8EB21DFF84C911A70E9
:100358000020AB68C9F8003016F09EFC464A92F8B7
:1003680000B000234FF0170A0BEB0301434A52F881
:10037800210003F1010840B1022380F806A0C371EF
:1003880080F80880012112F06DF84346032BEBD169
:10039800002016F081FCA369394843F00103A361EA
:1003A800402200211BF054FF364B4FF0FF321A60F9
:1003B800C3F80320D9F800301C0711D595F84C3242
:1003C800012B0DD816F0805600F0808608E093F8CF
:1003D8004F22012A04D1002283F84E2212F03CFB5E
:1003E800642014F0A3FD4FF48C7200212648274E98
:1003F8001BF02EFF0024B046A1590023244850F8D2
:10040800330081424FEAC30248D108EB020393F854
:10041800D00047E0AC1700201D9D0008B017002051
:10042800914C0020FC9F0020EFBEADDE00D8FF1FDE
:1004380004D8FF1F00ED00E0001002400005FA0597
:10044800800700200004004800080048000C00480D
:10045800001000480014004840420F006842002085
:1004680010E000E03F190100DC43002000200240BA
:10047800B0450020CA21002084EA010888EA010862
:10048800E83B0020EC3C002098400020B8C301085D
:1004980084C401084EE601089824002001330A2B81
:1004A800ACD100200C3416F089FACC2CA4D16E4CB7
:1004B80004F1CC06207911F045FF0C3414F8032C14
:1004C80014F8041C11F092FFA642F3D1674BDFF831
:1004D800C481674AD9F800401A604FF005093C22E8
:1004E8000021644888F800901BF0B2FE00224046C4
:1004F800DFF8A4C1DFF87C814B4604F0400696463D
:100508004FF0FF091CF9011F02F8081002EB080A56
:1005180056B91E39C9B201299FBF03F1FF338AF8C2
:100528000090DBB24FF0010E0C323C2AEAD1BEF14A
:10053800000F00D00370504B95F8058083F80080B9
:100548004E4B4F497B61A00603F1D8030B6058BF9F
:100558004C4B4D4A56BF03EBC80301235B789361AC
:100568004A4A002340F2DC5122F813100133082BC9
:10057800FAD100211C2213A81BF06AFEA1050AD596
:100588002022212301213A777B778DF858108DF8A6
:1005980066208DF86730B8F10E0F03D008F0EF032E
:1005A800082B02D101238DF86030012010F000FAE9
:1005B80018B14088003018BF012000F001008DF804
:1005C8005100022010F0F4F918B14088003018BF2B
:1005D8000120C4F340038DF85430C4F3403300368F
:1005E8008DF84C30C4F3C03318BF012600F0010069
:1005F8008DF84F3014F400638DF852008DF8566072
:1006080004D095F822325A1E534253418DF8503087
:10061800C4F300438DF85730C4F3C0038DF84E304F
:10062800BB69003318BF01238DF85930C4F3005358
:100638008DF85A30B5F8D230ADF85E30B5F8E03004
:10064800ADF85C3095F8E33004F001088DF84D8082
:1006580004F0080613BB0E4B93F8E23013F0FB0FBF
:100668000CBF012300231AE0B8C30108A84B0020DF
:1006780064480020AC4B0020D00D0020BC45002071
:100688002C4200204CCB010880070020F80E0020E7
:10069800B04500204C0F0020CFCA0108012395F86F
:1006A800E220079312F0FB0F14BF012100218DF8FF
:1006B80055108DF8612013B1B94BB3F8DE30ADF8A1
:1006C8006230B5F8D030ADF86430E30442BFB44BC3
:1006D800B3F8DA30ADF86430042A06D14FF480500C
:1006E80012F0E4F80023ADF86430AE4B95F8982288
:1006F8001A7000216422AC481BF0AAFD9DF86030F6
:10070800002B14BF02220022B8F1000F00D106B15D
:100718000132A64BA54CDFF8C08203EB8203D3F865
:100728001C319A1E203308930023049203930593E7
:10073800049B33F8022F04934FF6FF739A4200F09C
:10074800DD819DF85210D3B2120AD7B239B10C210B
:1007580001FB034109792A39012940F2CA819DF830
:10076800561031B10C21594360589149884200F024
:10077800C0819DF8571059B10C215943601865582C
:100788008C498D4200F0B5810179182900F0B181BA
:100798009DF8541031B10C2101FB0341097914294A
:1007A80000F0A7819DF84F1031B10C2101FB0341E6
:1007B8000979222900F09D819DF8501031B10C2152
:1007C80001FB03410979152900F093819DF8581020
:1007D80069B10C2101FB03419DF866000979884243
:1007E80000F087819DF86700884200F08281022A24
:1007F80002D19DF84C2003E0012A04D19DF84D2038
:10080800002A00F076819DF859206AB19DF8602091
:1008180052B9A3F10E02012A06D80C225A43A15854
:10082800654A914208BF04279DF85A200C2505FB0C
:10083800034532B19DF860201AB91A1F032A40F205
:100848003981012F43D14FF00C0B0BFB03FB04EB59
:100858000B0954F80B3003930026584B99F8040001
:1008680088F82060FF22C8F82C501E705E609E60D9
:10087800DE601E6483F8442083F8452083F84660D0
:1008880083F8476083F8486011F05CFD02228271AA
:10089800C771067299F8081011F0E4FD324699F80C
:1008A800051003980BF02EFC3A463146284614F002
:1008B800D5FA434B434AC8F83030434BC8F8343074
:1008C800C8F83860111F284614F020FA11E1022FE9
:1008D80046D19DF8142009921C264FF00C0B0BFBF7
:1008E80003FB06FB02F108EB010704EB0B064FF0D4
:1008F800010A4FF0000987F82120307987F8229003
:1009080087F82A9087F820A0FD62069111F01AFD59
:10091800099A80F806A05244027280F807A0317A3A
:1009280011F0A0FD4A46717954F80B000BF0EAFB70
:1009380052464946284614F091FA244B3B63244B0F
:100948007B63069BC7F8389003F11001214B1944CB
:100958000A1D284614F0DAF9059B53440593C8E0AC
:10096800032F40F0A5809DF84D109DF861200029C7
:1009780037D0002A35D04FF00C0B0BFB03FB039943
:1009880054F80B308B422CD1531E032B29D8DFE8A7
:1009980003F002250425082121E048211FE000BFBB
:1009A800B04500200C1F0020500F0020B8C30108DC
:1009B80000040040002C014000400140B81700200E
:1009C800BDB90008B407002019BB000849C10008D8
:1009D80097B90008A0070020800700201821B34B12
:1009E80019709DF85530B24EBDF8620073B3022AF3
:1009F80096F801A0BDF8643009D0032AAD4AAE4F7D
:100A08000EBF4FF0480E17464FF0080E02E0AB4FEE
:100A18004FF0180E5FFA8EF1DFF8AC9230B1A84AA9
:100A280002FB0EF2B2FBF0F292B202E003464FF67E
:100A3800FF72284611F03CFD49F82A0059F82A307F
:100A4800DF60B378192206EBC30327E0042A77781E
:100A580011D19C4AB2FBF0F2182192B2284611F04B
:100A680027FD994B43F82700984BC360B3780D22B4
:100A780006EBC30312E0BDF86430914AB2FBF0F212
:100A8800012192B2284611F013FD8F4B43F827003D
:100A98008F4BC360B378092206EBC3035A71B3784E
:100AA800727806EBC3010A7101328D6072701EE024
:100AB800042F1ED17E4EBDF85C20B378377806EB44
:100AC800C30301211F7128467D4B93FBF2F2BDF849
:100AD8005E3092B211F0ECFC7E4B43F82700B378FD
:100AE80006EBC3020A2151713278013232700133A8
:100AF800B370089B049A93427FF41AAE079B764E14
:100B080083F00102754B1A70754B1D78A5F1170318
:100B18000024022B34701ED8DFF8C8C1DFF8F8E1D2
:100B2800DCF814302344D3ED007AF5EE407AF1EE88
:100B380010FA04D16B4B03939A6952BB24E00FCB94
:100B480004EB0E0787E80F00337810340133C02C0C
:100B58003370E5D1EEE7644B13F835E086F800E032
:100B680003EBC503D3F804C0BCF1000FE2D0DFF8F3
:100B7800A8817445DEDA230103EB080763440FCB31
:100B8800013487E80F00F4E7584C2368DF0425D4C4
:100B98001EE0574B574A13F83500107003EBC50396
:100BA8005C68002CF0D0544F00238342ECDAC3EB8E
:100BB800C301621801EB070ED2F800C041F807C064
:100BC8009188AEF8041092798EF806200133ECE78C
:100BD80005F0EF03082B494B1FD120E03278012A9A
:100BE800F6D9474B03EB02121032F6EE007A1033B7
:100BF8009342EDD013ED047A27EE277A03ED047AB9
:100C080013ED057A27EE277A03ED057A13ED037ABB
:100C180027EE277A03ED037AE9E70E2D08D11A7833
:100C280042F010021A70182D08D113F06DFF05E07C
:100C38001A7822F010021A70192DF5E7314D13F0C9
:100C480045FF2B783F2043F004032B7011F07AFB0B
:100C58002D4A049510602D4A0121117038B11122D6
:100C680082710222C2710022027211F0FBFB284D30
:100C780000200BF055F8287E15F0A0FE2B7E03F01F
:100C88001F015B090122022B02FA01F208D0032B93
:100C980044D0012B46D11F498B6A1A438A6241E02E
:100CA8001C49CB681A43CA603CE000BFA40000207E
:100CB800500F002009BD0008A5BC0008DDBC0008D5
:100CC80040420F0000366E014C40002059BB00081E
:100CD80049BB0008101F00203F2500209440002039
:100CE800D00D0020800700204CCB0108982400205C
:100CF80064E40108B8410020B941002044160020EE
:100D0800F80C0020914C0020081800200C18002036
:100D18006C05002000100240F00C0020A9490B6966
:100D28001A430A61687D11F00DFB0C260B2302277C
:100D3800C37186710772E87D11F004FB4FF00D084E
:100D4800867180F807800772A87D11F0FBFA86711A
:100D5800C6710772687D11F0F5FA6A7E0E2111F0EE
:100D680045FBE87D11F0EEFA6A7E0E2111F03EFB9C
:100D7800A87D11F0E7FA6A7E0E2111F037FB287D75
:100D880030B111F0DFFA904B41465A7E11F02EFB3C
:100D980029698E4B99420AD103F56043DA6842F417
:100DA8008052DA60DA6822F48052DA6019E0884BFF
:100DB800994209D103F5EC331A6942F480421A6169
:100DC8001A6922F480420BE0824B994209D103F55B
:100DD800EA331A6942F400421A611A6922F400429D
:100DE8001A612B7F13B10023184601E0012302206A
:100DF8008A8822F480521204120C8A808A8892B25D
:100E080042F480528A8029690A8802F4415242F4E5
:100E18004572134303430B808B8823F470631B04D0
:100E28001B0C43F4E0638B808B8B23F400631B045F
:100E38001B0C8B8307230B822A6913889BB243F010
:100E480040031380287D18B111F07CFA11F0A3FA41
:100E5800236803F41073B3F5107F66D0262011F0D1
:100E680071FA0746272011F06DFA564D064675208F
:100E780015F0A4FD2B6B23F010032B632B6B43F0B1
:100E880010032B634FF001084FF00D09092387F871
:100E98000690FB7187F80880384604221E2111F05D
:100EA800A5FA0A2386F80690F37186F8088030467A
:100EB80004221E2111F09AFA474B484E1A6822F074
:100EC80001021A601968464A0A401A60454A1A61BE
:100ED8001A68002142EA08021A609960D96099608C
:100EE8009A6842F400429A601A681A605A6822F0B6
:100EF800784222F400425A601A6822F400321A60DA
:100F08001A6842EA08021A60D4F800A014273A4680
:100F180030461BF09DF91AF0020F0AF400490AF452
:100F28000068304618D0377016E02F492F4D0A78E0
:100F380000231846FF265F571F2F04BF5E5502F196
:100F4800FF3203F10C0304BFD2B201203C2BF2D1D3
:100F5800002883D00A7081E7B9F1000F01D022235D
:100F68004371B8F1000F01D01523C373204FDFF888
:100F780088A04FF00F0900264FF0060817F8010C5B
:100F8800002847D011F0DEF94FF0000B80F80680FA
:100F980080F8079080F808B017F8010C11F0D2F922
:100FA800132111F05FFA17F8011C5B46114810F87D
:100FB800130088424FEA430220D10AEB020393F858
:100FC8002D311FE0001002406C0500200030014068
:100FD80000380040003C004000540040AC21002094
:100FE800FFE0CF00300E50004C0F0020AC4B00202B
:100FF800AD210020E4C40108B8C301080133272B40
:10100800D4D1002307223B70FA70731C01227E7032
:10101800BA70DEB209F101095FFA89F9B9F1130F63
:1010280007F10507AAD1EB6A23F4F873EB62EB6AC0
:1010380043F4D873EB623C2015F0C0FC212015F076
:10104800BDFC7E487D4D0CF01AFD1AA80CF0ECFC96
:101058007B4B1A937B4B1B93022E4FF0000334BF3C
:101068001A4680221F924FF4807220924FF48062B9
:1010780021922022284622921AA94FF400521C934A
:101088001E9323922493ADF874600CF0DAFC2B685D
:1010980043F001032B606C4DAB6823F04053AB6009
:1010A800AB6843F08053AB600A2013F03FFFAB6896
:1010B80023F08043AB60AB68AB60AB6843F00043A0
:1010C800AB60AB68604A002B38DAFAE75F4B93F8FD
:1010D8004E32013B092B3FF683A92B2011F032F940
:1010E800182383710223C371044606720121C7F8CD
:1010F8009C0411F0B7F92046012111F051F93C2068
:1011080013F014FF95F84E22504B9642BFF65FA994
:10111800002015F0C1FD0021204611F041F978208A
:1011280013F0E2FE012015F0B7FD0121204611F071
:1011380037F9782013F0D8FE0136E3E7936844497D
:1011480023F040539360936843F00053936088689A
:10115800404B034043F468338B60D1683E4B3F48B3
:101168000B4043F40053D360136B013E23F00F038D
:101178001E43166300F1140C01234FF0380A4FF098
:10118800070B4FF0060E1F25C178002978D05E1C8A
:10119800042B41780779F6B20ED803EB4303D2F853
:1011A80030805B0005FA03F928EA090801FA03F31D
:1011B80043EA080313632FE0092B0ED8053BD2F846
:1011C80034800EFB03F305FA03F928EA090801FA4B
:1011D80003F343EA080353631EE00E2B0ED80A3BC1
:1011E800D2F838800EFB03F305FA03F928EA090858
:1011F80001FA03F343EA080393630DE00F3BD2F8C7
:101208003C800EFB03F305FA03F928EA090801FA02
:1012180003F343EA0803D363092921D90A399369F7
:10122800936901EB41010BFA01F823EA0803936182
:10123800936907FA01F11943916120E0080402401B
:1012480040010050C021002000010050B04500209E
:1012580000030050E010FCFF07C0FFFDAC21002098
:1012680001395369536901EB41010AFA01F823EA8C
:1012780008035361536903318F401F435761334655
:101288000530604580D1754B9A6842F001029A603A
:101298001A461168714BCD07FBD5DA68704D22F0FC
:1012A8000202DA60DA6842F00202DA60DA6842F0D2
:1012B8000102DA609A6842F004029A60D5F8C831EF
:1012C800002B40F0D687D5F8CC21002A40F0D187F2
:1012D800D5F8D021002A40F0CC8723689C031CD580
:1012E800C82013F023FEAE2016F07FFF08B112F0DD
:1012F80019FD039B5B4C83F80001C82013F016FE10
:10130800002323606360A3600223E3700BF093FE65
:1013180013F0CEFD544B0344A360B5F8D83195F8CB
:10132800D58195F8ED9195F8EEA1B5F9F0B1059351
:1013380095F8DA314D4D4E4F4E4E4F4806930024E6
:10134800182221462C606C60AC601AF081FF21469F
:1013580018223C8006F582701AF07AFF039B474AF0
:10136800C3F81C21232013F0E1FD0DF12E02012109
:10137800752005F0B1FE002864D0414AC6F808215E
:10138800404AC6F80C21432286F8042101210DF1B8
:101398002F02204605F0A0FE9DF82F2002F07E02C5
:1013A8008DF82F2038B1682A05D101223A701D2204
:1013B80086F8042146E09DF82E302D4C03F07E037C
:1013C800682B8DF82E3039D102232370039B062118
:1013D800D3F808311AAA084698479DF86D209DF859
:1013E8006B3092005B0003F0020302F004021A4320
:1013F8009DF8693003F00103134310D0012B01D18C
:10140800002302E0022B02D1012363701AE003F0EB
:101418000303032BF8D0032013F092FD12E0154BC1
:101428000EAAD3F8083101210C2098479DF83830CE
:1014380013F00F03EFD0042BE6D1E1E7702B04BFC4
:1014480004232370104900230B70094B1A78022AD1
:101458001CD0012013F074FD37E000BF00010050DC
:10146800B04500201C4C0020404B4C00442E00206E
:10147800402E002080070020CC2E002032C5010815
:10148800E170000833720008D8350020C34BC44807
:101498001860C4485860C448D860C4481861042318
:1014A8000B70C34B9DF814601A70C24A136843F05E
:1014B80001031360069B019300965B46524649461A
:1014C800404610F06DFB0028C3D0049B049A1B789B
:1014D800B94E43F002030020137015F0DDFB0A2417
:1014E80015F0CDFB192013F021FDD6F8D835DFF81B
:1014F800C88213F4803F02D101200AF011FC1920A0
:1015080013F014FD00200AF00BFC013CE8D1A94EB1
:10151800204615F0C1FB3368180705D5A74B1B6893
:101528009847A74B01221A70A64B9FEDA78A1B6804
:10153800A64F1B7B00EE103AB8EEC00A20EE080A50
:1015480009F091FAA24B9FEDA37A83ED000A934B21
:10155800D3ED047AA04B67EE887AC3ED007A2B8925
:101568009E4D07EE903AF8EEE77A9D4BC7EE276A54
:101578009FED9C7AC6EE877AC3ED007A13F006FBDE
:10158800FF211E2238461AF063FE974B01221A707B
:1015980000223A702A6812F4800F01BF02211970E4
:1015A8001B21797038463768B9070ED519784FF07E
:1015B800010E00F801E001F1020E0131C9B283F811
:1015C80000E04FF0020E00F801E0790708D519781D
:1015D80001F1010E83F800E04FF0030E00F801E07E
:1015E80017F00A0F0ED01978042747544F1CFFB282
:1015F8004FF0050E00F807E0CF1C0231C9B21F708A
:1016080006274754110608D51978092747548F1C0F
:101618000131C9B21F700A274754970504D51978B4
:101628004F1C1F7015274754D10504D519784F1C36
:101638001F701A27475498F80570082F01D00E2FED
:1016480008D1197801F1010E83F800E04FF00B0E74
:1016580000F801E0197801F1010E5FFA8EFE4FF0F3
:101668000C0C12F4803F83F800E000F801C009D0A8
:10167800DFF874C102318CF8001054494FF00E0C99
:1016880001F80EC0110308D5197801F1010E83F88D
:1016980000E04FF0190E00F801E0197801F1010E91
:1016A8005FFA8EFE4FF01D0C12F4805F83F800E0A5
:1016B80000F801C009D0DFF830C102318CF8001001
:1016C80042494FF01C0C01F80EC0910608D5197854
:1016D80001F1010E83F800E04FF0070E00F801E079
:1016E800510708D5197801F1010E83F800E04FF091
:1016F800100E00F801E0510308D5197801F1010E28
:1017080083F800E04FF0120E00F801E0520507D50B
:1017180098F8E02222B11A78511C197013218154CB
:10172800182F0DD11A7816218154511CC9B24FF0C7
:10173800170E00F801E0D11C0232D2B2197087549A
:10174800982200212948DFF8C4A0DFF8BC901AF0DD
:101758007FFD10F041F8264B264A1A60264BB8F850
:10176800DC1019802549DFF8A8C000230B808B7096
:1017780023490A60234A1370B8F8542211B2D9F8E1
:1017880000002AF8131000F596704CF82300013376
:10179800122BDFF878E01C4FF1D13BE0CC2E002073
:1017A80035740008016C0008E96B000890C1793DA8
:1017B8005C050020542E0020B0450020D0350020C4
:1017C800703E00208817002035FA8E3CDA2400206D
:1017D800984200200AE81C418842002098240020F2
:1017E800243E002000401C46D92400203C2D002027
:1017F8008C150020F44700208A150020A42400201E
:10180800942400205815002084240020E42D002072
:10181800101500202868C30458BFB8F96012AEF844
:101828000610954901F1500C91F82935FBB991F84A
:101838002B9591F82C35994519D2B9F1000F08D09C
:1018480009F1FF3909EB890909EB890909F5617380
:1018580006E0013303EB830303EB830303F56173B2
:1018680091F82A9509F104099BB22EF81930043130
:101878006145D9D1030740F1658198F84C120829D0
:1018880000F25A81DFE811F009000C00130044004F
:10189800650086008600CB002A0145F2F05201E07F
:1018A80042F6F822754B1A8010F02AF943E1734B7F
:1018B80042F6F821198072490A23120192FBF3F2C9
:1018C8000023A2F5B06241F823200133122BFAD18C
:1018D8006C4A6D4911606D4A402013700FF0A6F8EC
:1018E8008146002800F0288115F07EFF98F84D32D7
:1018F80099F900E0002B0CBF0622072200280CBF34
:1019080001230323019200938046614B614AA9E0B9
:101918005A4B42F6F8221A805A4B5F4A1A605B4BC0
:10192800102240201A700FF081F88046002800F03D
:10193800038115F059FF002200280CBF012303235F
:1019480098F900E00192009380464FF4E133534A3E
:1019580088E04A4B42F6F8221A804A4B504A1A60ED
:101968004A4B082240201A700FF060F88046002881
:1019780000F0E28015F038FF002200280CBF012398
:10198800032398F900E00192009380464FF4E13375
:10199800444A67E0394BDFF83091DFF83081DFF8EF
:1019A80030C1DFF830E1404842F6F8221A80374A61
:1019B8000C23137006294FF0000289F8002088F8DC
:1019C80000208CF8002009D01B220370374B8EF8BA
:1019D800002005221A704FF4E13907E00370334BF9
:1019E800DFF8F490197021228EF80020254B304A38
:1019F8001A6040200FF01AF88046002800F09C80FA
:101A080015F0F2FE002200280CBF0123032398F9E9
:101A180000E00192009380464B46264A22E0174B8D
:101A280044F620621A80174B234A1A60234B4FF062
:101A3800000983F80090154B0E2240201A700EF012
:101A4800F5FF8046002877D015F0CEFE1C4A98F99D
:101A580000E048450CBF012303238DE808028046B7
:101A68004FF4E133402170460EF04CFFB8F1000FFF
:101A78005ED0144B18605BE0B0450020260C0020B7
:101A8800B42200205805002045E40008342E002028
:101A9800A086010019E6000809E400081DE5000811
:101AA800F5E30008D5E400088F2400207021002009
:101AB80045D800085DD80008C5E400085D2400206A
:101AC80059E700083C2E0020902400204D210020DA
:101AD8004C2100206F21002090D00300C04B41F220
:101AE8007C521A80BF4BC04A1A60C04B10221A7031
:101AF800BF4B4FF0000883F80080BE4B28224020DF
:101B08001A700EF093FFB8B1032390F90000BA4A97
:101B1800CDF8048000934021B84BDFF850830EF0D5
:101B2800F1FE0121C8F800000AF0BCFAD8F800005C
:101B3800003018BF012028B9082010F0B7FEA94BC3
:101B4800AF4A1A602B68A94A13F4804F04D01221B7
:101B58001170A449AB48086042F20101194003F032
:101B6800010003F4005EA1B19D4944F6206CA1F880
:101B780000C0BEF1000F06D0082111709949DFF8A6
:101B8800F0E2C1F800E020B10C21117095499E489F
:101B9800086011781806A1F1040151705FD54FF063
:101BA8000009DFF8D0829948DFF8CCA288F80190C4
:101BB80015224946C8F80490C8F808901AF048FB5E
:101BC800934BCAF80030484611F008FF3B68C8F844
:101BD8000C3002200EF02AFF18B9802010F066FEA3
:101BE80036E0427998F80130DFF828C249464FF0CC
:101BF8000C0909FB03CE9EF801E0964507D0013396
:101C0800DBB2042B4FF00101F3D9002300E009B146
:101C180088F80130DAF8003098F801201B7890F93C
:101C28000000002B7B4B4FF00C0E0EFB02330CBF59
:101C38000121032100225B788DE8060002210EF0C5
:101C480061FE754B18600028C7D0012011F0C6FE50
:101C5800724B734A1868734B1A6011F0D7FF2B68E0
:101C6800DFF8F08113F4007F58D06F4A936943F08E
:101C78000103936198F81C0010F064FB6B4A4FF065
:101C8800000A10604FF00A0B0222C271012180F88D
:101C980006B080F808A010F0E5FB98F81D0010F0D9
:101CA80051FB0123C37180F806B080F808A05146A3
:101CB8008146C8F8380110F0D5FB5D4BC8F83C31B7
:101CC8008022102308F59E71484610F012FD484600
:101CD80014F0EAFF3B68574A9FED570A3C3B1360F4
:101CE800336843F0100333604FF4C873A8F84031E9
:101CF800524BC8221A8008F0B6FE514BDFED517ADC
:101D080083ED000A20EE270A4F4AFDEEC07A17EE4F
:101D1800903A13804D4B4FF0FF321A604C4BC8F885
:101D280044312B68DFF854A14A4F0026D9038AF8BA
:101D3800006040F1118114F053FA4FF0010940F2AC
:101D48002A32314607F5A4708AF800901AF080FA12
:101D58003549414B48699A6A02434A613F4A1A62C7
:101D6800DE621AA893F825308DF868308DF86990EE
:101D78008DF86B908DF86A6014F024FF182010F02D
:101D8800E1FA1623C7F87404837107F5A4790223CE
:101D9800334FDFF8D4E0C371067257F83620314963
:101DA80072454FEAC60301F1CC0A03D10B4493F8FC
:101DB800D12003E001360A2EEFD100222E2110F0A7
:101DC80015FB294800235AF83310274F81424FEA60
:101DD800C30255D1234B134493F8D00054E000BFFD
:101DE800260C002058050020ADE40008342E002001
:101DF800182400201924002071E6000848E8010092
:101E080079E400089DE400087DE40008A0080020AB
:101E18005548002080E60108184C00200C250020B9
:101E2800DA4700206017002000100240483E0020DA
:101E3800496D0008443E0020DB0FC93E043E0020E7
:101E4800FC3D00200000C8430C3E0020003E00205E
:101E5800A448002080070020A8000020FF6C00088C
:101E680084C40108B8C30108002C014014170020DD
:101E78008DE40008743E0020943E0020184D002098
:101E880001330A2B9FD1002014F098FD3B88B648F7
:101E9800DFF81CA323F45C731B041B0C3B801D237D
:101EA800FB6200264FF0010B02233B850EA93E86FC
:101EB8006023C7F814B00E93ADF83E601096ADF8E5
:101EC8004460ADF84660ADF84860ADF84A60ADF8DA
:101ED8003CB00BF0E7FEBB6943F00803BB617B6CC9
:101EE80043F400437B6450460BF0C9FD1AA80BF07D
:101EF8009BFD9E4B1A9310231C9340F22A33ADF896
:101F0800743080231F934FF4807320931AA94FF4E1
:101F1800005350462393CDF86C901E962196229636
:101F280024960BF08EFDFB68914943F40073FB6027
:101F3800DAF8003043F00203CAF80030FF2288F8CC
:101F480078B4631866520434802C9A70DA70F8D129
:101F580005F0D2FB05F0D0FB2B685A0560D5854FFC
:101F6800854B3A681A6004200EF060FD0421C8F819
:101F78007C040EF031FD814B3A6888F88004082013
:101F88001A600EF053FD7E4B7E4C186008210EF04F
:101F980023FD2C2288F88104002120461AF058F9E4
:101FA8008E2363707C26E0237D25E370267084F8F9
:101FB8002B50754C00212C2220461AF049F98A230F
:101FC8006370A023E370714B3A681A602020267072
:101FD80084F82B500EF02AFD2021C8F884040EF056
:101FE800FBFC88F8880410200EF020FD1021C8F8AA
:101FF8008C040EF0F1FC664B88F890043B221A70B2
:1020080001225A703A221A719F229A711E221A725C
:10201800A4225A7200229A72DA721A7315F0F1FB2E
:102028005C4C2688002E7AD12C2010F08BF90F23D7
:1020380083710E230D210546C3710672C8F89404F6
:1020480010F010FA284610F0A6F9534A138823F026
:1020580040031B041B0C1380138823F038031B0454
:102068001B0C138013889BB243F04003138032206B
:102078009F238DF838308DF839608DF83A608DF8E7
:102088003B6012F053FF28468DF8696010F07EF926
:1020980004220EA91AA814F019FE284610F07BF99C
:1020A8009DF86A309DF869201B0243EA02429DF8B8
:1020B8006B301343394A934217D00CDC384A9342A9
:1020C80015D00132934217D0A2F51A42033A93422F
:1020D80020D120230CE0334A934208D001329342A6
:1020E8000AD0314A934215D101E0402300E0802311
:1020F80023804FF4807302E04FF480732380638061
:10210800A38822881B02A3605343E360012388F855
:10211800983404E0002323806380A360E360E468CC
:10212800002C47D0E40A264600270DF16808A7428C
:1021380008DA3D196D1010224146E80215F09CF9A5
:102148000F2805DC15F05AF9184BF6021E6031E02D
:10215800002358F82320013240F088800133042BF3
:10216800F7D12E462C46E2E7002C0140342C0140E2
:102178001A4D00205C1700203C1600208C16002009
:10218800D81600205C16002090160020F0160020BB
:10219800082E002044050020003800401620C20008
:1021A80017BA20001740EF001720C20008250020AA
:1021B8001C000240674C684AB4F8D8315269674D30
:1021C800013B9BB2052B9EBF012384F8EA3184F8BA
:1021D800DA3194F8EA315343614A13602B68614A53
:1021E80013F4002318BF012313706379052B02BF72
:1021F8005D4B4FF4C8721A800BF047FF5B4BC82247
:102208001A805B4A137843F008031370594A13780D
:1022180023F0020313702A6840F6020313406BB1DF
:10222800554B56491960564B03211970554B0121DE
:102238001970554900230B8054490B80930306D528
:10224800534B06221A71DA7842F00102DA70A36859
:102258002B60504B01221A704F4A137863F07F03AA
:1022680013702FB0BDEC068BBDE8F08F6F1C2546B0
:1022780078E71BB208EE103AB5F9CC31DFED477AB2
:10228800474A09EE103AB5F9D031B8EEC88A08EED7
:10229800903A28EE278AB8EEC99AF8EEE88A002123
:1022A800B0EE480A29EE279A68EEA78A117008F05E
:1022B800DAFBF0EE409AB0EE480A16F0D9FAB0EE22
:1022C800408AB0EE490A08F0CEFBB0EE40AAB0EE64
:1022D800490A16F0CDFAF0EE40AAB0EE680A08F006
:1022E800C2FBB0EE409AB0EE680A16F0C1FA69EE89
:1022F800806A68EE097AF0EE665AEAEEA75A294B28
:1023080029EE896A28EE007AC3ED035AB0EE465AE0
:10231800F1EE6A5AA5EE875AEAEEA67AA5EE867A13
:102328002AEE099A2AEE400A28EE4A8A69EE8A9A23
:1023380083ED009A83ED010AC3ED02AA83ED045AE6
:1023480083ED058A83ED067AC3ED077AC3ED089A13
:10235800FEF7C3BFB0450020CC2E002098240020F3
:1023680040250020EA2C0020A0150020E83D002090
:1023780044160020D8240020A4210020C6470020AD
:10238800882400204005002024400020264000200A
:102398001C4C0020D80E0020914C002035FA8E3CB1
:1023A800FC010020802100202DE9F04FBA4B1B686A
:1023B8009A6ABA4B2DED048B1A80B94B1978A3B0E1
:1023C8000129079304D1B74B1A80B74A12885A805B
:1023D800B64B1A789B46002A01F0AD8112F068FDD1
:1023E800B34B06909B6813B10BF102009847B14BB1
:1023F800B14CD3F8008018F0080F3BD0AF49B04D6E
:10240800888800F10E039BB21C2BAE4BB3F9043045
:102418002CD8AD4A1288520728D50A2293FBF2F22B
:102428002B88D21A92B213B213F1B30FB8BF02F5C8
:10243800B473A64AB8BF1BB2B32B1278C4BFA3F5B6
:10244800B4731BB2170715D594F9D421524212FB65
:1024580003F29F4B1B685B7A12B213FB02F26FF018
:102468001D0392FBF3F303448B8003E00A2293FBE2
:10247800F2F32B80974BB3F90650974B1B685A8998
:1024880095420CDB197AB5F5FA6FBFBFAB1A4B430F
:10249800C2F5FA6193FBF1F1C1F1640100E0642136
:1024A80094F9D431B4F8540294F826C294F82792D7
:1024B800824E5B429BB205930022884BD154854BD8
:1024C80033F912703B1A03F2F31440F2E63A54451A
:1024D8004FEA420E794C10D883EAE37A022AAAEB33
:1024E800E37A0ED0E24502DDCCEB0A0300E00023DC
:1024F800874226F80E3011DB15E0022A4FF4FA7AEB
:10250800F2D1CA45C8BFC9EB0A03BDF814A0D8BFA9
:10251800002313FB0AF38742B38007DA36F80E303C
:102528005B4226F80E300132032AC6D16C4B1E6876
:1025380016F480560ED0B5F57A7F06DBB5F5FA6F3E
:102548002A46A8BF4FF4FA6201E04FF47A72A2F566
:102558007A7214E0584BB3F856128D4206DBB5F583
:10256800FA6F2A46A8BF4FF4FA6200E00A46521AE8
:102578004FF47A735A43C1F5FA61B2FBF1F264235E
:10258800DFF874E192FBF3F101F1010C3EF91170EF
:102598003EF91CE06FF0630CC7EB0E0E0CFB01213B
:1025A80001FB0EF292FBF3F2D3199BB2E380B6B1B2
:1025B8004C4A1268D60012D54B4AD2787AB9A3F59C
:1025C8007A731BB24FF47A721B0393FBF2F3C0F5D4
:1025D800FA6212B2534300EB2330384BD8803A4B9F
:1025E800B3F800A01AF0400F994639D0354BDFED0B
:1025F8003F7AB3F904300A2293FBF2F33C4A12887B
:102608009B1A1BB208EE103AB8EEC88A28EE278A41
:10261800B0EE480A08F027FAF0EE408AB0EE480A11
:1026280016F026F9B4F9023007EE103AB4F9003082
:10263800B8EEC77A06EE903A67EE407AF8EEE66AA8
:10264800E8EEA67A20EE260AFDEEE77AA8EE870ADB
:1026580017EE903AFDEEC07A238017EE903A638029
:1026680018F0140F114F144E00F0AA801AF4027FCC
:1026780000F0A680154B1B7803F0100303F0FF024F
:10268800002B3BD01B4B96F9A422B3F900106388AA
:1026980001FB0233638093E0402200208C24002059
:1026A800CA210020CC21002028210020200C002055
:1026B800CC2E0020542E0020B04500201C250020E0
:1026C800A615002028250020D0240020441600202C
:1026D8000C250020E42D0020F43C00203C2500209F
:1026E80098240020D4240020A424002035FA8E3C0D
:1026F800A81500203C3E0020D22C0020964B97497C
:102708001B68DFF8A8E2D8789B7870B3BEF90000A0
:10271800C0EB050C8CEAEC7EAEEBEC7E9E450DDD45
:10272800DFF88CE28542CEF800204FF001023A71C2
:10273800C8BF5B42E2889BB2134440E03B7933B1A7
:10274800874B3A71D3F800E0864BC3F800E0864B1C
:102758001B681844854B1A681388528898422EDBE8
:1027680082421346A8BF034629E0BEF900E0CEEB3B
:10277800050282EAE27CACEBE27C9C4509DD02239F
:1027880092FBF3F27A4B1A607A4A012313703B7179
:1027980008E03B7933B1724B38711A68714B1A6093
:1027A800744B1870704B1B689E44704B1A681388E2
:1027B80052889E4503DB72451346A8BF7346CB80FB
:1027C8006D4B1B78ABB1B6F85632AB4211DB6B4B95
:1027D8005B79012B01D0192B02D196F89F2242B9BF
:1027E8000E2B06D0082B04D00023A380644B0022B4
:1027F8009A6096F8145295B31AF0030F2FD0614BD4
:10280800DFED617A93ED080AB4EEE70AF1EE10FA0B
:1028180021D917F075FC5D4BD3ED007A20EE270A1D
:1028280017F0DCFBB0F5617FA8BF4FF4617007EECD
:10283800900AB8EEE77ADFED567A87EE270A16F0A7
:1028480017F807EE905AF8EEE77A27EE800A17F0A5
:10285800C5FB00B200E00020E3881844E08096F849
:102868005A324C4A23B9B9F80010002900F0A48064
:102878001278002A4FD0022B09D0032B19D196F8D1
:102888005B32C3EB431203EB8203DB000FE0424BE6
:10289800D3F8F820B2F57A7F05DB44F6206393423B
:1028A800A8BF134601E04FF47A7303F57A739BB21D
:1028B80000E0FB88394A1068394AB3FBF0F0127817
:1028C800451C2DB2092A3D8105D1364A218811803F
:1028D80061885180D380B7F90A90DFF880A000237F
:1028E800314F3AF913C007F1140E07F10C083EF8FE
:1028F800132038F913102EF813C0C2EB0C0201FB99
:1029080009F191FBF5F10A4428F813200133042B4F
:10291800E6D1788102E07B89013B7B81224AB2F9CA
:102928000A0000284FF0000314DD0C4FB2F90850DC
:102938000C32DFF880E032F913103EF813E041431F
:1029480091FBF5F1C1EB0E0127F813100133042BAD
:10295800EFD136E0538134E0A01700201C25002079
:10296800041700202C3E00203C3E0020A417002025
:10297800303E0020403E00209C000020B045002052
:1029880010250020404200208FC2753C941700207B
:10299800EFB6B044101600200002002040250020A9
:1029A800CA210020CC210020200C00201216002073
:1029B800383E0020340C002013787981002B00F079
:1029C8009D80C34B93F85C3223B1C24A12689100D0
:1029D80001F1F884C04BC1481968079BC04D1F78A6
:1029E800C04BDFF858C31B689FEDBF5A93F800E04F
:1029F800DFEDBE4A9FEDBE4ADFEDBE3A9FEDBE3A1F
:102A0800DFF83C83F7EE005A0C1D0022F0EE652A31
:102A1800022A14BF91F800A091F801A03CF91230E5
:102A280007EE10AAB8EEC77A06EE903AC7EE057A16
:102A380014BF8B784B7A4FEA4209B0EE007AF4EE75
:102A4800C77AF1EE10FAF8EEE66AC4BF37EEC77A35
:102A5800E7EE247A86EE847AB5EEC07AF1EE10FAC3
:102A6800D4BFF1EE476AF0EE476AE5EC016A8BB134
:102A780006EE103AB8EEC66A86EE052A26EEA66A73
:102A880066EE866A35EEC26A66EE876A26EE077AD1
:102A9800A2EE267A14F8013F67EEA37A67EE877AEA
:102AA800002B41F0E3840C2F02BFBDEEE77A17EE4E
:102AB800103A29F80830BEF1000F41F0FF849FED6D
:102AC8008F7A67EE877A9FED8E7AF4EEC77AF1EE09
:102AD80010FA01F105859FED8B7AF4EE477AF1EE55
:102AE80010FAC8BFF0EE477A0132032AC0ED007A27
:102AF80000F104008CD1844B00221A70834B1B68B0
:102B08009F0640F19B80824B1B8803F03003002B0B
:102B180000F094807F4B1B78DD0740F18F807E4B5F
:102B2800DFED7E7AB3F90430DFF81892DFF8188207
:102B38000A2293FBF2F308EE103AB8EEC88AF2EED6
:102B4800048A28EE278AB0EE480A15F091FEB0EE06
:102B5800409AB0EE480A07F086FF714B1B6893F85D
:102B680003A0B0EE408ABAF1000F43D06D4FB9F917
:102B78000200B7F90240001B10F0ECFFCAF1000593
:102B8800A84203DB5045A8BF504600E02846204431
:102B980003B2B7F90040B9F900000593BDF8143045
:102BA8007B80001B10F0D6FF854203DC824555462A
:102BB800A8BF0546DDED057A25442DB2B8EEE77AC3
:102BC80007EE905AF8EEE77A3D8027EEC96A68EE7C
:102BD800277AA8EE076AE9EE077AC6EE286A87EE32
:102BE800A87AFDEEE66AFDEEC77A16EE903AA8F8E6
:102BF80000301FE0B9F9023007EE103AB9F9003099
:102C080000EE103AB8EEC00AB8EEC77A60EE496A2C
:102C1800E8EE076A28EE008AC6EEA87AA9EE078AC7
:102C2800FDEEE77A17EE903AC8EE287AA8F8003059
:102C3800FDEEE77A17EE903AA8F802303A4B18788A
:102C4800002840F06B85394F3B681C0340F16685CE
:102C5800374C2378033B052B1CD81D4B354D93F877
:102C6800D53533B1012B08D114F0E0FAC0F17F005B
:102C780003E0686A03689B689847AB6A95F82C205C
:102C88001344B3F5807FA8BF4FF480738342D4BF49
:102C9800AB62A8622378023B092B00F2A784DFE825
:102CA80013F00A0055008600A600BB00D300E5001B
:102CB8005604780488040023CBF82830CBF8303049
:102CC8001D4B1B68CBF83430032300F08EBC00BFCB
:102CD800B0450020D4240020F43C0020102500201A
:102CE800642C00200C2500200000C842D7A36841AE
:102CF8000000FA43000048430AD7233C333383409B
:102D080000F0FFC500F0FF4510160020542E0020EB
:102D1800D0240020441600202825002035FA8E3CB7
:102D280060170020B6150020784C00209824002059
:102D3800EA2C0020200C0020842400201C250020E0
:102D4800CC210020BA15002024250020994B9A4D4B
:102D58001A686B6B6433934280F04884402015F006
:102D680049FA002840F04284DFF850924FF04008BA
:102D78002E462B6B19F8030058B115F015FBB36AF2
:102D8800013BB362336BB8F1010803F1010333630C
:102D9800EFD12A6B8949884B8A5C002A40F0268447
:102DA8001A634FF0FF325A63042300F01EBC844AB2
:102DB8000292A2F10C0301932A2300935021A2F15D
:102DC8000A034920163A09F0F5FD002840F00E8460
:102DD8003B6813F08002784B4FF0FF3119BF18633E
:102DE80059631A63596314BF05230723FDE30223BC
:102DF8000093744B002102910191A3F1080248202D
:102E080009F0D8FD002840F0F1836B4B4FF0FF32FA
:102E180018635A630623E8E36B4A0292A2F10C0393
:102E2800072501930095A2F108030021143A4720D1
:102E380009F0C0FD002840F0D9835F4B25704FF0A2
:102E4800FF3218635A63D1E3052300935F4B0021D7
:102E580002910191A3F10802532009F0ABFD00286B
:102E680040F0C483544B18630823BEE3402015F098
:102E7800C1F9002840F0BA834F4D2B6B492B01F262
:102E88003383DFE813F04A004D0052005600590022
:102E9800600065006A006E0072007E0089008C0088
:102EA800D300D700DC00E100F000FF000E011D0197
:102EB8002C013B014A0159016C0176018301900103
:102EC8009D01AA01B701C401D101DE01E801F501A4
:102ED800FF01090213021D02270231023B024502CB
:102EE8004F0259026302B702C102CB02D502DF02C8
:102EF800E902EE02F302F802FD02020309031203DB
:102F08001F03240329032E03330338033D0342031D
:102F180047034C03510356035B032D492D4810E327
:102F28002D4B2E4A2E492F4833E02F4A2F4930483F
:102F3800B8E23049304804E3304B314893F8D4259F
:102F480093F8D315AEE22D4B2E48B3F8CC10F8E227
:102F58002A4B2D48B3F8CE10F3E22C4B2C481969B4
:102F6800EFE22C4B2C481989EBE2AB6BD90404D562
:102F7800224B2A4893F81612E3E20F4B0B221A63EE
:102F8800E1E21E49264891F8193291F81B2291F87E
:102F98001A1215F0E3FAD6E2A98F2248D1E23B686B
:102FA8001A0540F1D082154B1F48B3F91E22B3F819
:102FB800201277E284240020200C0020B0C50108EC
:102FC80026C6010810C801082CC8010874C80108E1
:102FD800FCEE010808EF010819EF010824EF0108C9
:102FE8002CEF010832EF01085AEF010863EF0108DE
:102FF8006FEF0108924B002083EF0108B0450020D5
:1030080091EF0108A2EF0108B1EF0108CC2E0020D2
:10301800C0EF0108442E0020D0EF0108DAEF0108C4
:10302800E7EF010800F001080BF00108CC4BCD4890
:10303800596986E2CC4BCD4893F8DA1181E2CA4B44
:10304800CB4893F8EA117CE296F82825C9486C2306
:103058005343F2180C2192F8282401FB02331E4432
:1030680096F82A146DE296F82825C3486C23534332
:10307800F2180C2192F8282401FB02331E4496F81A
:103088002C145EE296F82825BC486C235343F218AA
:103098000C2192F8282401FB02331E4496F82B14C5
:1030A8004FE296F82825B6486C235343F2180C21B2
:1030B80092F8282401FB02331E4496F8331440E2A8
:1030C80096F82825AF486C235343F2180C2192F840
:1030D800282401FB02331E4496F82D1431E296F899
:1030E8002825A9486C235343F2180C2192F8282468
:1030F80001FB02331E4496F82E1422E296F8282586
:10310800A2486C235343F2180C2192F8282401FB9F
:1031180002331E4496F8321413E296F828259C4888
:103128006C235343F2180C2192F8282401FB023334
:103138001E44B6F8341404E296F8282595486C2302
:103148005343F2180C2192F8282401FB02331E4441
:1031580096F8313496F8302496F82F1419E7824BF4
:103168008D4893F828256C2101FB023393F8E4136A
:10317800E7E196F8283589486C2202FB036696F841
:10318800F93396F8EF2396F8E51302E796F8283511
:1031980083486C2202FB036696F8FA3396F8F0230C
:1031A80096F8E613F5E696F828357E486C2202FB79
:1031B800036696F8FB3396F8F12396F8E713E8E6EA
:1031C80096F8283578486C2202FB036696F8FC339B
:1031D80096F8F22396F8E813DBE696F82835734854
:1031E8006C2202FB036696F8FD3396F8F32396F8F3
:1031F800E913CEE696F828356D486C2202FB036683
:1032080096F8FE3396F8F42396F8EA13C1E696F892
:10321800283568486C2202FB036696F8FF3396F857
:10322800F52396F8EB13B4E696F8283562486C2235
:1032380002FB036696F8003496F8F62396F8EC132A
:10324800A7E6494B5D4893F828256C2101FB02331A
:1032580093F8ED1375E196F8283559486C2202FB6E
:10326800036696F8023496F8F82396F8EE1390E67B
:103278003D4B544893F828256C2101FB023393F801
:1032880003145EE1384B504893F828256C2101FB64
:103298000233B3F8041454E1334B4C4893F828250F
:1032A8006C2101FB0233B3F806144AE12E4B48485F
:1032B80093F828256C2101FB0233B3F8081440E188
:1032C800294B444893F828256C2101FB0233B3F8B5
:1032D8000A1436E1244B404893F828256C2101FB59
:1032E800023393F80C142CE11F4B3C4893F8282523
:1032F8006C2101FB0233B3F80E1422E11A4B384853
:1033080093F828256C2101FB0233B3F8101418E157
:10331800154B344893F828256C2101FB0233B3F888
:1033280012140EE1104B304893F828256C2101FB4C
:10333800023393F8161404E10B4B2C4893F8282514
:103348006C2101FB023393F81714FAE0064B284866
:1033580093F828256C2101FB023393F81814F0E048
:10336800CC2E00201EF00108B04500202AF00108EC
:103378003DF0010852F001085CF0010866F0010810
:1033880073F0010880F001088AF0010895F001083F
:10339800A2F00108B4F00108C3F00108D4F0010854
:1033A800E5F00108F7F0010807F1010817F1010835
:1033B80027F1010838F1010849F101085BF101081A
:1033C8004BF1010865F101087AF101088AF1010859
:1033D80098F10108AAF10108C0F10108CFF101082C
:1033E800EBF1010801F2010810F2010827F20108C7
:1033F80040F20108A34BA44893F828256C2101FB4F
:10340800023393F819149CE09E4BA04893F82825A2
:103418006C2101FB023393F81A1492E0994B9C48F3
:1034280093F828256C2101FB023393F81B1488E0DC
:10343800944B984893F828256C2101FB0233B3F884
:103448001C147EE08F4B944893F828256C2101FBCF
:103458000233B3F81E1474E08A4B904893F826128E
:103468006FE0884B8E4893F827126AE0854B8D48A9
:10347800B3F8D81165E0834B8B4893F8DB1160E013
:10348800804B8A4893F8DC115BE07E4B8848B3F8A0
:10349800E221B3F8DE1105E07A4B8648B3F8E4215F
:1034A800B3F8E01115F05AF84DE0764B9FED827AAB
:1034B800D3ED7E7A814867EE877AFDEEE77A17EEDC
:1034C800901A3EE06F4B7E4893F8D51139E06D4B6A
:1034D8007C4893F8EE1134E06A4B7B4893F8ED1181
:1034E8002FE0684B794893F899122AE0654B7848A1
:1034F80093F85A1225E0634B764893F85B1220E064
:10350800604B7548B3F85E121BE05E4B734893F846
:103518004C1216E05B4B724893F8E31011E0594BDC
:10352800704893F8E2100CE0564B6F48B3F8DE1081
:1035380007E0544B6D4893F8EB1102E0514B6C488F
:10354800996815F00BF82B6B01332B634EE0694B30
:103558001B689B011AD5684DB5F84030B3B9674B65
:10356800D5F844801E68452014F01EFF0E2014F084
:103578001BFF404614F0D2FF304614F0CFFF4FF443
:103588008053EB870A23237008F0E6FE09F0F0F970
:103598002CE0594B93F84820002AF5D0554A126878
:1035A8009601F1D493F84930002BEDD1092323700B
:1035B800ECE7534B504D1A686B6BC833934204D2F7
:1035C800304B93F8D5657EB904E014F059FE002815
:1035D800F6D10BE0686A0DF080F995F84A306E6212
:1035E800022B01D10EF0F8F80123237014F032FEFB
:1035F80058B101232370404B93F84920002A00F06A
:103608008D80002283F8492088E01E4B93F8D62548
:103618001946002A00F082803B68DD044FF000065E
:103628004CBFB1F8DA20B1F8D020364D334635F921
:1036380013000133904218BF46F001060C2BF6D157
:103648002F4B2D4D1B6826B103F59C530833EB64B3
:1036580002E0EA6C9A4257D92378012B5ED195F89B
:103668004930002B5AD191F8D5352BB113F0C8FB4E
:10367800012385F8493051E080200EF0A5F8002894
:103688004CD1F3E7B045002054F2010869F2010873
:103698007FF2010896F20108ABF20108C1F20108B5
:1036A800BDF20108CDF20108D9F20108EBF20108D8
:1036B800FEF2010812F301080000C8422AF30108CB
:1036C80038F3010848F3010859F3010869F30108C0
:1036D80082F3010896F30108B3F30108D0F3010857
:1036E800E5F30108FAF301080FF4010821F40108D1
:1036F8002FF40108D4240020200C0020E03D0020F5
:10370800842400202C4C00202378012B06D095F827
:1037180049301BB109F0FEF985F84960B84B1B78B0
:10372800072B05D111F0C4FB069BC01AB54B588076
:10373800B54B00221A70B54C13A863689847A14688
:10374800002800F04981B24DBDF94C302B60BDF91D
:103758004E306B60BDF95030AB60AE4BDFF8F48291
:103768001A78294628460AF0A3FCAB4B1A889A46D1
:10377800002A00F0A580A94BDFEDA98A1B681B78F9
:10378800002608EE103AA8F14807A8F13C04304694
:103798004FF47A71D9F81430B1FBF3F3C3EB43114A
:1037A80003EB8103BAF800E0DB009BB29E4508BF3B
:1037B80038603B6808BF20611A4655F826301A441D
:1037C80055F826303A6007EE903A23690133012B09
:1037D8004FEA8601F8EEE77A236106D1C4ED017A53
:1037E800C4ED007AC4ED028A1BE0D4ED005A07EE5E
:1037F800103A37EEE56AF8EEC76A86EE267AD4ED17
:10380800026A37EE257A77EEC77A84ED017AE6EE1A
:10381800276A84ED007AF0EE667AC4ED036AC4ED97
:10382800026ABEF1010F685048F8010035D12369DA
:103838000690012BC3BF03F1FF3307EE903A94EDD6
:10384800037A9FED770A0591C4BFF8EEE77A87EE11
:10385800270A16F0C7FE0599069818EE103A4BB1DC
:10386800F8EEC87AF4EEC07AF1EE10FA02D50AF052
:103878000CFC25E04FF47A72D9F81430B2FBF3F35C
:10388800C3EB431203EB8203DB003A689BB202EB03
:10389800530292FBF3F248F801200136032E07F198
:1038A800040704F114047FF473AFBAF80000012888
:1038B80001D10DF0A7F9BAF80030013BAAF80030A1
:1038C800002355F8231058F82300514A091A45F8DF
:1038D80023100133032BF4D1524F534B397800296D
:1038E80068D0DFF81C81DFF81C911C46151F0026E4
:1038F800C24698F80030032B04BF6B6829F81630CD
:103908004A4B1B78012B0AD1D5ED017A484B1C2074
:10391800B8EEE70A00FB063015F05EF81AE073B956
:10392800444BD5ED017AD3ED000A434B39780C208E
:10393800B8EEE70A00FB063015F008F90AE0D5ED05
:10394800017A3E4B4FF4F870B8EEE70A00FB0630F8
:1039580014F0EEFF84ED000A9AF80030082B05D128
:1039680094ED000A16F03AFB29F81600344B1B8830
:103978004BB1344B94ED000A1C2000FB063015F0C7
:103988002BF884ED000A304B1B884BB12F4B94ED7C
:10399800000A1C2000FB063015F01EF884ED000A12
:1039A800B4EC010A16F01AFB0136032E45F8040F91
:1039B8009FD111E0D2ED007AF8EEE77AC3ED007AF4
:1039C800D2ED017AF8EEE77AC3ED017AD2ED027A08
:1039D800F8EEE77AC3ED027A0B4A92F8C83023B1C1
:1039E800013B82F8C83000F08ABD194B93F8DC21FE
:1039F8001D468AB393F8EA31013BDBB22DE000BFE4
:103A0800CA210020CC210020200C0020CC2E002030
:103A180030250020D83500207221002058170020BA
:103A280000000000E42E00204C2C0020E82E00208E
:103A3800EC2E0020402F0020C40C0020442F002032
:103A4800E62E00201C350020143500207435002097
:103A5800B0450020B80C002001238BF8C83011F0C5
:103A680027FAB74BB74C1F68B74BB5F83612A3F116
:103A7800520206462068B847B44B1A78072A1D46F2
:103A880004D111F015FAB24B801B988011F010FA8E
:103A980095F800A00590BAF1010F0AD1AD49DBF8FD
:103AA800CC30AB4A0968CBF8CC00C31A93805B1AB8
:103AB800D380A94B22681B68EBB192F83320CAB1B6
:103AC800A64A1268940718D5A54A1178012914D96D
:103AD800DB78A44859430088CB1A98420AB203DB22
:103AE80088420346A8BF0B461BB2120392FBF3F2AF
:103AF800012305E013461A4602E001234FF48052E1
:103B08009949C9780D912BB1BDF954105143091346
:103B1800ADF854109549964E91F800809549DFF814
:103B28003092B1F902000890B1F90000099092486A
:103B3800B1F90410D0F800C006910025294628469E
:103B480040453DD29CF90040069FD6ED016A96EDAE
:103B5800026A64427C4307EE904AB8EEE77ADDEDEC
:103B6800097AF8EEE77A0DF1540E67EEA67ADDEDE4
:103B7800086AF8EEE66AE6EE867AD6ED036AE7EEBC
:103B8800267AFDEEE77ACDED077ABDF91C400BB138
:103B9800544324132EF8104015AC34F910408C42CD
:103BA80003DCA542A8BF254600E02146BAF1050F6F
:103BB80003D1042898BF29F8104001301036BFE718
:103BC800664B6E4C1868491B10F4805209B240D0FD
:103BD8006B4B6C4D1B78DFF8B4E16B4F13F0040F9F
:103BE80001BF2B681E8A694BA3F89061B4F906607F
:103BF800674C2B6824681B8AE588C5EB030C66456F
:103C080008DCB4F900303C68AEF89061B4F90040C3
:103C180035440AE02B449E4209DB3B68B4F9024074
:103C2800B3F90230AEF89061751B2DB219E0BEF9F8
:103C380090319C45ABBFB4F900303B683C68B4F99F
:103C48000240ABBFB4F90040B3F902301D46254627
:103C580007E04D4BB4F906501B68B3F90040B3F9BF
:103C680002304A4E9BB2A4B2C4EB030A0FFA8AFA96
:103C780051451ADD4FEA0A33002793FBF1F1C6F8E4
:103C88009411B8450AD915AB33F917E001FB0EFEBC
:103C98004FEA2E3E23F817E00137F2E702239AFB9A
:103CA800F3F31C4424B20A9407E0022791FBF7F1CE
:103CB8005B1A0C441BB224B20A93B6F99031324E07
:103CC8000C9337682E4E2F4B36783149DFF8C4E015
:103CD8001B680968DFF8C09006F00406F6B207967C
:103CE80000F01000BEF906600B964FF0000B0E9026
:103CF800D84540F2898015A807EE905A30F81BC0C5
:103D08001B4800EB0B1090ED007AF8EEE77AA64618
:103D180067EE877AFDEEE77A17EE900AA04204DB99
:103D28000A9E8642A8BF0646B6460CEB0E000D9EBC
:103D380000B229F8020F8EB3B7F804E042E000BFE2
:103D4800A00000200C250020F4470020CA210020F4
:103D5800CC21002040250020A42100209824002008
:103D680040050020F4210020A42400203F25002045
:103D7800F00C0020A42B0020701700201C25002028
:103D8800D824002074170020B4410020200C002003
:103D9800B0410020E42D00207A40002082B1B3F821
:103DA80010E0B1F806C00C9ECCEB0E0E764504DC94
:103DB800B7F800E0B1F800C006E0B1F802E001E0B1
:103DC800B7F800E0B7F802C0704503DB8445E64663
:103DD800A8BF86460E98A9F800E090B1079880B170
:103DE8007AB9119210910F930CF0E6FE0F9B10997F
:103DF800119A30B9588A0B9E8642BCBFB888A9F878
:103E080000000BF1010B73E73C894CB3A0494FF458
:103E18007A700968B0FBF1F1B4FBF1F1012905D919
:103E280042F210708142A8BF014600E0022109B2A7
:103E38008A4515DD974D98483C8835F918E000EB20
:103E48004807A645B7F9987103DB7C187445A8BFE5
:103E5800744624B200EB480025F81840A0F89841B1
:103E6800079919B90E468D488A4906E08A4991F89A
:103E7800B001192800F2478107E0B045F6D930F8BB
:103E8800164021F816400136F7E7012101FA00F043
:103E980083490140002900F0368182490988C80514
:103EA80008D5814B1A88ADF86C205A88ADF86E2079
:103EB8009B8812E0BDF82410ADF86C10BDF82010F6
:103EC800ADF86E10BDF81810ADF870103AB11B8A35
:103ED8000B9A9A4203DA069B5B42ADF8703073483E
:103EE800B0F902304FF47A7203F5E1634FF461617F
:103EF800534393FBF1F3A3F5FA73ADF88430B0F9AB
:103F0800003003F5E1635A43624B92FBF1F21B88E0
:103F1800A3F2DC53ADF87230654BA2F5FA72ADF836
:103F280086201B68634A1B8A1188C91AADF8741069
:103F38005188C91AADF876109188C91AADF8781069
:103F4800D188C91AADF87A101189C91AADF87C1050
:103F58005189C91AADF87E109189D289C91AD31A24
:103F6800ADF88230544AADF880100023194622F883
:103F780013100133082BFAD1504A514B126806929C
:103F8800504A1B78126850490792072202FB031314
:103F98004E4DDFF824A10A934FF064084FF0010951
:103FA8000A9B8B4200F094800B782BB11533069A4C
:103FB80009FA03F3134067D011F806EC079B11F9CF
:103FC800010C11F805CCCEEBCE0703EB47074FEAFF
:103FD8004C06B7F90230B7F9002009909A1A92B244
:103FE80011F9023C11F8030C4FEA520B534393FBAF
:103FF800F8F3CBEB03031BB2089328B922A80644B5
:1040080036F81C0C288019E022AB1E44B5F9004094
:1040180036F91C6CB44208DA2044844203DC864238
:104028003446A8BF04462C8008E007DD201AB042B9
:1040380003DB8442A8BF044626462E80D7F80A0030
:1040480011F9046C089B09FA0CFC10EA0C0FB5F97D
:1040580000000CBF01244FF0FF3416FB00F090FB6A
:10406800F8F0984209DB099B534393FBF8F3CBEB39
:1040780003031BB28342A8BF03463AF81EB004FBF1
:1040880003B32AF81E3000E02B800235073187E79A
:10409800402500207C400020200C00202C4C0020D3
:1040A80032413003D02400201C2500202825002080
:1040B80074170020E42D0020F80E0020D4240020DE
:1040C800B841002030420020BF410020D20D00201E
:1040D800AD4BAE4ED3F8008000254FF00E09642793
:1040E80009FB0583E8B293F9064036F9023F14FB51
:1040F80003F494FBF7F4348010F02EFD01352044CE
:10410800082D3080ECD1A24C9F4D236813F0200F6E
:1041180033D0002010F020FD9E4E0746308001204D
:1041280010F01AFD9C4B70801B68190625D59B4B17
:104138009B4A1B681B78012B24D1D5F80080B2F963
:10414800021098F90630B2F900205B424B434FF059
:10415800320C93FBFCF31FFA83FE98F914306FF0CE
:10416800310113FB02F393FBF1F17144791A93FBCC
:10417800FCF373443180184470802B68834A03F140
:1041880070061AE0D5F800E0B2F902309EF9061080
:1041980011FB03F1322391FBF3F1394431809EF98D
:1041A8001470B2F9001017FB01F292FBF3F21044FD
:1041B800E2E70E339E4211800CD032F9020FB3F9B8
:1041C8000010B3F902708842F3DB87423946A8BF72
:1041D8000146EEE7734B744E1A6892F904209A462A
:1041E800A2B996F8B0717B1E182B00F29980DFE80F
:1041F80003F0549797709797976997979797977B36
:104208009797979797708997977B5400DFF884B1B1
:104218000023A6F8D231B046D946B6F9D271072F95
:10422800DFDC98F8D421614B92B9DAF800200693C4
:10423800528800EE102A5E4A1C20116800FB0730E5
:10424800B8EE400A14F052FC0122069B88F8D421EB
:104258003BF9172000EE102A1C2000FB0730B8EEAF
:10426800C00A14F0B9FB15F0B9FE2A6800B2C7EB12
:10427800C7032BF8170002EB4303B3F90020B3F987
:104288000230904203DB8342A8BF03461A4629F84E
:1042980017200137A6F8D271BFE7DAF800305B784B
:1042A8001BB13C4B0020598908E0424B1B7803F0B6
:1042B800040303F0FF01002BF3D1084607F06CFF5D
:1042C80001252EE0334D0020E98807F065FF298994
:1042D80005E0304D0020298907F05EFF698901203B
:1042E80007F05AFF02251CE0DFF8A8800225A81E67
:1042F80038F81510C0B2013507F04EFF082DF6D179
:1043080006250EE0DFF88C800325E81E38F8151026
:10431800C0B2013507F040FF072DF6D1042500E0B3
:10432800002523689A0601D4052F0BD1194F28467A
:10433800398807F031FF681C7988C0B207F02CFF74
:104348000235EDB22368DB0205D496F8B83273B1B2
:1043580010F05AFB0BE0184F0024281937F8021FF9
:10436800C0B207F019FF0D2CEFD00134F5E7134B5D
:104378001B78072B05D110F09BFD059BC01A104B2D
:10438800D88001233370BAE030420020F60E0020B6
:1043980098240020F80E0020D42400206C17002058
:1043A8002825002070170020200C0020F80D002080
:1043B80040250020D8240020EA2D0020CA21002012
:1043C800CC210020504A128852063EF503AB4F4FCD
:1043D8004F4D3A7F9A4214D007EE903A9FED4D8A9E
:1043E8003B77F8EEE77A27EE888AB0EE480A06F0BF
:1043F8003AFB85ED000AB0EE480A14F039FA87ED69
:10440800080AB4F90030DBED085A95ED006A424A13
:1044180007EE903AB4F9043006EE903AF8EEE66A00
:10442800F8EEE77A25EEE67AA7EE867A67EEA57AC1
:10443800BDEEC77AE6EE267A17EE103AB3F5FA7FA4
:10444800A8BF4FF4FA739342FDEEE77AB8BF13465C
:10445800238017EE903AB3F5FA7FA8BF4FF4FA73AA
:104468009342B8BF1346A380FEF7B4BA06EE903A5B
:10447800F8EEE66AB5EEC07A86EE856AF1EE10FAD5
:10448800D8BFB1EE477AF0EE656AE6EE476AF4EE19
:10449800C36AF1EE10FAB0EE667A07D4F4EE656AF4
:1044A800F1EE10FAC8BFB0EE657A01E09FED1B7A15
:1044B800C2EE876A67EEA67AFEF7F5BA9FED187A1C
:1044C800F4EEC77AF1EE10FA0AD49FED167AF4EEFC
:1044D800C77AF1EE10FAC8BFF0EE477AFEF704BBD0
:1044E800F0EE477AFEF700BB13F0CAFE00283FF44F
:1044F8007DA84FF48053EB870A23FFF776B823B0E3
:10450800BDEC048BBDE8F08FD0240020200C0020E7
:104518000000002035FA8E3C0CFEFFFF0AD7233C32
:1045280000C0F9C400C0F9442DE9F04F914BADB07B
:104538001D780093002D00F0A7808F4B1868002885
:1045480002F097800EF076F9DFF85C92DFF85C8273
:10455800D9F8000007F0B2FD002802F08A80D9F8E7
:104568000000864C07F0A7FD092801D03F2855D147
:104578004FF0000A2668574655460AEB080B36B135
:1045880032465AF808107E4817F0A7FE20B90DB138
:104598005F4601E05D465F460AF1100ABAF5147FEE
:1045A800EBD1F5B1D5F800A0D7F800B0DFF8D0C14D
:1045B80023681AF803001BF80310814211D15A1C12
:1045C800DFF8BCE149B92D2B07D86C4802602020E0
:1045D8000EF803000EF8021003E00CF80300226046
:1045E800E6E723680BB1BD420FD0664813F020FC04
:1045F800BD4207D855F8100B13F01AFC092013F028
:1046080079FAF5E70CF034FE00265D4D23689E42EA
:104618009ED2A85D13F06EFA0136F7E723686BB9EE
:10462800042804D1564813F0E1FC02F022B80C2803
:1046380042F01B80544813F0FBFB22E00C28F9D011
:104648000A2841F0C6874E4E504813F0F1FB23214B
:10465800304617F034FE354608B1801B20602368C9
:104668000022002B41F0B987002A41F0D18730227F
:104678000021434817F0ECFD009B1B78002B01F04C
:10468800F8870CF0F5FD63E7414B03F13007414B28
:10469800EA18EB58002B01F019813F493F4C0B6099
:1046A8000593002322608DF819303D4A3D48049255
:1046B80014238DF8183004AB0360264689469246C9
:1046C800D9F80000DFF8D08007F0F8FC002801F0E6
:1046D800E980D8F8000007F0EEFC336893F848103A
:1046E800834619B9242863D101221DE0012903D189
:1046F8004D2808BF022204E0022907D13C2808BF40
:10470800032218BF002283F8482085E003290ED130
:1047180040284FF0000102D983F84810D0E75871BB
:104728001971D9719871042283F84820C8E70429BF
:1047380007D1997983F8490080EA01029A71052224
:10474800F2E7052968D1587919798842987908D902
:104758008BEA00009871481C18710B4483F808B064
:10476800AEE7584503D1062283F848205AE00022D4
:10477800DAE700BF784C0020284C0020744C002059
:10478800444C002050F5010855F501085D0D02085C
:1047980094C801083C2D002000250020F8240020A2
:1047A800D1C00008FC240020144C002000EC0108B3
:1047B800DC490B7803F0040303F0FF0E002B7FF4B1
:1047C8007FAF23281DD1009AD8F80000019101235A
:1047D8001370D54B1860D54B1860D54B5860102016
:1047E8001872D448C3F800A0036083F809E0D248DF
:1047F80013F01EFB0CF03CFD01990B7843F002030B
:104808000B70CE4B1B681B785B4505D1CC4BCD4A52
:104818001A60CD4BCD4ADA60336893F84820062AEF
:104828007FF44EAF93F84980B8F15A0F00F0B28781
:1048380000F2FC80B8F1360F00F0B68674D8B8F1F3
:10484800240F00F0E8852DD8B8F1040F00F0788225
:1048580015D8B8F1020F00F0588200F26582B8F15D
:10486800010F40F0FF8703200AF0DEFC00200AF069
:1048780096FC40460AF093FC152000F0F0BFB8F112
:104888000A0F00F09A82B8F1220F00F03A84B8F1CA
:10489800050F40F0E7871A200AF0C6FC0026DFF86B
:1048A800C4825DE2B8F12C0F00F0E3851BD8B8F1A3
:1048B800280F00F0C585B8F12A0F00F0D485B8F1AB
:1048C800260F40F0CF87A24E06200AF0ADFCB6F8BE
:1048D800C8010AF0ACFCB6F8CC010AF0A8FCB6F89E
:1048E800D00100F0ABBFB8F1300F00F089860BD8CB
:1048F800B8F12E0F40F0B687954E40200AF094FC90
:1049080006F1400800F06CBEB8F1320F00F01A86CC
:10491800B8F1340F40F0A6878D4E5A200AF084FC77
:1049280006F15A0800F00EBCB8F1460F00F0C88630
:104938002AD8B8F13D0F00F07B8311D8B8F13A0FAF
:1049480000F04B83B8F13B0F00F0D483B8F1380F77
:1049580040F0888704200AF067FC7D4E00F061BDB6
:10496800B8F1420F00F0FF85B8F1450F00F0DC8682
:10497800B8F1400F40F0768708200AF055FC002671
:10498800DFF8CC8100F0E5BDB8F14D0F00F0B78538
:104998002BD8B8F1490F00F05783B8F14B0F00F04E
:1049A8009385B8F1470F40F05D870AF0EFFB0646A4
:1049B80084200AF039FC30460AF042FC654BDA687C
:1049C80006F1800393428CBFC6EB02094FF08009C1
:1049D8000DF1300812F012FD4A463046414612F0F9
:1049E8004BFD0026814600F07FBEB8F1500F00F065
:1049F800848611D8B8F14F0F40F034870B200AF0A5
:104A080013FC00200AF0CBFB00200AF0C8FB0020B2
:104A18000AF0C5FB00F095BEB8F1520F00F07F8692
:104A2800B8F1540F00F07B8600F01CBFB8F1720F8C
:104A380000F0F18300F2C780B8F1680F00F06682D9
:104A480000F29480B8F1640F00F0A78139D8B8F16A
:104A58005E0F00F0BE86B8F1600F00F0F286B8F184
:104A68005C0F40F0FF863A4EDFF8FC8011200AF018
:104A7800DBFB96F8DC010AF092FBD8F80030188CC2
:104A88000AF0D5FBD8F80030588C0AF0D0FBB6F8FD
:104A9800DE010AF0CCFBB6F8E0010AF0C8FBD8F852
:104AA8000030988C0AF0C3FBD8F80030D88C0AF094
:104AB800BEFBB6F8E2010AF0BAFBB6F8E40100F072
:104AC800BDBEB8F1660F00F08A8100F2B5810B20F7
:104AD8000AF0AAFB204B18880AF0A9FB1F4B18887C
:104AE80080B20AF0A4FB1E4B1B68C3F3C000C3F3DB
:104AF8008002800040EA4200C3F340021043C3F33F
:104B0800401240EAC20003F0100318430AF08FFB7A
:104B18000AF072FA0AF094FB0D4B93F8280500F09E
:104B28009EBE00BFD8240020144C00201C17002073
:104B3800DC0E0020284C002080F50108A84B00203E
:104B4800FC9F0020EFBEADDE00ED00E00400FA059A
:104B5800B0450020440500208C2400208A24002031
:104B6800542E002063EF01080C250020B8F16C0FCB
:104B780000F0E68112D8B8F16A0F00F08E8300F2D7
:104B8800D383DFF81084DFF8109498F80000400011
:104B980000F0FE000AF048FB0026C6E1B8F16E0FEF
:104BA80000F02082C0F00E82B8F16F0F00F0528240
:104BB800B8F1700F40F056861E200AF035FB00262B
:104BC800DFF8D88378E2B8F17D0F00F0C18529D8E5
:104BD800B8F1760F00F0B9830AD8B8F1740F00F075
:104BE8008F8040F24F832F200AF01EFBDC4E79E2C3
:104BF800B8F1780F00F02F81C0F0ED82B8F17C0F8A
:104C080040F03086D74E06200AF00EFBB6F8D600E4
:104C18000AF00DFBB6F8D8000AF009FBB6F8DA007E
:104C280000F00CBEB8F1A00F00F0E7833FD8B8F150
:104C38007F0F00F0F284C0F09E85B8F1960F40F027
:104C480011860F200AF0F0FAC74B18880AF0EFFA1D
:104C5800C64B188880B20AF0EAFAC54B1B68C3F342
:104C6800C000C3F38002800040EA4200C3F3400260
:104C78001043C3F3401240EAC20003F01003184384
:104C88000AF0D5FA0AF0B8F90AF0DAFAB54B93F84F
:104C980028050AF084FAB74B18886428A8BF64204E
:104CA8000AF0C5FA03200AF07AFAB34B27E2B8F102
:104CB800F00F00F0978314D8B8F1A40F40F0D28514
:104CC800DFF8DC8298F82F0080000130C0B20AF0CB
:104CD800ABFA98F82F000AF062FA002608F1300AB9
:104CE8005CE3B8F1F10F00F0EA80B8F1FE0F40F094
:104CF800B98508200AF098FA0026DFF8A88269E347
:104D08004FF000094FF0010B42E204200AF08CFA40
:104D1800DFF89482002618F8060001360AF03FFAF8
:104D2800042EF8D100F0B8BD03200AF07DFA032064
:104D38000AF035FA00200AF032FA012000F08FBD9F
:104D480006200AF071FADFF86482002618F80600D7
:104D580001360AF024FA042EF8D1002000F06EBDC6
:104D680018F8060001360AF01AFA0B2EF8D1DFF807
:104D78004082002618F8060001360AF010FA082EBC
:104D8800F8D1DFF83082002618F8060001360AF05C
:104D980006FA072EF8D100F07FBD07200AF044FA82
:104DA800E7200AF0FCF96F4B58790AF0F8F900206F
:104DB8000AF0F5F9042000F0C8BC7048704E13F0F2
:104DC800F1FE5FFA80F840460AF02EFAB044B0458A
:104DD80000F0628516F8010F0AF0E1F9F7E71220F2
:104DE8000AF022FA674BDFF8D0911B89B3F5007FF0
:104DF80094BF4FF001084FF00408002659F8260028
:104E080090FBF8F0013680B20AF011FA032EF5D1C2
:104E18005D4E30880AF00BFAB0880AF008FA30893B
:104E28005A4E0AF004FA30880AF001FAB0880AF0FB
:104E3800FEF9308900F002BD10200AF0F5F9DFF81C
:104E48007C81002618F8060001360AF0A8F9102E11
:104E5800F8D100F021BD7020424E0AF0E5F94FF07C
:104E6800000AB0464FF00E09B6F854010AF0DFF90F
:104E7800B6F856010AF0DBF9B6F858010AF0D7F986
:104E880096F85A010AF08BF996F85B010AF087F94F
:104E980096F85C010AF083F996F85D010AF07FF94B
:104EA80009FB0A830AF1010AD3F85E010AF0C8F97E
:104EB800BAF1080F06F10E06D6D100F0EDBC70204D
:104EC800284E0AF0B1F906F1700896F8E4000AF0E5
:104ED80066F996F8E5000AF062F996F8E6000AF035
:104EE8005EF996F8E7000AF05AF996F8E8000AF031
:104EF80056F996F8E9000AF052F9073696F8E300F1
:104F08000AF04DF9B045E0D100F0C6BC10200AF017
:104F18008BF9DFF8AC80002618F8060001360AF095
:104F28003EF9102EF8D100F0B7BC98F800309E4238
:104F380080F0B28439F816000AF079F90136F4E7FE
:104F4800134E06200AF070F930880AF070F970885C
:104F58000AF06DF9B6F904300A2093FBF0F061E02D
:104F680093C80108B04500208C2400208A24002022
:104F7800542E0020282100208E240020924B00204F
:104F8800914B0020442E002030250020543E002064
:104F980028250020342E0020E42D00200C25002098
:104FA800DC0E0020CC210020B8F50108BDF5010871
:104FB8005AEF010824EF010820160020F80E0020FF
:104FC8007C40002006200AF02FF9C34B18680AF02D
:104FD80037F9C24B188800F031BC04200AF024F9D4
:104FE800BF4B16E207200AF01FF9BE4B1888FF28AE
:104FF800A8BFFF20C0B20AF0D2F8BB4B186880F3F4
:10500800100080B20AF013F9B84B18880AF00FF9AB
:10501800B74B93F82322B74B186832B10A23584389
:1050280080F3100080B200F009BC00F30F00F9E72C
:10503800AF4E02200AF0F8F896F89B020AF0AFF893
:1050480096F89A0200F00BBC02200AF0EDF8AA4B81
:10505800988AF3E3A94E0C200AF0E6F8336818782A
:105068000AF09DF8336898780AF099F84FF000092B
:10507800B046D8F80030A14E4B4409F101095879DF
:105088000AF08DF8B9F1030FF3D13368187A0AF0F2
:1050980086F83368D8780AF082F8336818790AF005
:1050A8007EF8336858890AF0C2F83368587A0AF0EB
:1050B80076F833685878D2E3D8F800303344587813
:1050C8000AF06DF8D8F800303344D87A0AF067F857
:1050D800D8F8003033440136587D0AF060F80A2EBB
:1050E800EAD1D9E316F8010F002800F0D5830AF0B9
:1050F80056F8F7E701200AF097F8814B1B681878F3
:10510800ADE350207A4E0AF08FF806F150084FF0C0
:105118000C097C4A96F8293509FB0323043693F8D1
:1051280038000AF03CF896F826050AF038F896F8A0
:1051380027050AF034F896F828050AF030F8B04543
:10514800E7D1A9E396F87E050AF029F896F87905DB
:105158000AF025F896F87A050AF021F896F87B0502
:105168000AF01DF896F87C050AF019F8063696F844
:1051780077050AF014F8B045E4D18DE3BBF1000FD0
:1051880000F08A835FFA89F00AF04EF84FF0000BBE
:1051980000265D4B1B789E42F0DA5C4BF05C0021E8
:1051A8004FF00C0E0EFB01F313F807C0844503D033
:1051B80001311F29F6D10CE0524A1344D3F834A028
:1051C800504613F0EFFC0146BBF1000F00F084835A
:1051D80089440136DDE7DFF83081DFF830A198F83F
:1051E8000000DFF820910AF01FF8002698F8003038
:1051F8009E4280F0518316F80A1000220C2000FB12
:1052080002F313F807E08E4500F0738301321F2A7A
:10521800F5D10136EAE7364E16200AF005F8B6F859
:1052280054020AF004F8B6F8CC000AF000F8B6F810
:10523800CE0009F0FCFFB6F8D00009F0F8FFB6F888
:10524800AC0209F0F4FF96F8A50209F0A8FF0020C7
:1052580009F0A5FF96F8A60209F0A1FF96F8230227
:1052680009F09DFF96F8500209F099FF002009F017
:1052780096FFB6F9F0310A2093FBF0F080B209F0FE
:10528800D6FFCEE0082009F0CFFF0126F0B20136A4
:1052980009F085FF092EF9D1FEE2102009F0C4FFBC
:1052A8001B4B1C4E187800F0020009F078FF1A4BCF
:1052B800187809F074FF306809F0C2FF706809F0C7
:1052C800BFFF164B188809F0B2FF154B188809F074
:1052D800AEFF144B988DB1E2041700202C16002065
:1052E800003E0020F4210020A8210020C44D002009
:1052F800B045002040160020CC2E0020F43C0020B1
:105308000C25002094C80108D9240020DA240020A4
:10531800441600204C1600204A160020481600208B
:1053280046160020DC0E0020052009F07DFFD54B35
:10533800188809F07CFFD44B188809F078FFD34B04
:1053480093F82E0000F0010089E209F009FF814678
:10535800122009F069FFB9F1000F01D1CC4B03E02D
:10536800B9F1100F04D1CB4BD3F800805E6801E08F
:105378000026B046484609F012FF404609F060FF93
:10538800304609F05DFFC44B186809F059FF00204A
:1053980009F04DFF002009F04AFFC3E198F82F30CB
:1053A8009E4280F07982DFF80C931AF8060009F023
:1053B800F6FE19F8060009F0F2FE09F1100309F1EA
:1053C8002009985D09F0EBFE19F8060009F0E7FEE0
:1053D8000136E3E738F81600013609F028FF042EF5
:1053E800F8D159E2AD4E042009F01EFFB6F8F401D9
:1053F80009F01DFFB6F8F20120E20C2009F014FFB5
:10540800A74B186809F01CFFA64B186809F018FF8D
:10541800A54B186899E1042009F006FF9F4B98688E
:1054280093E196F8160209F0BAFE96F81A0209F006
:10543800B6FE96F8190209F0B2FE96F81B020EE2C3
:10544800964E072009F0F0FEB6F81E0209F0EFFEAE
:10545800B6F8200209F0EBFE96F8220209F09FFE4A
:10546800B6F82402EAE1012009F0DEFE8B4B5879F8
:10547800F5E18A4E102009F0D7FE96F84C0209F0A3
:105488008EFEB6F8580209F0D2FEB6F8540209F0BA
:10549800CEFEB6F8560209F0CAFE96F84E0209F09A
:1054A8007EFEB6F8600209F0C2FEB6F8620209F0A4
:1054B800BEFE96F85A0209F072FE96F85B0209F0F1
:1054C8006EFEB6F85E02B9E1744E082009F0ACFE33
:1054D80096F8AA0209F063FE96F8AB0209F05FFE9F
:1054E800B6F8AC0209F0A3FE96F8AE0209F057FE32
:1054F800B6F8B00209F09BFE96F8B202AFE16B4E27
:10550800DFF8B481307800EB4000C0B209F08CFEBF
:105518004FF000093378994508F1020880F0BC8102
:1055280018F8020C09F03BFE18F8010C00EB80009B
:1055380000EB800000F2EE2080B209F078FE09F15D
:105548000109E7E7012009F06FFE544B93F8500278
:1055580085E106EB0803013693F8440209F01FFEC3
:10556800082EF6D198E14D4E102009F05DFE7079B5
:1055780009F015FEB06809F063FE96F84C0209F0D0
:105588000EFEB6F8C80109F052FEB6F8CC0109F0D3
:105598004EFEB6F8D00109F04AFEB6F81E0209F030
:1055A80046FEB6F8200249E1384B3C4E93F87000AD
:1055B800DFF80891C0EBC000C0B209F035FE06F173
:1055C800280896F9B602002313F90920824200F050
:1055D80096810C333C2BF7D10836B045F1D15BE10D
:1055E800B6F8740309F023FE96F8760309F0D7FDA0
:1055F800043696F8730309F0D2FDB045F0D14BE1BB
:1056080080202B4E09F010FE06F1800856F8040F92
:1056180009F016FE4645F9D13EE18D2009F004FE59
:1056280000264FF0060A0AFB06F94FF0000B5FFA56
:1056380086F8404609F0B3FD5FFA8BF009F0AFFD3C
:10564800164B0BEB090119440BF1010B91F8B4034C
:1056580009F0A5FDBBF1060FEBD10136062EE2D10C
:105668000026062009F09BFDF0B209F098FD0B4BCF
:105678003344013693F8D80309F091FD0B2EF0D18D
:105688000AE100BFBC160020BE160020DC0E002078
:1056980008170020AC1500202C3E0020B045002043
:1056A800ACF7FF1FB0F7FF1FB4F7FF1F342E002021
:1056B800A04800201C0F002014480020AC4B0020FC
:1056C8000D2009F0B1FD11F0C1FDD04E40F00200EF
:1056D800C0B209F064FD308809F0B2FDF06809F045
:1056E800AFFD11F093FD30E04E4580F2D58018F8FB
:1056F800060009F054FD0136F6E7C54E042009F00E
:1057080093FD012009F04BFD96F8D50509F047FDFA
:1057180096F8D30509F043FD96F8D4059FE00120DB
:1057280009F082FD00209AE0132009F07DFDDFF8E2
:105738000083002618F80600013609F030FD0B2E0C
:10574800F8D1002009F07CFD002009F079FDA3E0E4
:10575800AF4E052009F068FD96F8260209F01FFDF6
:1057680096F8270209F01BFD96F8280209F017FDA4
:10577800B6F8DC0062E0A64E032009F055FD96F865
:10578800C50109F00CFD96F8C60109F008FD96F868
:10579800C70164E09E4E062009F046FDB6F8D831F0
:1057A80023B1082009F0FBFC012005E096F8DA0196
:1057B80009F0F5FC96F8EA0109F0F1FC96F8E30027
:1057C80009F0EDFC96F8E20009F0E9FCB6F8DE0015
:1057D80034E0904E112009F027FD3368588D09F008
:1057E80026FD3368988D09F022FD3368D88D09F0BD
:1057F8001EFD336893F8280009F0D1FC336893F84C
:10580800330009F0CCFC336893F8360009F0C7FC84
:10581800336893F8370009F0C2FC002009F0BFFC98
:10582800002009F0BCFC336893F8350009F0B7FC98
:105838003368588F09F0FBFC3368188F09F0F7FCC0
:105848002AE0734E032009F0EFFC96F8D50109F021
:10585800A6FC96F8EE0109F0A2FC96F8ED0109F015
:105868009EFC19E0B8F15D0F61D040F29880B8F164
:10587800D20F40F0188309F073FC020600F10B8385
:10588800654B1B785B0704D4032828BF00200DF064
:10589800D1F8002009F0C8FC09F092FC2368002226
:1058A80083F848205D4B5E4C18680CF0C3FF94F8F1
:1058B80071305BB15B4B58590BF004F80FF01FFBCC
:1058C800002384F87130584B584ADA604C35982DCB
:1058D8007EF4DDAE00F0CDBED046CAEB08008842AB
:1058E800BFF677AC18F8010B019109F058FC019943
:1058F800F3E74B4493F8380009F051FC89E4C0B24F
:1059080009F04DFCB6F8B80209F091FC96F8BA0215
:1059180009F045FC96F8BB0209F041FC96F8BD0277
:1059280009F03DFC96F8BC0209F039FC54E609F090
:1059380017FCDFF8E080364ED8F8009086F8DC01D6
:1059480009F01AFCA9F82000D8F8009009F014FC16
:105958002368A9F822005B79052B13D909F00CFC00
:10596800A6F8DE0109F008FCD8F80090A6F8E001D6
:1059780009F002FCA9F82400D8F8008009F0FCFB23
:10598800A8F8260023685B790D2B82D909F0F4FB6F
:10599800A6F8E20109F0F0FBA6F8E40179E7B8F10E
:1059A800370F47D15B794FF00708B3FBF8F8C8EB1E
:1059B800C8029B1A13F0FF0F02D00CF00FFC68E727
:1059C8005FFA88F808F1FF385FFA88F8B8F1FF0F36
:1059D8003FF45FAF09F0C4FB4FFA80F948460AF07C
:1059E800E7FF06460028E8D080F8009009F0C4FBDD
:1059F800708009F0B5FB307109F0B2FB707109F0E5
:105A0800AFFBF07109F0ACFBB071DBE74405002097
:105A1800B04500200C250020D8240020FC240020BC
:105A2800DC0E00203C2D002000ED00E00400FA050B
:105A380063EF010800F23D81B8F12B0F2AD109F07C
:105A48008FFBC64B24E0B8F14E0F71D109F088FBEB
:105A580011280646B1D8DFF8048309F081FB06F562
:105A6800987608EB4603187109F086FB40F2ED239F
:105A78009842424640F30C8240F6CA039842A8BFB7
:105A8800184602EB4603A0F2EE20192290FBF2F032
:105A98005871FEE675D8B8F1250F08D1AF4E00232E
:105AA800B36009F073FBB3681843B060F1E642D8FD
:105AB800B8F10B0F19D111220021A948DFF89C92E7
:105AC80016F0C6FB4FF0000833685B79102B28BF2F
:105AD80010239845BFF4DDAE09F042FB08EB09033B
:105AE80008F1010883F8E205EEE7B8F1230F1FD1AA
:105AF80009F036FB132806463FF65FAF09F030FB86
:105B080000220C2101FB02F307EB030E9EF808E0CC
:105B1800864500F0398501321F2AF3D14DE7B8F1E7
:105B2800FA0F40F003858F4B1B785A0740F16983C1
:105B38000CF054FBB0E6B8F1270F0DD109F01CFBAF
:105B4800864EC6F8C80109F017FBC6F8CC0109F063
:105B580013FBC6F8D0019CE6B8F1290FE8D109F08B
:105B68000BFB7E4EA6F81E0209F006FBA6F82002E3
:105B780009F0F6FA86F8220209F0FEFAA6F82402DD
:105B880087E6B8F1310F14D109F0EAFA1F28064662
:105B98003FF613AF23685B79052B7FF40EAF09F04E
:105BA800F5FA6E4B03EB8603C3F8F40210F018FB0A
:105BB8006FE64BD8B8F12D0F32D109F0D1FA674E04
:105BC80086F84C0209F0D8FAA6F8580209F0D4FA77
:105BD800A6F8540209F0D0FAA6F8560209F0C0FA5D
:105BE800236886F84E025B79082B07D909F0C4FAB6
:105BF800A6F8600209F0C0FAA6F8620223685B7989
:105C08000C2B7FF646AE09F0ABFA86F85A0209F07B
:105C1800A7FA86F85B0209F0AFFAA6F85E0238E642
:105C2800B8F12F0F84D14D4E06F1400809F0A4FABF
:105C3800A6F8740309F094FA86F8760309F090FA46
:105C4800043686F873034645F0D122E6B8F1330FDF
:105C580005D109F085FA414B83F8500219E6B8F1ED
:105C6800350F7FF465AF09F07BFA0E2880463FF6C2
:105C7800A4AE09F075FA03283FF69FAE374B062607
:105C880006FB083686F87E0509F06AFA86F8790573
:105C980009F066FA86F87A0509F062FA86F87B0553
:105CA80009F05EFA86F87C0509F05AFA86F87D054F
:105CB800EFE5B8F1440F04D12B4B012283F8712092
:105CC800E7E500F28380B8F13E0F09D109F048FA00
:105CD800224E86F89B0209F043FA86F89A02D8E524
:105CE8002BD8B8F1390F11D109F03AFA1B4E86F8C2
:105CF800160209F035FA86F81A0209F031FA86F820
:105D0800190209F02DFA86F81B02C2E5B8F13C0F1A
:105D18007FF40EAF154ED6F8008009F021FA01285D
:105D2800A8BF012088F8000033681B78012B104BAE
:105D380014BF104A104A1A60ABE5B8F1410F1DD1E3
:105D4800DFF81880002609F00BFA06EB0803013685
:105D5800082E83F84402F6D19BE500BFB045002029
:105D6800924B0020D8240020DC0E00200C250020B7
:105D7800A0000020B7FE0008D9010108B8F1430FC0
:105D88007FF4D6AECB4E09F0EBF90023B360707107
:105D980009F0FCF9B3681843B06009F0E1F986F836
:105DA8004C0209F0E9F9C6F8C80109F0E5F9C6F8A6
:105DB800CC0109F0E1F9C6F8D00109F0DDF9A6F83F
:105DC8001E0209F0D9F9A6F8200262E5B8F14C0FD5
:105DD80019D109F0C5F9B74E86F8AA0209F0C0F939
:105DE80086F8AB0209F0C8F9A6F8AC0209F0B8F9D0
:105DF80086F8AE0209F0C0F9A6F8B00209F0B0F9C9
:105E080086F8B20245E513D8B8F1480F09D111F068
:105E18005DFBA94A00231370A84A1370A84A1360AF
:105E280037E5B8F14A0F7FF483AE09F0A5F930E5FC
:105E3800B8F1510F12D1A34B1B78012B3FF629ADB6
:105E480009F08EF99B4E86F8D50509F089F986F890
:105E5800D30509F085F986F8D4051AE5B8F15B0F82
:105E68007FF4F1AD09F07CF9924E86F8DA0109F079
:105E780077F986F8EA0109F073F986F8E30009F082
:105E88006FF986F8E20009F077F9A6F8DE0000E578
:105E980040F2EE20F5E500F07F00032828BF00203F
:105EA8000CF00CFDF5E400F2F481B8F1CC0F52D1FE
:105EB8005B79092B7FF681AD834ED6F8008009F017
:105EC8004FF988F80000D6F8008009F049F988F8F9
:105ED800020009F045F933686428A8BF64205871A6
:105EE80009F03EF933686428A8BF6420987109F066
:105EF80037F93368FF28A8BFFF20D87109F030F9B7
:105F0800D6F80080642828BF642088F8080009F0C3
:105F180027F988F80300D6F8008009F021F988F8F5
:105F28000400D6F8008009F027F92368A8F80A00C9
:105F38005B790A2B05D9D6F8008009F011F988F8A1
:105F4800090023685B790B2B7FF6A3AC366809F050
:105F580007F970709DE400F2EE80B8F1C80F28D1FF
:105F68005E797608122E3FF628AD4FF00008B0454E
:105F780007D209F001F90CAB23F8180008F1010861
:105F8800F5E75249324600239E4206DD0CA830F858
:105F9800130021F813000133F6E74C4B0021122AB5
:105FA80003D023F812100132F9E7494B01221A7085
:105FB8006FE454D8B8F15F0F3FD1464ED6F8008051
:105FC80009F0DAF8A8F82A00D6F8008009F0D4F821
:105FD800A8F82C00D6F8008009F0CEF8A8F82E0012
:105FE800D6F8008009F0BCF888F82800D6F80080B8
:105FF80009F0B6F888F83300D6F8008009F0B0F850
:1060080088F83600D6F8008009F0AAF888F8370032
:1060180009F0A6F809F0A4F8D6F8008009F0A0F86D
:1060280088F83500D6F8008009F0A6F8A8F83A00F4
:10603800366809F0A1F830872BE4B8F1610F7FF4D6
:1060480077AD09F08DF81B4E86F8D50109F088F870
:1060580086F8EE0109F084F886F8ED0119E4B8F144
:10606800C90F45D109F07CF81B4B1A7810B142F0E2
:10607800020201E022F002021A7009F071F8174BCF
:10608800174E187009F082F8306009F07FF87060D8
:1060980009F072F8134B188009F06EF8124B134A86
:1060A800188092F82E3043F0020382F82E30FFF762
:1060B800F0BB00BFB04500200425002005250020C6
:1060C80008250020EA2C0020F43C0020142300209E
:1060D8001D4000200C250020441600204A160020F0
:1060E8004C1600204816002046160020DC0E002022
:1060F800B8F1CA0F7FF41CADCC4E4FF00008D6F8AB
:10610800009009F02DF8C14489F80100D6F80090F4
:1061180009F026F8C14489F80B00D6F8009009F078
:106128001FF8C14408F10108B8F10A0F89F81500F1
:10613800E5D1FFF7AEBBB8F1CF0F39D109F01CF8A4
:106148006FF4AF6E00EB0E039BB2B94EC62B98BF2F
:10615800A6F8540209F010F8A6F8CC0009F00CF8DB
:10616800A6F8CE0009F008F8A6F8D00009F004F85F
:10617800A6F8AC0208F0F4FF86F8A50208F0F0FFD4
:1061880008F0EEFF86F8A60208F0EAFF86F8230278
:1061980008F0E6FF86F8500208F0E2FF08F0ECFF8E
:1061A80000EB80004000A6F8F00108F0D9FF9EE55A
:1061B8001DD8B8F1CD0F0AD19E4B1B7858073FF573
:1061C80068AB9D4B4FF4C8721A80FFF762BBB8F1F9
:1061D800CE0F7FF4ADAC974B1B7859073FF559AB01
:1061E800964A137843F004031370FFF752BBB8F1D3
:1061F800D00F0CD18F4B1B785E073FF54AAB04F0EC
:10620800E7F90CF07BFB03F0AFFDFFF742BBB8F1F9
:10621800D10F7FF48DAC08F0A3FF824608F0B6FFDB
:10622800814608F0B3FF804608F0B0FF064608F044
:10623800A3FF08F0A1FF08F093FFBAF1000F13D1F4
:106248007F4B1020C3F80090C3F804800CF00EFBBD
:106258007A4A137843F001031370002E3FF419AB08
:10626800784B1E60FFF715BBBAF1100F7FF411AB26
:10627800754BC3F80090C3F804800EB1714B1E60D3
:106288007249734B0222081F1A700DF075FCFFF754
:1062980000BBB8F1DB0F05D1644B186803F024FF8D
:1062A800FFF7F7BA75D8B8F1D60F0BD1DFF8A88188
:1062B800002608F061FF28F816000136082EF8D1EC
:1062C800FFF7E7BA3CD8B8F1D30F05D108F054FF6F
:1062D800604B1880FFF7DDBAB8F1D40F7FF428AC13
:1062E8005B790F2B7FF469AB08F03AFF07288046EB
:1062F8003FF663AB08F040FF4D4B0E2606FB083611
:10630800A6F8540108F038FFA6F8560108F034FF43
:10631800A6F8580108F024FF86F85A0108F020FF73
:1063280086F85B0108F01CFF86F85C0108F018FF8E
:1063380086F85D0108F02AFFC6F85E01FFF7A9BAE2
:10634800B8F1D90F0ED108F017FF394EA6F8D600CC
:1063580008F012FFA6F8D80008F00EFFA6F8DA0039
:10636800FFF797BAB8F1DA0F7FF4E2AB08F0F8FE5E
:106378002F4E86F8260208F0F3FE86F8270208F06A
:10638800EFFE86F8280208F0F7FEA6F8DC00FFF713
:1063980080BAB8F1EF0F0AD108F0EEFE244EA6F845
:1063A800F40108F0E9FEA6F8F201FFF772BA55D831
:1063B800B8F1DC0F0ED108F0D3FE1D4E86F8C501EA
:1063C80008F0CEFE86F8C60108F0CAFE86F8C701B6
:1063D800FFF75FBAB8F1DD0F7FF4AAAB08F0C0FE93
:1063E800804608F0BDFE064608F0BAFE0F283FF6C4
:1063F8009FABB8F1050F0BD8052E3FF699AB0C4BA8
:10640800062101FB0832931983F8B403FFF741BA58
:10641800B8F1060F7FF48CAB0A2E3FF689AB044B1C
:10642800334483F8D803FFF734BA00BF0C250020A3
:10643800B0450020D8240020A015002044160020D4
:10644800081700202C3E0020AC150020B0150020B5
:10645800AA150020A61500202C4C0020B8F1F50F35
:106468007FF45DAB012008F0DFFE0026824BDFF8E9
:1064780040A282481E70314630228AF80060DFF858
:1064880034B2DFF8F89115F0E3FE8DF80F607C4E1A
:10649800D0469DF80F3096F876209A4232D99DF86A
:1064A8000F3006EBC30393F87930DB0723D59DF84B
:1064B8000F3006EBC30393F878303BF91330002B09
:1064C80019DD9DF80F3006EBC303DB6F18790BF06D
:1064D80039FF98F80030202149F823000BF0C2FF5B
:1064E80098F8003059F823000BF055FF98F8003061
:1064F800013388F800309DF80F300133DBB28DF896
:106508000F30C6E79AF8000008F049FE08F058FE78
:106518005C4B18680CF08EF9236818680AF0D2F9F9
:10652800236818680EF014FEFFF7B3B9B8F1F20F3C
:106538007FF4FEAA08F014FE0F2806463FF63DAA8F
:1065480008F00EFE504BC6EBC6061E4486F8E40063
:1065580008F006FE86F8E50008F002FE86F8E60078
:1065680008F0FEFD86F8E70008F0FAFD86F8E80076
:1065780008F0F6FD86F8E90008F0F2FD86F8EA0072
:106588000EF0C2FAFFF785B9404ADFF8FC801344E1
:1065980006F5A57608EB860693F83030737008F098
:1065A800DFFDB07008F0DCFDF07008F0D9FD384B65
:1065B80038491A68307108F1CC030B60364B00205B
:1065C8001A6010F0CEFB354B80F001001870FFF711
:1065D80060B90D2828D1FEF736B8591E685C202806
:1065E80019D101220B46FEF73CB81035B5F5147FDA
:1065F80016D055F808102A4805EB080609F082F964
:106608000028F2D0274B9E420AD2F368984700230D
:106618002360FEF72CB802B123600025F554E8E7A3
:10662800214811F005FCF2E77F2809D1013B1C4AFB
:106638001E4823600021D15411F0FAFBFDF788BFF2
:106648002F2B3DF685AFA0F12002D2B25E2A3DF68F
:106658007FAF13B920283DF47BAF5A1C2260104A43
:10666800D05411F047FAFDF773BF7F28EBD1FDF73F
:106678006FBF2DB0BDE8F08F64050020FC2C002012
:10668800DC0E0020FC240020B045002094C801083E
:106698000C25002050170020541700209C000020D3
:1066A800444C002050EE010860F501087CF5010813
:1066B8007B4200207C400020426A806A131A5842BC
:1066C800584170474171704743799B070AD5436A1F
:1066D8008269D154436A01690133B3FBF1F201FBCA
:1066E800123343627047427902F0020202F0FF035C
:1066F80042B10369426A806A013BDBB2101A23EA9D
:106708000000704718467047437913F001031FBF14
:10671800C369026A9A1AC3681ABF03F1FF3302EA0F
:10672800030018467047437913F0010310B501467A
:106738000DD0FFF7E9FF58B10B6A4A69CC68D05C05
:106748000133B3FBF4F204FB12330B6210BD18469D
:1067580010BD90F8433230B583B990F8423290F8C2
:10676800411201248B4209D2B0F8482204FA03F5F9
:106778002A430133A0F84822DBB2F3E730BD704763
:106788002DE9F74F6A4CDFF8ACE10091DEF80030F4
:106798002188B4F90280C1EB231252434900C1EBAE
:1067A800E3011313B4F90420534308FB01F89B13C6
:1067B80003EBE82303EB83028032B3F5FA384FEAA0
:1067C80022224FEAE37949F1FF390192B4F908200E
:1067D800A361A8FB08AB08FB09F30BEB430B02FB17
:1067E80009F1D31708FB0311A2FB08230B441F036D
:1067F800160347EA1257B4F90A2002FB0BF1D31724
:106808000AFB03130546A2FB0A011944020A42EADD
:10681800016292194FEA2123E6887B41003243F551
:106828000043A2FB060106FB03114A10CB1752EAEC
:10683800030170D0B4F9100000FB0BF6C1170AFB76
:106848000166A0FB0A013144B4F90E6006FB09FC9D
:10685800F71708FB07C7A6FB0889B9444FEA484A57
:106868004FEA494B1AEB000A4BEAD83B4BEB010BBA
:10687800DEF80410B4F90C80C1F5801E7646F717CF
:1068880000264FEACE70F90716EB0A064FEAC8074A
:1068980041EA5E0147EB0B0740F6354E861B61EB7C
:1068A8000707A6FB0E010EFB071112F025FEB4F92F
:1068B80016204E13470B47EAC14702FB06FED317C3
:1068C80007FB03EEA2FB07237344564307FB03664B
:1068D800A2FB07233344560E46EAC3163218B4F90E
:1068E80014604FEA636747EB01037143F71700FB36
:1068F8000717A6FB00013944C60C46EA4136B6180C
:106908004FEAE147B4F912005F41330A43EA0763EB
:106918000201134400E000230DB11B0A2B60009B09
:1069280013B11A46019B136003B0BDE8F08F00BF96
:10693800AC2E0020B40F002070472DE9F043334AF5
:10694800334C138965892689B4F90490B4F9027027
:10695800B4F90EE0B4F90080B4F920C05D1B7543AA
:10696800EB13B4F91250EE02B4F914501D4496FB1F
:10697800F5F50A261D44E5616E43A5F57A6505FB24
:1069880005F36F4305FB09F5B4F90C901B1303FBE2
:106998000EFEFF1203FB09F31B1407EBEE2E03EBAD
:1069A80065350EEB8808E388D468023508FA0CF8D8
:1069B800AD1008F102084CF25032A4EBA80405F51A
:1069C800004542FA0CF26B4362434FEAD33547BFA6
:1069D800B2FBF5F35B005400B4FBF5F31A12524313
:1069E80040F6DE3505FB02F40A4A02FB03F52214E1
:1069F80002EB2542083602F6CF62361103EB22136A
:106A080000B1036001B10E60BDE8F083B40F00204F
:106A18005C2E002043E3FFFF6B4B6C4A2DE9F04FDF
:106A28005E891469B3F804804FEA062AB4EB0A0AAF
:106A38001C894FF000054FF0000B65EB0B0BA4FB16
:106A48000A6704FB0B77F40944EA47644FEA0846EF
:106A580014EB06084FEAE715DC884FF0000745EB12
:106A6800070987B0A4FB0A67CDE90489B3F8028057
:106A780004FB0B77340A44EA07644FEAC83614EB80
:106A880006089C894FEA27254FF0000745EB0709C0
:106A9800A4FB0A6704FB0B77F40D44EA472414F5BA
:106AA800FA664FEAE75545F10007B6F5FA6F77F150
:106AB8000003CDE90089CDE90267964667DA052625
:106AC800A4FB062306FB053302FB05F604FB03665D
:106AD800DDE90489A2FB042333445F104FEA320640
:106AE800B8EB06084FEA920669EB070946EA83768F
:106AF8009F10DDE90023921B63EB0703DDE90267C2
:106B0800CDE90023324A4FF0FF33964277EB030377
:106B1800CDE9048928DA40F6AC52A4184FF00003F6
:106B28005D4104FB05F3A4FB044505EB43056FF049
:106B38000602664202FB0566A4FB0223334418EBF7
:106B4800020649EB0307CDE904670B26A4FB0623DD
:106B580006FB0533DDE900455B104FEA3202A41A53
:106B680065EB0305CDE900450AFB0BF3DDE90245BA
:106B7800AAFB0AAB0BEB430B4FEADA7242EA4B0271
:106B8800A41A4FEAEB7365EB0305CDE90245DEF87D
:106B98001440009B019DA4FB032304FB0533560D01
:106BA80046EAC3265F15DDE90434F31A67EB0404EB
:106BB800DB0B43EA444300B1036009B1029B0B605D
:106BC80007B0BDE8F08F00BF982E0020B40F00205A
:106BD80024FAFFFF014B01221A767047B40F0020F8
:106BE800044B1A7E02F0FF0012B100221A7601202F
:106BF800704700BFB40F002037B5104B04465D68DE
:106C080018786A460621A847A8B19DF800209DF883
:106C1800013043EA022323809DF802209DF80330C7
:106C280043EA022363809DF804209DF8053043EA77
:106C38000223A380012003B030BD00BF84080020D8
:106C480013B5104B04465B686A4606213B209847FB
:106C5800A8B19DF800209DF8013043EA0223238063
:106C68009DF802209DF8033043EA022363809DF8D3
:106C780004209DF8053043EA0223A380012002B0D6
:106C880010BD00BF84080020026D036B70B5044678
:106C9800D5699BB9A90611D5C36A1BB1908C80B27E
:106CA80098470BE0E169928C40694E1CD2B2E661CC
:106CB8004254E169E268914228BFE361616BA1B97E
:106CC8002A0612D5636AA26A9A42236D09D0501C1B
:106CD800A669A062B25C1A852369984205D3A162AD
:106CE80003E01A6822F080021A602B0742BF236D66
:106CF80008221A6270BD0168027B30B502230C6855
:106D080003FA02F222420BD0064A002414704468A7
:106D180025684FF6FE722A402260027B93404B6042
:106D280030BD00BF194D00208379406BDB0744BF9D
:106D3800B1FA81F1490909B10BF02DBB0BF026BB63
:106D4800094B10B51868094C0BF034FB18B10EF05C
:106D5800AFF8E06110BD0EF0ABF8E369984282BF6E
:106D6800C01A034B186010BDB8080020B40F0020EB
:106D78009C0500201FB50123ADF80830ADF80410BC
:106D8800002301A9ADF80A30ADF80C30ADF80620A3
:106D980006F002FF05B05DF804FB38B5A0F51574E0
:106DA8006379DB0743D5A57994F8403205F00105EE
:106DB800EBB1A16B0868C36A5B08436294F844327C
:106DC80023B1B4F84A320133A4F84A326A00497947
:106DD800FFF7D0FF012384F84332002384F84132BF
:106DE80084F8423284F84032A4F8483238BD94F826
:106DF8004332012B04BF94F8413284F842322046D2
:106E0800FFF7A7FC94F84322A36B2AB9012284F860
:106E1800432205FA02F205E00022954284F8432253
:106E280008BF022259791868BDE83840A2E738BD82
:106E380010B5A0F5147494F84422BAB9A36A616A2B
:106E4800994228D0591CA069A162C35C2069DBB2B1
:106E58005B0043F400738142A4F846324FF00A0302
:106E680084F8453228BFA262012312E094F9453222
:106E78007BB1B4F846124B08A4F8463201F0010180
:106E88002046FFF751FF94F84532013B84F845321C
:106E980001E084F8443294F84032002B4ED194F843
:106EA80041320133DBB2092B84F8413203D1204649
:106EB800BDE810404DE40A2B40D194F843322BB979
:106EC800B4F8483243F00103A4F848326379D9078B
:106ED8001CD5B4F84802820501D4C30705D4B4F818
:106EE8004C320133A4F84C3210E0E36AC0F3470097
:106EF8000BB198470AE0E3696269D054E369E16835
:106F08000133B3FBF1F201FB1233E361012284F890
:106F1800402294F843220023012A84F841320DD1FB
:106F2800A27984F84332A36B12F0010F0CBF02223E
:106F3800002259791868BDE810401BE710BD13B549
:106F4800062204466B4603211E200FF0C1FD0028CF
:106F58003DD09DF800209DF801309DF8021043EACD
:106F680002231BB21B4A07EE903A92ED007AF8EE24
:106F7800E77A012067EE877A92ED027AFDEEE77AEA
:106F880017EE903A23809DF8033043EA01231BB2A1
:106F980007EE903AF8EEE77A9DF8041067EE877AE4
:106FA80092ED017AFDEEE77A17EE903AA3809DF80C
:106FB800053043EA01231BB207EE903AF8EEE77A70
:106FC80067EE877AFDEEE77A17EE903A638002B0B3
:106FD80010BD00BF0400002007B506226B46F7214C
:106FE80076200FF075FD9DF801309DF800100C4AD1
:106FF8001B0143EA01339DF8021043EA1113536061
:107008009DF804309DF803101B0143EA01339DF8F5
:10701800051043EA1113136003B05DF804FB00BFC9
:10702800B40F002007B5032201ABF62177200FF03B
:107038004FFD9DF805309DF804201B0243EA0243EA
:107048009DF806201A43064BB3F92030C3F1080314
:1070580022FA03F3034AD36003B05DF804FB00BFD0
:107068005C2E0020B40F002007B5022201ABF621E8
:1070780077200FF02DFD9DF804209DF8053043EA98
:107088000223024A138103B05DF804FBB40F002009
:1070980007B5032201AB002177200FF019FD9DF8F9
:1070A80005309DF804001B0243EA00439DF80600E2
:1070B800184303B05DF804FB08B5FFF7E9FF014B7F
:1070C800586108BDB40F002008B5FFF7E1FF014B78
:1070D800186108BDB40F002013460A46014668200F
:1070E8000FF0F6BC1FB504460DF10703012202217B
:1070F8000C200FF0EDFC08B900203BE09DF80730AC
:10710800DB07F9D502AB062203210C200FF0E0FCC7
:107118000DF10703012209210C200FF0D9FC0028EA
:10712800EAD09DF8073013F00C0FE5D19DF809203F
:107138009DF8083043EA0223C3EB83339B009DF894
:107148000B2023809DF80A3043EA0223C3EB8333E4
:107158009B009DF80D2063809DF80C3043EA0223C4
:10716800C3EB83339B00A38001220A210C200FF07C
:1071780043FC012004B010BD07B500220A210C20F1
:107188000FF03AFC14200DF0D1FE0F220A210C203A
:107198000FF032FC0A200DF0C9FE01AB03221021CA
:1071A8000C200FF095FC0A200DF0C0FE00220A21E9
:1071B8000C200FF021FC0A200DF0B8FE0DF103039E
:1071C800012202210C200FF083FC0DF103030122A0
:1071D80009210C200FF07CFC01220A210C200FF061
:1071E8000BFC03B05DF804FB3122F42176200FF08C
:1071F80003BC054B93F820209201343202F0FC02C4
:10720800F42177200FF0F8BB5C2E00202E22F42109
:1072180077200FF0F1BB0122482177200FF0ECBB5B
:107228000122582177200FF0E7BB0A460146682063
:107238000FF0E2BB2DE9F74332200DF077FE112263
:1072480000211E200FF0D8FB602201211E200FF024
:10725800D3FB64200DF06AFE6846FFF770FE002439
:10726800DFF86C810A2726462546012202211E20C6
:107278000FF0C2FB32200DF059FE6846FFF75FFEA3
:10728800BDF90220BDF90010BDF904308A42164448
:10729800A8BF0A4693421D44A8BF134643450C4461
:1072A80004DB013FE1D14FF0010801E04FF0000895
:1072B800122200211E200FF09FFBDFF814910A27ED
:1072C800012202211E200FF097FB32200DF02EFE26
:1072D8006846FFF734FEBDF90220BDF90010BDF97C
:1072E80004308A42A6EB0206A8BF0A469342A5EBE1
:1072F8000305A8BF13464B45A4EB010402DB013F7D
:10730800DED101E04FF0000807EE904ADFED2A6A6F
:107318002A4FF8EEE77A702286EEA77A00211E201F
:10732800F0EEC77AC7ED007A07EE906AF8EEE77AD2
:1073380086EEA77ADFED226AF0EEC77AC7ED017A0A
:1073480007EE905AF8EEE77A86EEA77AF0EEC77A5B
:10735800C7ED027A0FF050FB202201211E200FF00A
:107368004BFB002202211E200FF046FB64200DF08B
:10737800DDFDB8F1000F04D14FF07E533B607B6018
:10738800BB60104B1B68187898B10AF0DBFF0E4DF4
:10739800044628620BF00EF858B129460B4B41F809
:1073A800243F20460823F0220BF0A3F920460FF0D3
:1073B8007BFC03B0BDE8F08300406F46040000206A
:1073C80001C05E46CC350020B40F00208767000856
:1073D80001F0FFFF124B1B6870B5FBB118780AF07B
:1073E800B1FF04460AF0E6FF0146B8B9142308269F
:1073F8000C4DA3712072E67120460BF033F8294634
:10740800094B41F8283FF022334620460BF071F92A
:1074180020460FF049FC012385F82C3070BD00BFD1
:107428009C080020B40F0020DD6B0008184B93F86F
:107438002C3070B505460BB9FFF7CCFF154C8021F1
:10744800A3686B20984764200DF070FDA3680321A2
:107458006B209847104AA3681178192098470F2085
:107468000DF064FDA36829461A209847A3681821DF
:107478001B209847A36818211C209847A36802215D
:1074880037209847A36801213820BDE87040184785
:10749800B40F002084080020C82E00200A4B93F85F
:1074A8002C3010B504460BB9FFF794FF074B5B78F7
:1074B80013B1012B03D010BD4FF4806301E04FF4EA
:1074C8000063238110BD00BFB40F0020402E0020B0
:1074D80010B4047B016843690222A2404A604168F3
:1074E80008684FF6FE7202400A60596A9A6A914229
:1074F80004D018465DF8044B04F01EBC012283F842
:1075080044205DF8044B704738B5154C0546206893
:107518000AF03CFF134940F2E93322460889800704
:107528000DD511490F480D7040F2E9330489E4077D
:1075380010D50B781068BDE838400AF02CBF013B25
:107548009BB2002BEAD109494B8B01339BB24B8389
:107558004B8BEFE7013B9BB2002BE7D1F3E700BF72
:10756800140C0020003800400C3800406C05002046
:107578002DE9F04F564D85B099464FF4167305F135
:10758800300743430646019207EB030810B92B4422
:10759800504A03E0012805D14F4A2B449A660C3221
:1075A800C3F86C214FF416737343EC184B4A2263EB
:1075B800019AA263032284F83520FA183C3203F5B5
:1075C800A0733B44D4F86CB1E16562644FF48071F8
:1075D80000224FF0010AA364E1632265E26421649A
:1075E800A265626584F8742284F87122A4F87A226C
:1075F800A4F87C2284F8369084F870A284F87E621D
:107608009BF804000AF09EFE60669BF804000AF0EE
:1076180099FE06EB0A0B05225FFA8BFB8271C27199
:1076280080F808B0514603920AF01CFFA16E02913F
:1076380008790AF087FE0299206608790AF082FE26
:10764800039A82710622C27180F808B022210AF0DA
:1076580009FF51464046FFF767FB32200DF066FCF4
:10766800D4F86C411E4B019AB3FBF2F1B1F5803F9F
:1076780003D3012BF7D05B08F5E72046482289B2EF
:107688000DF0ECFB4FF416735E43354406F51476A3
:10769800144BC5F8803237440022394620460DF095
:1076A80035FBAC6E19F0010F0CBF02220022617984
:1076B8002068FFF75FFB0C4BC5F884322046002298
:1076C800391D0DF023FB404605B0BDE8F08F00BF23
:1076D800B40F0020E8C3010800C4010838CA010833
:1076E80000A24A04396E0008A36D000883790A468F
:1076F800C16A90F84E023BE72DE9F04F894A85B000
:107708001378029203F0FF05002B40F00881864EA3
:10771800019696F8E42496F8E59496F8E634A6F8E7
:10772800E054A6F8E25429462F46AE46AC46AB468E
:107738003C240FFA85F8B8F1200F00F0BF807B4891
:1077480000EB880C9CF803009CF802C0CCF1FF0CFD
:107758001FFA8CFCBCF1000F00F08280734ECCF154
:10776800FF0C00FB0CFC36F828804FEA2C2C3C263A
:10777800B8FBF6FABAF1050F75D8DFE80AF003107E
:107788002233485A5FFA8CF3CCEB000C08FB0CF858
:10779800B8FBF4F8984402465FFA88F05CE0B8FB5E
:1077A800F4F204FB128292B25FFA8CF3C2F13C024B
:1077B800CCEB000C0CFB02F2B2FBF4F21A44D2B28E
:1077C8004AE0B8FBF4F304FB13885FFA8CF21FFA63
:1077D80088F8CCEB000C08FB0CF3B3FBF4F3134470
:1077E800DBB239E0B8FBF4F304FB13881FFA88F81E
:1077F8005FFA8CF2C8F13C08CCEB000C0CFB08FCDF
:10780800BCFBF4FC944403465FFA8CF024E0B8FB1C
:10781800F4F204FB12885FFA8CF11FFA88F8CCEBBB
:10782800000C08FB0CF2B2FBF4F20A44D2B2034695
:1078380011E0B8FBF4F304FB13839BB25FFA8CF1FD
:10784800C3F13C03CCEB000C0CFB03F3B3FBF4F3E8
:107858000B44DBB20246084601210F468E4603E080
:1078680003460246F8E748464FEA02284FF0170C4D
:1078780048EA00480BEB0C0648EA03080396039E07
:10788800CCEB0609012606FA0CFA1AEA080F1FFAC9
:1078980089F9274E14BF4FF0110A4FF0090A1CF15D
:1078A800FF3C06F809A0EAD20BF1180C01351FFAC3
:1078B8008CFBADB24FF0010C81463AE7BCF1000FEA
:1078C80002D00198A0F8E0B4BEF1000F02D00198F0
:1078D80080F8E42417B1019A82F8E59411B1019A6D
:1078E80082F8E634BCF1000F03D0019A2023A2F8F5
:1078F800E234029A012313700E4B1B787BB10E4AB7
:107908000E4940F22A33536000234B620B889BB226
:1079180043F001030B80136843F00103136005B0C3
:10792800BDE8F08F194D0020B40F00201A4D00203B
:10793800C8080020F80B00201C000240002C014061
:1079480070470148FFF7A0B9B81800200148FFF7B1
:107958009BB900BF641800200148FFF795B900BF24
:1079680010180020F7B506460D46002401272A887E
:1079780007FA04F31A421AD0AA78009302F0030314
:107988008DF80430EB78022B03D0032B0CBF0323B4
:1079980001238DF805306946C2F301133046C2F35E
:1079A80081028DF806308DF8072006F029FB013496
:1079B800102CDCD103B0F0BD0348D0F8103113B15E
:1079C80000F5847018477047A80000200348D0F8D5
:1079D800F8300BB1F0301847704700BFA8000020FE
:1079E8000348D0F8E0300BB1D8301847704700BFD3
:1079F800A80000200348D0F8C8300BB1C0301847A1
:107A0800704700BFA80000200348D0F8B0300BB181
:107A1800A8301847704700BFA80000200348D0F8D6
:107A280098300BB190301847704700BFA80000206D
:107A38000348D0F880300BB178301847704700BF42
:107A4800A80000200248836E0BB1603018477047C9
:107A5800A80000200248036D0BB148301847704752
:107A6800A80000200248836B0BB1303018477047DC
:107A7800A80000200248036A0BB118301847704765
:107A8800A80000200248836803B11847704700BF68
:107A9800A8000020034A138801339BB213800020FA
:107AA800704700BF8A2400201549D1F8883043F474
:107AB8007003C1F88830134B1A6842F001021A604B
:107AC8005868114A02405A601A6822F0847222F4F7
:107AD80080321A601A6822F480221A605A6822F4E6
:107AE800FE025A60DA6A22F00F02DA62186B074A5D
:107AF80002401A6300229A604FF000638B6070475F
:107B080000ED00E0001002400CC07FF8CCFC00FF44
:107B1800A2490A682DE9F04F02F59C43A04C203396
:107B28002360A04B89B01E7802911EB9DFF89882B5
:107B38009D4F18E09D4909688A4240F20181013E43
:107B48001E70FDE0072D98BFD8F80030984898BF00
:107B5800595D3B6888BF29469847032D09D904EB2E
:107B680045050136A88007F08BF9F5B28542E9D3BF
:107B780020E0D8F8002005F1100302EB8303998870
:107B8800DA880028EBD04FF47A73401A5843531A16
:107B980090FBF3F040F6C90300F57A70984205DCD3
:107BA80040F2EE239842B8BF184601E040F6CA00FA
:107BB80080B2D4E77F4B1A6842F2010A02EA0A0A45
:107BC8007D4A136801939046BAF1000F06D094F8E5
:107BD800292084F82820794A5178117094F828606F
:107BE8001EB1764A167886F00106754F0F2284F882
:107BF8002A20002507F1460B07F042F9854264DA8E
:107C08004FEA45091EB16F4B33F8150000E03046C6
:107C18006D4B19688A8B82424FEA850E6B4A02D8EF
:107C2800C98B81421CD25BF80E00019B5C499842CB
:107C380002D932F8090018E0E8B20492039107F07B
:107C480037F9032D049A10DC03994FF0010E0EFA50
:107C580005FC91F82AE02EEA0C0E81F82AE004E0EF
:107C6800019B03F596714BF80E10BAF1000F27D05F
:107C780094F8BC100322B1FBF2F202EB42028A1A1A
:107C880009EB050E5EFA82F204EB4202908594F845
:107C9800BD202AB9022912D9414A012182F8BD1012
:107CA80037F8020C3A884A490244788810FA82F276
:107CB80012B221F80920032092FBF0F080B2434A67
:107CC80022F809000135063796E794F82A300F2B79
:107CD8000CBF0123002384F8D6303E4B0ED13E4A18
:107CE800126850010AD4D8F80020D9689A60521A4C
:107CF800C82A20D9012283F821201CE02F4A334EBC
:107D0800012151701170D8F800209968DA605B6819
:107D1800521A9A4282BF2F4B002283F82120002555
:107D280007F0AEF8854206DAE8B207F0C1F826F89F
:107D380015000135F4E794F8BC30013384F8BC3001
:107D48001C4B1A6812F4805F9B4605D0224B1B68B7
:107D5800D90701D410F0F6F9029B18681A4B1E686F
:107D6800337B002B3CD0194A013B32F91330B27BEC
:107D78001AB1C3F53B6308331BB2A3F57A73B3F5A5
:107D88007A7FA8BF4FF47A7323EAE37307EE903A39
:107D9800DFED126AF8EEE77A5CE000BFE03D002014
:107DA8009C140020A0240020580500209C240020BA
:107DB800342E002098240020842400202000002055
:107DC800CA140020A014002094240020E42D0020D0
:107DD8005A150020A4240020D424002000007A444E
:107DE800DBF80020120441D5D4F8D820AE4D821A11
:107DF800002A3BDB00F59C422032C5F8D820AB4A6C
:107E0800D179AB4A32F811108AB2717B92FBF1F149
:107E180095F8DC20013202F00F0285F8DC202A44B4
:107E2800DD3582F8DD1019464A5D01311A44102902
:107E380013B2F9D193FBF1F31BB2002B03DB642BD4
:107E4800A8BF642300E0002307EE903ADFED996AAB
:107E5800F8EEE77A87EEA67A974ADFED987A67EE2A
:107E6800277AFCEEE77A17EE903A1380DBF80030B9
:107E7800DFF870A213F4807F00F0FA80904BDFF8EF
:107E88004492984205D999F8022012B9012289F83A
:107E9800022099F80220002A00F0EA80894A8A49DB
:107EA80092F8215008689AF80020039102F004071C
:107EB80000F08063012DFFB2029305D012F0080F85
:107EC8000CBF0023022300E00023804EDFF8188255
:107ED800019399F82020052A00F2C580DFE802F016
:107EE80003485C7D8DADB7B3B4F8EE10D4F8F0005C
:107EF80008F022FE012808D1D8F800103268C98895
:107F0800642000FB0122C9F81020029B5BB1D8F85D
:107F1800002012793AB10CF097FE032289F820204C
:107F28004FF47A7235E0012D00F09D803168D9F860
:107F38001000644A88420AD204920CF085FE049A22
:107F4800032182F8201040F6B831D161C1E7012140
:107F580082F82010BDE7029B4FF4806013B10AF04D
:107F680095FC01E00AF082FC0022C9F810207AE0B2
:107F7800012D56D0D8F80020127A012A02D00CF030
:107F880063FEA6E70CF060FE032289F8202040F685
:107F9800B832C9F81C209CE7012D04BF052289F8D6
:107FA80020206FB1D4F8F020B2F91010484A11809F
:107FB80051809180D8F8001003234988D18001931B
:107FC8003268D9F81410914201D3002F48D147F2F2
:107FD8003052C9F81C20032224E09AF8002042F00D
:107FE80002028AF8002010F0ADF83268D9F81C10A7
:107FF8000A44C9F81820042214E0012D15D132686A
:10800800D9F8181091422ED2324B1A781AB9039B1C
:108018001A68D30727D49AF8002022F002028AF8B7
:108028000020052289F8202053E7284AD9F81C1097
:1080380012680A44C9F8182015E0D8F80010326808
:10804800C988642000FB0122C9F810204FF4806021
:10805800002289F8202089F803200AF007FC38E775
:10806800012D3FF436AF019B13B1184608F0CAFD45
:10807800194EB6F8DC1006F5117008F05DFD0546DE
:1080880008F09AFDB146154E80B39AF800305807AB
:108098002CD5134BB3F90620B9F85E329A4239DB76
:1080A800012384F8F4303AE09C140020AC2100202D
:1080B800C02100200000C842C44D002000C07F44F9
:1080C800404B4C00A4240020D42400208424002009
:1080D800E42D00209C000020B0450020B82B002093
:1080E8001C250020D824002064420020002384F8A6
:1080F800F430A5B99E4B9F4900221A605A609A60D5
:108108009D4B1B6893F834300020086048608860F5
:108118002BB905E01DB994F8F430002BEAD00123FF
:1081280033709AF80030590737D5DBF80030DA0693
:1081380033D5924A1278D7062FD4DE042DD408F00E
:108148003BFD50BB8E4B1B7883B199F89B329DB990
:108158006BB18C4B1A68D4F8F8309B1A002B06DAEE
:108168000FF0F0FF884B83F8FC5016E06DB9102033
:1081780008F048FD01230EE03BB1824A12684FF433
:108188007A7101FB0323C4F8F83094F8FC3023B16A
:1081980008F020FD002384F8FC30002299F89A1298
:1081A800B9F85662B9F85872DFF8F0E113463EF9AB
:1081B80012009B08B042C4BF63F07F03DBB20132F8
:1081C800B842B8BF43F04003042AF0D194F8FD2028
:1081D8006D489A4205D190F8FE20F92A04D8013258
:1081E80000E0002280F8FE20654F84F8FD303B78DF
:1081F800654A664E23BB3068C00709D582F8FF3050
:10820800F5B99AF80030DA071AD50FF023FF17E00E
:108218009AF800305B0713D592F8283083B15C4B8D
:10822800DB786BB992F8FF300133DBB2032B82F8AD
:10823800FF3005D911B10FF085FF01E0002DFAD00C
:1082480094F8FE30504D142B65D13B7893B195F8D6
:10825800FD305F2B0ED19AF8003003F0040303F0D1
:10826800FF0813B10FF06EFF04E00B2008F0CAFC02
:1082780085F8FE809AF8003003F0040303F0FF024B
:10828800002B48D194F8FD503F4B572D0FD105F0E6
:10829800FCFEDBF800301D0601D50BF019FD3D4B47
:1082A8001B68580737D53C4B0A221A8033E0DBF8A5
:1082B8000010490717D55A2D15D193F8001129B187
:1082C80083F80021012283F8012124E093F8022198
:1082D80082F0010283F802210AB10C2000E00D208F
:1082E80008F090FC17E05D2D00F01D845B2D00F078
:1082F8001C845E2D02D1032000F018BC562D01D13C
:108308000AF0AAFB3B78002B00F016846F2D40F092
:1083180013840FF09FFEDBF80030580750D594F80F
:108328000231194A9BB19AF8003059070FD51B4BF7
:10833800B3F90610B9F85632994208DD336813F0DC
:10834800010302BF3221A2F8061182F80231336814
:10835800DA0325D594F808210B4B2AB993F80021A4
:1083680012B93222A3F80621012384F8083127E044
:10837800582C0020442500200C25002044160020FD
:108388009C000020842400209C140020D424002079
:10839800A4240020542E0020E83D0020E42D0020D5
:1083A80094F80031B54A5BB19AF8003003F0040341
:1083B80003F0FF0123B9012382F8001182F801318B
:1083C800AF4D0023336005F150074FF001082946EF
:1083D80015F8010C08F08AFB30B115F8023C08FAD0
:1083E80003F23368134333600435BD42EFD1A54B24
:1083F8001E783EB1A44EA54F336813F0020F40F02B
:10840800C581BCE1A24DA34F05F15A08294615F8CC
:10841800010C08F06BFBE8B1AB789F4A297995F815
:1084280003C0013B03EB430313440C2202FB01FE90
:1084380007EB0E00426893420CD04360012303FA15
:1084480001F194F8093107F80EC023EA01018660AA
:1084580084F809110635A845D8D1904B904E1D686F
:10846800904B1B68039394F8283004938E4B029327
:1084780000230193029B1A68002A00F0758117787F
:10848800002F00F071815B680399CB1A002B0DDB7C
:1084980001F5FA7302994B600199012303FA01F17E
:1084A80094F8093123EA010384F80931049B002B6D
:1084B80000F05A81029B517813F8043C0433DBB274
:1084C800002940F01A81794931F91310B9F854326A
:1084D80003F1C800814202DD92F8028016E0C83B31
:1084E800994203DA9178C1F100080FE0019A01235B
:1084F80003FA02F294F8093123EA020384F80931F5
:10850800039B029A03F5FA7353602DE1019B94F8DB
:1085180009211A41D30700F12781B8F1000FCCBF18
:108528000220012008F0AEFB7A1E132A00F2138104
:10853800DFE812F014001E00280038005000570031
:1085480071008B00C000CB00D80011013800460034
:10855800570071008B00660080009900297841441B
:10856800FA29A8BFFA2121EAE17129700120B6E0B1
:10857800A97841446429A8BF642121EAE171A9705E
:108588000220ACE02F794A4B4744642FA8BF6427E8
:1085980027EAE77719682F71284608F04FFA394615
:1085A80003209CE0A97941446429A8BF642121EAF9
:1085B800E171A9710D2008F0DFFA0D2F00F0CB80D2
:1085C800697941446429A8BF642121EAE17169718C
:1085D8000E2084E0E979414481F30801E97105201E
:1085E8007DE0326891784144C829A8BFC82121EAB2
:1085F800E17191700F2008F0BFFA0F2F00F0AB80E7
:10860800326851784144C829A8BFC82121EAE171DC
:108618005170122063E03268117B4144C829A8BF19
:10862800C82121EAE1711173102008F0A5FA102F72
:1086380000F091803268D17A4144C829A8BFC82186
:1086480021EAE171D172132049E03268917D4144F9
:10865800C829A8BFC82121EAE1719175112008F045
:108668008BFA112F77D03268517D4144C829A8BFB1
:10867800C82121EAE1715175142030E09C140020D2
:10868800DB4A0020784C0020D4240020542E0020FF
:108698002A4B00202017002060CA0108F43C002063
:1086A800541700208424002024170020E42D0020E3
:1086B800501700203268D1784144C829A8BFC82182
:1086C80021EAE171D170092009E03268517B414407
:1086D800C829A8BFC82121EAE17151730A2008F00E
:1086E8004BFA38E03268D17D4144C829A8BFC82177
:1086F80021EAE171D1750B20F1E701292BD1B949A4
:1087080031F91300B0F5617F05DB40F6330383428E
:10871800A8BF034601E04FF461730C2F1BD190787A
:108728004FF4966292FBF0F0AF4A1278A3F56173AA
:1087380093FBF0F3DBB29A420DD0184605930AF08A
:10874800BDF8059B3846194608F016FA059B581CD3
:10875800C0B208F097FA019A012303FA02F294F8DA
:108768000931134384F80931019B01330193029BBA
:108778000C330293019B042B7FF47CAE3AE6DBF8C2
:108788000030D8050FD5994BDB7863B13B68990762
:1087980009D5974B1B8813F0010509D101200AF070
:1087A80075F82B4605E001200AF060F8012300E087
:1087B8000023326852070BD553B101200AF056F84E
:1087C8008B4B1B889B0706D402200AF05FF802E057
:1087D80002200AF04BF83B6813F00A0F2ED03368DA
:1087E800DD060FD5824B1B8858070ED404200AF0EB
:1087F8004DF8804B0A22B3F9043093FBF2F3A4F846
:108808000A3102E004200AF031F83368990607D5E6
:10881800774B1B885A0606D440200AF037F802E046
:1088280040200AF023F833685B0607D5714B0A220B
:10883800B3F9043093FBF2F3A4F80C313B689D06BE
:1088480008D43368180540F198804FF480700AF016
:108858001DF896E0684BDFF898811B7813F0020F3B
:1088680053D0664B1B78042B4FD9336813F400732D
:108878000FD0B8F80030D9063BD410200AF006F81B
:10888800202009F0F3FF5E49081F0BF075F9022359
:108898002BE0B8F8005005F01005ADB23DB110203E
:1088A800019309F0E3FF019B84F80E310125336839
:1088B8005A0512D5534B54491B685A89B1F90030EF
:1088C800002BB8BF5B42934207DAB1F90230002BA4
:1088D800B8BF5B429A4200F37D81B8F800309B062E
:1088E80008D5202009F0C2FF002384F80E310125A5
:1088F80000E0002594F81831BBB90E2008F082F981
:10890800424B012283F818210FE0B8F8003003F039
:108918003003002B95D0102009F0A8FF202009F083
:10892800A5FF002384F80E3101E0002D89D03849D5
:10893800002300220B80A4F81A31A4F81E31C4F8D1
:108948002421C4F82831C4F82C21C4F84C21C4F8D7
:108958005031C4F854214B80A4F81C31A4F82031BC
:10896800C4F83821C4F83C31C4F84021C4F8602167
:10897800C4F86431C4F8682163E74FF4807009F0E3
:1089880075FF99F80530082B01D00E2B02D1402035
:1089980009F06CFFDBF80030580519D599F8E0327A
:1089A80023B99AF8003013F0040F02E0336813F487
:1089B800002F09D03C2008F007FF48B106F0B0FBB3
:1089C8003C200EF0E5F9F8E70EF01BFF08F004FF75
:1089D8009AF800300120590784F874011AD50EF06E
:1089E8005BF95BE0E42D00208E240020A424002005
:1089F800D024002028250020441600204A160020F4
:108A08000C170020601700201C2500209C14002053
:108A1800242500203268D20703D57B4A92F87521B5
:108A28001AB143F001038AF80030784B784A1B7872
:108A38001D075EBF9AF8003023F001038AF8003062
:108A48003B6813F0040F02D07249098871B9B4F871
:108A5800041109B1980709D46F4B1B88003318BF5C
:108A680001231BB96D490988642908D902231370A9
:108A78009AF8003023F001038AF8003005E09AF8EC
:108A88000010C90758BF022313700CF011FA644B89
:108A98001B68C01A002801DB06F092FA3B685D07E4
:108AA8001BD53368180703D4082009F0DFFE14E04B
:108AB8005C4B1D8805F00805ADB275B9082009F0B2
:108AC800E5FE594B1A68594B1A60594BDB88A4F8D4
:108AD8007631584B1D60584B1D603B68D90640F1F4
:108AE800908033689A0206D44FF4007009B0BDE84C
:108AF800F04F09F0BBBE4B4B1D8805F40075ADB2B5
:108B0800002D7ED14FF4007009F0C0FE464B1A6864
:108B1800464B1A60464BDB88A4F87631454B1D60FE
:108B2800454B1D606DE0012000E002200138C0B215
:108B380009F080FFFFF7EFBB972D05D14FF4C873FD
:108B4800A4F80431FFF7E7BBA72D06D12F4A137805
:108B580043F004031370FFF7DEBB0023BB2D07931C
:108B680001D1022303E0B72D04D14FF6FE73ADF80F
:108B78001E3009E0BE2D01D1022303E0BD2D18D11E
:108B88004FF6FE73ADF81C30B9F8F221BDF81C3071
:108B98001344A9F8F231B9F8F421BDF81E30134492
:108BA800A9F8F43109F058FF002384F8FE30FFF7E4
:108BB800B2BB792D04D1214AD37823F0010306E012
:108BC8007A2D7FF4A8AB1D4AD37843F00103D37004
:108BD800FFF7A1BBB8F800309B063FF58BAE20200D
:108BE80009F054FE164B17491A685B68C4F810213F
:108BF800081F0125C4F814310AF0BEFF84F80E518D
:108C080078E609B0BDE8F08F9C14002044160020D7
:108C1800C8240020E83D00207221002028210020DF
:108C2800CC240020D0240020041700202C3E002053
:108C3800E42D0020383E00203C3E00201C4C002043
:108C48004C160020B01500202DE9F04F2DED028BB9
:108C580087B00EF0D6FDC04B1D78002D40F0CF87B1
:108C6800BE4E3368580540F1CA87BD4CBD4F2378C6
:108C7800002B00F00B823A686368D31A7C2B40F211
:108C88000582B94BDFF80CA3B3F8DC80237A9FED9B
:108C9800B78A62600133237205F12400DFF8C092BD
:108CA800C0B20EF055FD09F10C0353F8253006EE5D
:108CB800903ABAF8083007EE103AF8EEE66AB8EEDD
:108CC800C77A0135C6EE877A67EE887AFDEEE77ACD
:108CD800CDED017ABDF904000EF028FD032DDBD19E
:108CE80030200EF035FDB9F918000EF01FFD0EF01A
:108CF80027FD99F80830990732D1D9F8042041F2B4
:108D080088339A4219D910200EF022FD6425D9F82B
:108D18001C0090FBF5F000B20EF008FD21200EF0CB
:108D280017FDD9F81C0090FBF5F305FB130000288C
:108D3800B8BF404200B20EF0F9FC14200EF008FD56
:108D48008B4BB3F904000A2390FBF3F00EF0EEFC12
:108D58001C200EF0FDFC00200EF0E8FC0EF0F0FCEC
:108D6800237A5A0740F06A8102200EF0F1FC7C4B0E
:108D7800186A6423323090FBF3F000B20EF0D6FC90
:108D88007C4B0320B3F906500EF0E2FC7A4B1B78BB
:108D98005B074FF0050995FBF9F5ADB20BD54146D8
:108DA800764807F0C9FE20B9336813F0100F18BFD2
:108DB800002528B205E0724B1B68D889B0FBF9F092
:108DC80000B20EF0B3FC33689D076FD5DFF8C89189
:108DD800A58CDFF8C88199F80010B8F800202D019B
:108DE8006423ADB203FB02124B00B2FBF3F345EA76
:108DF8000325ADB2C3F303231D4306200EF0A8FCE0
:108E080028B20EF093FCA38C99F8001001339BB2A2
:108E180093FBF1F201FB1233A26AA384937B012B2B
:108E280005D139200EF094FCB8F9000021E0B8F81B
:108E380000506E236B43152593FBF5F5D37BADB23C
:108E48000BB195FBF1F53A200EF082FC4FF0640966
:108E5800B5FBF9F80FFA88F00EF068FC09FB185515
:108E68003B200EF075FCA8B2451D0A2095FBF0F0DA
:108E780000B20EF05BFC28200EF06AFCE36A0A20C0
:108E880093FBF0F000B20EF051FC04200EF060FCF1
:108E98003B4B1B68DB8913B105F08CF903E0394BB8
:108EA800186880F3100000B20EF040FC364B1B68C7
:108EB800980640F1B88094F83030DFF8A48099071C
:108EC8001DD511200EF044FCB8F832002F4B4FF49A
:108ED800F365684390FBF3F000B20EF027FC19200D
:108EE8000EF036FCB8F832004543642095FBF0F5E7
:108EF80095FBF0F300FB135000B20EF017FC94F84A
:108F08003030A58E13F0020F08BF002501200EF0A7
:108F18001FFC28B20EF00AFC09200EF019FC0020F4
:108F28000EF004FC1A4B94F836501A88B2F5967F66
:108F38000AD90B4B1B7A03F00F03072B04D842F214
:108F48000F75954228BF154605200EF001FCA36A4F
:108F58005B7B3BBB28B241E0784C00209824002082
:108F68001416002084240020B045002000007A4414
:108F7800282500201C250020D8240020F4470020A4
:108F8800A4210020A8210020542E0020A086010042
:108F980024000020442E002040050020F421002059
:108FA8006666E63F203D07EE905A5FED036AF8EEED
:108FB800E77A87EEA67AF6EE006AB5EEC07AF1EEA9
:108FC80010FAFEEE007A58BFF0EE667A37EE277A8E
:108FD800FDEEC77ACDED017ABDF904000EF0A6FBCF
:108FE80094F83020C44B920703D493F83720012A11
:108FF80004D1012384F83730C0481BE09B6ADFEDB9
:10900800C06A93ED017AD3ED027A27EE267A67EEED
:10901800A67ABDEEC77AFDEEE77A8DED047ACDED3E
:10902800057A04A806E0B74A92E8030004AB83E88F
:10903800030018460EF09CFB0EF082FB237A282BC7
:1090480024D1AD4B3D6800224FF03C0817201A721E
:109058000EF07EFB4EF66020B5FBF0F0B0FBF8F3A7
:1090680008FB1300000200B20EF060FB18200EF09F
:109078006FFB4FF47A70B5FBF0F5B5FBF8F008FB21
:10908800105000B20EF052FB0EF05AFB94F840302C
:10909800994D002B00F05C810BF00AFF6B6C9A4A2B
:1090A800C31A9342804640F2C080002385F84A30B4
:1090B80085F84C30954B1B88DAB21B0A85F8662078
:1090C80085F8673085F85C2085F85D306A6F3B6805
:1090D8009A1AAB6F197C4FF47A734B439A420DD3AB
:1090E8008B4B1B686B678B4B1B78013B012B9FBF1E
:1090F800102385F84A30022385F84C300A20E26AAA
:10910800854B92FBF0F284F86420121284F86520F3
:1091180094F830201B6893FBF0F384F868301B1236
:1091280084F86930970794F83630734984F8963094
:1091380003D42D2381F8973074E0042BD4F838A099
:10914800DFF8E491E06B754A9AFBF2F58CBF3323A4
:10915800322381F897304FF0060C09FB05A1704BBC
:1091680090FBF2F20CFB01F109FB020991FBF3F70A
:109178004FF0640E03FB17110CFB09FC91FBFEF189
:1091880002EB820284F88810091284F8891002EB35
:1091980082029CFBF3F103FB11C349B201EB82028B
:1091A80092B284F88B20120A93FBFEF384F88C2089
:1091B80084F88D30628E1B1284F88E30242353433A
:1091C8004FF47A7293FBF2F384F88330C3F30723E6
:1091D80084F88430B4F8A83084F88F301B0A84F8F7
:1091E8009030A38E05EB850505EB85057FB203F569
:1091F800FA739BB207EB8505ADB284F891301B0A70
:109208004FEADA7A84F88650C00F2D0A84F8923033
:10921800B4F8AA3084F885A084F8875084F88A00C6
:1092280084F89830344BC3F84480334C94F8AC70CD
:1092380077B9D4F8B40002F041FFC0B2012807D9C9
:109248000228384D00F09D840EF062FA0123AB70BD
:10925800D4F8B850284B002D7AD093F8AC2042B1FE
:10926800D3F8C02040F6B731C2EB08028A4218D8BA
:109278006EE0012283F8AC20D3F8C4201278022AC9
:1092880006D8D3F8B400022104300EF02BFA04E01B
:109298000221D3F8B40002F005FF002384F8C83097
:1092A80054E093F8BC20BAB9C3F8B82083F8AC20CE
:1092B800D3F8C4201278022A06D8D3F8B4000121C2
:1092C80004300EF00FFA04E00121D3F8B40002F0E4
:1092D800E9FE0EF01DFA39E0013AD2B283F8BC205B
:1092E80093F8C81093F8C90002BB4A1C013083F8F0
:1092F800C82083F8C90025E0141600204C16002069
:109308008096184B9CCA01083F0D0300F4210020E9
:109318008424002088240020A8210020809698001A
:1093280040420F0024000020806967FF2A46013070
:1093380012F8017BC3F8B8207D1883F8C85083F869
:10934800C9003946D3F8B40002F0BBFEC4F8C080A7
:10935800C04CC14F94F8CA803B680193B8F1000F24
:1093680000F0F281D4F8CC30002B00F0ED8194F8B5
:10937800D030013B012B00F2E781A2464FF0020BEF
:109388000125D4F8CC00DFF8CC9202F097FED8B1D2
:10939800DAF8CC0002F08FFE9AF8D1103A687E29EC
:1093A80081460ED11B288AF8D0B00AD1DAF8CC0051
:1093B800029202F083FE20B9029ACAF8D4208AF8F1
:1093C800D85084F8D190DCE7D9F8D4103B685B1A00
:1093D80041F658318B4203D9032389F8D030B3E1E1
:1093E800DFF890A2054694F8D8E094F8D930002226
:1093F800BEF1000F00F0A58139680198091A01290A
:1094080006D90AB184F8D930002384F8D8309BE112
:109418000AEB4302108910B903464FF40360013385
:10942800B0F5E06FDBB2424600F02F815ED8B0F5B0
:10943800047F00F092800BD8B0F5887F00F0FD80A3
:10944800B0F5007F00F09F80B0F5807FD0D1A8E014
:10945800B0F5826F00F02481B0F5C06F00F0AD80E8
:10946800B0F5806FC4D184F8D93094F8E030794AE7
:109478000133DBB2032B88BF012382F8E03094F874
:10948800E01042F210735943744B1B78D80748BF59
:1094980001319A0748BF02315B07714B1B8848BFEF
:1094A8000431D80748BF0A319A0748BF1431180653
:1094B80048BF2831DA0548BF2831580748BF64310A
:1094C8001A0748BFC831980548BF01F5C8719A0600
:1094D80048BF01F57A71D80648BF01F5FA615A0606
:1094E80048BF01F57A614FF48060A1E0B0F5026FE2
:1094F80000F0FC800ED8B0F5E46F00F0CA80B0F53B
:10950800006F63D0B0F5E26F7FF472AF84F8D930A2
:109518002169C1E0B0F5046F00F0AE80B0F5116FBD
:1095280000F0FB80B0F5036F7FF462AF84F8D930A8
:109538004C4BDFF820B11B689A067FF554AF9BF8B7
:1095480030309B077FF54FAFBBF8321024234B43D5
:109558001233642193FBF1F1DAE084F8D9303368EF
:1095680098077FF540AF3B4BD3F8DC30DA7B3E4BB6
:109578001B881AB13D4A117893FBF1F30A2159432C
:109588004FF4047054E084F8D9303368DFF8C4B07D
:1095980019057FF528AFDBF82C100A2391FBF3F1AE
:1095A800B6E084F8D9302F4BDFF8A8B01B685A070B
:1095B8007FF519AFDBF81C10AAE084F8D9303368BE
:1095C8001B057FF510AF2A4B1968B4E02549214ADD
:1095D800096884F8D93089067FF505AF92F830100C
:1095E80088077FF500AFD90711D5D36B83EAE371FC
:1095F800002BA1EBE37101EB51014FF01902B1FB14
:10960800F2F1ACBF41F0004141F040410EE0936BF4
:1096180083EAE371A1EBE371002B01EB51014FF0F9
:109628001902B1FBF2F1B8BF41F080414FF400607C
:109638000EF024F884F8D850D5E684F8D930094BD0
:10964800DFF810B01B685B077FF5CDAEDBF81810AC
:109658005EE000BF1416002084240020D8240020D7
:10966800D0240020542E0020F421002040050020A2
:10967800A82100209CCA010884F8D930AE4BB3F960
:10968800041001EB81014900D2E784F8D930E16880
:1096980002E0616984F8D9302C2391FBF3F1C7E724
:1096A80084F8D930A54BDFF8A0B21B6813F0200965
:1096B80012D09BF8302012F0020F14BF4FF47A71C9
:1096C800002112F0010F14BF4FF4FA6300230B447A
:1096D80094F836101944ABE7326813067FF583AE69
:1096E80049460DF0CBFF8BF8D8907CE684F8D9304A
:1096F800924BDFF854B21B6899067FF574AE9BF85D
:1097080030309A077FF56FAEBBF834306421594387
:109718000DF0B4FF8BF8D85065E684F8D93033687B
:109728009B077FF560AE864B864A19880A234B4310
:10973800117893FBF1F10DF0A1FF834B83F8D8501A
:1097480051E60AB184F8D93094F8E130DFF8F881AD
:10975800002B00F0D880D8F8E430002B00F0D3803C
:109768003E68D8F8E830F31A632B40F2CC80724F89
:1097780041200DF06BFF0A25B7F9020090FBF5F0C8
:1097880080B20DF05AFFB7F9000090FBF5F080B2F7
:109798000DF053FFB7F9040090FBF5F080B20DF01F
:1097A8004CFF0DF01FFF98F8EC5015F0010535D06F
:1097B800624B1A6812F0200F99467AD098F8303028
:1097C800980706D598F83630052B34BF02270327AB
:1097D80000E0012747200DF039FFA06BDFF8688112
:1097E8000DF01AFFE06B0DF017FF6425608EB0FBDB
:1097F800F5F0C0B20DF000FFD9F8003013F0140FE7
:109808000ABFB8F83400D8F8F00068430DF004FF38
:1098180094F8360047EA8000C0B246E04B4B1B88FC
:10982800D90518D4DA060DD49F060DD458060DD4E0
:1098380019070DD4DA070DD413F0020F14BF03254E
:10984800012508E00D2506E0092504E0042502E0CD
:10985800082500E002253E4B1F783E4BDB78C7F316
:10986800800713B147F00207FFB253200DF0EEFE58
:10987800334B188800EB800000EB8000800080B23A
:109888000DF0DBFE00200DF0D8FE334B1888FE23C8
:10989800584340F2FF3390FBF3F0C0B20DF0ACFE3A
:1098A80000200DF0A9FE47EA85000DF0A5FE0DF099
:1098B80099FE94F8EC70244DC7B94F200DF0C6FE00
:1098C800D5F8F4000DF0A8FED5F8F8000DF0A4FEC8
:1098D80038460DF0A1FE01200DF08EFE95F83000FF
:1098E80000F001000DF088FE0DF07CFE94F8EC30DD
:1098F800C4F8E8600133DBB20A21B3FBF1F201FBE3
:10990800123384F8EC30154D95F80080B8F1020F49
:10991800AA4640F01E810BF0CBFA114B1E6840F6A8
:10992800B833861B9E421DD900232B70B4F8FC3037
:109938000133A4F8FC3062E128250020542E0020D1
:10994800F42100204005002014160020D024002017
:10995800D8240020A4240020C44D00201B2400206B
:1099680054240020DFF8BC9299F804303A2B40F0D8
:10997800048199F80210484605F00AFB002840F0D7
:10998800FC80A14BA14D1B88EB61E36AEB62E369A4
:10999800EB639F4BEE661B68D4F80061EB64B4F888
:1099A800FC30EB65304601F0E4FFDFF870B20746A3
:1099B800002840F0CE804146304602F073FB042375
:1099C80085F8743099F8033001939BF80431642BBF
:1099D80047D19BF80531072B08BF8BF8057194F820
:1099E800058105EB08167168039108460FF0DAF84F
:1099F800B36802935FFA80F918460FF0D3F85FFA5C
:109A080080FB844E039909EB0B020832F27128F0AF
:109A18000F02B27208F00F0272730BEBC902B27335
:109A280006F10F004A4610F0E9F8029B06EB090020
:109A380019465A460F3010F0E1F816F8079F4946C4
:109A4800304605F089FA06F80900019808F038F858
:109A580008F10108002384F8043184F805816D4E6B
:109A680060E095F87560DFF8B0C1330708BF0136CC
:109A7800684B08BFF6B2072E4FF0000203F10D0144
:109A880028BF01269A729B468E46330105EB0308D0
:109A9800481C98F81020D8F80C8043EA0209624460
:109AA80081F8009092F82A10012900F1010207D9E3
:109AB800013902F8018C10464FEA1828C9B2F3E7B9
:109AC8002B4401365B7C28F06008F6B248EA0308AC
:109AD800082E114680F800800CD04C4B4E4803EB02
:109AE80006131B7C034493F82A00CEEB02030344BD
:109AF800132BCADDCEEB020808F106085FFA88F8D6
:109B0800DFF8249148F040038BF807304146484677
:109B180005F022FA09F80800019885F8756007F041
:109B2800CFFF9CE7B37807F10108FFB2BB4206D923
:109B3800F15DD4F8000102F0C4FA4746F2E794F860
:109B480004310322013385F8742084F804318AF83B
:109B580000202E4D95F87430032B50D1D4F8000115
:109B680002F0A3FA00284AD02C4B0121D3F80001B7
:109B780002F098FA022385F8743000238AF800303E
:109B88003DE0AB7823B1C4F8B080AF70FFF760BB9D
:109B9800D4F8B030C3EB0803B3F57A6FFFF458ABD1
:109BA8000123D4F8B400AB7002F085FA0546D4F866
:109BB800B40002F080FA6D067FF44AAB8A2803D01D
:109BC8008E280ED0FFF744BB154B1B6899067FF50E
:109BD8003FAB94F8AC30002B7FF43AAB04F17C0334
:109BE80006E094F8AC30002B7FF432AB04F1480364
:109BF800C4F8B8302D2384F8BC30FFF729BB07B070
:109C0800BDEC028BBDE8F08FF42100202400002079
:109C1800A8210020082E00209CCA01081416002044
:109C2800542E0020482400200F2E0020F0B50124D7
:109C3800B0FBF4F58D4201D34C43F9E70026CCB1D3
:109C4800B0FBF4F504FB1500B4FBF1F41EB9002DCC
:109C580001DC002CF3D1092D03F1010E04DD002AEB
:109C680014BF3727572700E030273D441D700136C1
:109C78007346E4E71C70F0BD03685A1C0260197053
:109C880070472DE9F041002B069B06460F46144607
:109C980014BF4FF030084FF0200813F8012B0AB911
:109CA800254605E0002C01DD013CF6E7002408E02C
:109CB800002D04DD41463046B847013DF8E724EA67
:109CC800E474069D641B281915F8011B11B1304670
:109CD800B847F8E7BDE8F081F8B52A220021044624
:109CE80012F0B6FA0A49234604F128000522042690
:109CF800002511F9017F9F709A71DE715D7203F87A
:109D0800082F8342F5D10123A38052232370F8BD85
:109D1800CFCA0108014B186802F0D3B91C170020FC
:109D28000F4B1A78922A18D1598840F2F45291426E
:109D380013D11A79BE2A10D193F8E025EF2A4FF0F3
:109D480000000CD1074A13F8011B934280EA010076
:109D5800F9D1B0FA80F04009704700207047704789
:109D680000F00308F4F503082DE9F74FFFF7D8FFD3
:109D780010B904200BF0E4F8BC4CBD4EBD4D05F005
:109D8800D5F840F2F452BC4920460FF037FF94F85A
:109D98002835BA49022B84BF002384F8283594F863
:109DA80028256C235A43A31803F579733360A31845
:109DB80093F828340B700C2101FB0323234403F28E
:109DC8002A432B60A36846F209021A401AB9A74A27
:109DD80043F001039360A368D80703D54FF40050FC
:109DE80008F064FDA368590409D5082008F05EFD51
:109DF8004FF4005008F05AFD012008F057FDA36801
:109E08001A0706D54FF4005008F050FD012008F05D
:109E18004DFDA3689B0402D5402008F047FD984BF0
:109E2800984F1F604FF00009C8464FF0FF0A04EB37
:109E38000903B3F8B802410801F07731830803F049
:109E48003333C1EB000CC3EB0C01C30803F011332F
:109E5800CB1A03EB231310F0010E03F00F3292FB21
:109E6800FAF3C3EB032318BF08F10108A2EB0303BD
:109E780018BF5FFA88F8012B10DD022B40F0F18043
:109E8800BEF1000F02D010F0BC0F07D109F2B620C6
:109E980020440DF0A9FC002800F0E38009F108092E
:109EA800B9F1280FC3D108F1FF38B8F1010F00F25A
:109EB800D880DFF828922868734DDFF824A2494635
:109EC80006F0BCFD30220021281D12F0C1F93368CC
:109ED800AB630020C5F834900CF043FF6B4BB4F82B
:109EE800E011B4F8E22194F8DCC194F8DBE1C5F89C
:109EF8003CA080F001001870B4F8DE018842984652
:109F08009CBF0023A9F81231B4F8E43101939A42B6
:109F18009EBF564A0020A2F8E2015D4AB4F8DE016D
:109F280082F800C05B4AB4F8E2B110805A4AA2F83D
:109F380000B05A4A82F800E00EF0DEFD019B584A54
:109F48001946584682ED000A0EF0D6FD554B30688A
:109F580083ED000A0AF1F4032B640378012B14BF84
:109F6800514B524BC8F80430DFF87881C5F844806B
:109F780009F04CFE4E4B94F8AA029FED4E7AAF655D
:109F880008F180021A6064214B4BC82211FB0022A1
:109F98005A6000229A60DA601A615A619A61DA613D
:109FA80083F8202083F8212008F10E03AB64D4F84D
:109FB800F831EB64414BA8F1D6021A60A8F16603A8
:109FC8002B653F4BA8F5AA721A603E4BB4F81222D3
:109FD800C3F8009008F174036B65B4F8E63107EE36
:109FE800903AF8EEE77AB4F8E831C7EE876A07EEF8
:109FF800903AF8EEE77AC5ED196AC7EE876A94F8E1
:10A00800103285F85D3094F89C3285F868303368F2
:10A0180007EE102AC5ED186AB8EEC77ADFED2A6A8E
:10A028002A4AEA66C6EE877AA8F12E022A67284AE3
:10A038006A67A8F12A02EB67A8F10403C5F8802033
:10A04800C5F88430C5F88890C5F88C209FED217A32
:10A0580067EE877AC5ED1E7A03B0BDE8F04F04F0CD
:10A0680051BF1D48FFF738FE23E700BFB045002069
:10A078000C250020F43C002000F003088E2400206A
:10A0880094240020F44700201C1700209C00002086
:10A09800E42E0020E62E002014350020E82E0020B3
:10A0A8001835002070350020B7FE0008D9010108D6
:10A0B8006442002000401C46A424002030420020B6
:10A0C800B0410020B441002000006144781700200E
:10A0D8003661023D4C3D0F44644800207C46002018
:10A0E8009C470020DA470020F0B52D2646730F263E
:10A0F8004671222686710E26067435262825867610
:10A1080019262B22C572C671457221263725427041
:10A118003A211422162446748572532605754FF485
:10A12800FA7501234275817084753221C275C6762D
:10A1380000224B26C58546244FF42F7503700677F9
:10A14800867705860173C470017182730276C273C3
:10A158004276017281744284C37780F8283080F88F
:10A1680034301E23822580F83630C8234FF4827796
:10A17800458580F837302025DC238585878464254C
:10A18800A02703874FF08043C784C36380F84060EB
:10A19800058480F83320428780F8352080F84120F4
:10A1A800034600F124064FF00A0E40F2726783F866
:10A1B800465083F8475083F8482083F8491083F8BD
:10A1C8004A2083F84EE083F84F20A3F8507083F8B4
:10A1D8004B4083F84C4083F84D400C33B342E6D1F2
:10A1E800002380F84430F0BD2DE9F04F2DED028BAF
:10A1F800044640F2F452002183B012F029F840F6E8
:10A20800C412A4F8E621042284F8DA21022284F890
:10A21800EA215A2284F8DC2120204FF49672E24B7E
:10A22800A4F8E02184F8EC01C8226E20A360A4F809
:10A23800E2219223642284F816020A202370A4F8EB
:10A24800E42103234FF42F7284F817022B204FF4D4
:10A25800C8716371A4F836220023012284F8190218
:10A268002120A4F8DE1184F8D42184F8ED2184F8A3
:10A27800EE2184F8182284F82835A4F8E831A4F8E7
:10A28800D83184F8DB3184F8EB31A4F83A32A4F8F9
:10A298003832A4F83C3284F8C53184F8C63184F8E1
:10A2A800C73184F8D53184F81A0284F81C2284F85E
:10A2B800222284F8E12284F84D2284F84F2240F2C9
:10A2C800DC52A4F8542240F24C42A4F8562240F240
:10A2D8006C72A4F8582240F275322320A4F81E129A
:10A2E800A4F86022052140F643029FEDB08AA4F845
:10A2F800622284F81B02A4F82032A4F8243284F8DD
:10A30800E03284F8EC3284F8ED3284F8EE3284F8E6
:10A31800EF3284F8F01284F84C3284F84E32A046BA
:10A328002246032BCCBF0121002103F1010382F84F
:10A3380064120CBF05211E21122B82F8651202F14E
:10A348000202EED100231E2284F8503284F85122F2
:10A3580084F85232022284F85C32062384F85A22A6
:10A3680084F85D32132240F2465384F85B22A4F845
:10A378005E3204F5277204F523734FF47A704FF4B4
:10A38800FA6123F8040C23F8021C04339A424FF4B0
:10A398007A774FF4FA6AF4D1052384F89B321923AB
:10A3A80084F89C3240F22E43A4F8CC3040F27E531D
:10A3B800A4F8D63040F2EA53A4F8D83040F2B453A7
:10A3C800002501264FF4C872A4F8DA3040F2DC5BAD
:10A3D8003223A4F8A022A4F8DC30A4F8DE20A4F8E4
:10A3E800E03084F8985284F8995284F8A252A4F87C
:10A3F800D45084F8A55284F8A65284F8A85204F5DB
:10A408002D7084F89A6284F89E6284F89F6284F8BA
:10A41800A462A4F8CEA0A4F8D070A4F8D2B084F8AE
:10A42800E26084F8A76204F57979FFF755FC48469D
:10A43800FFF75AFE152284F800225D4A5D4BC4F8E6
:10A4480004225D4AC4F8F831C4F8082228235B4A7C
:10A45800A4F8F251A4F8F451A4F8F05184F8FC31AE
:10A4680084F8FD31C4F80C2204F51171544884F8BD
:10A478001062019304F0EAFC019B84F828324FF43F
:10A488004873A4F8123264220A2384F8265284F806
:10A49800275284F8145284F8AA3284F8AB3284F82C
:10A4A800AE5284F82962A4F8AC72A4F8B02284F8F9
:10A4B800B26204F1700023465A21FF25A3F85471B3
:10A4C800A3F856A1A3F858B183F85A2183F85B1171
:10A4D80083F85C1183F85D510E339842EED1002366
:10A4E80084F8C431C823A4F82A32142384F82C32FF
:10A4F8001E2384F82D32012384F82E326423A4F815
:10A5080030324FF49673A4F832322823A4F8343248
:10A5180004F1C00388ED038A08F110084345F9D116
:10A5280004F55D7538220021284611F091FE254A70
:10A53800002352F8230045F8230001330E2BF8D1ED
:10A548008022002104F53D7011F082FE24221E496C
:10A5580004F56D700FF052FB0B221C4904F5767060
:10A568000FF04CFBA36843F400230022A3600123EF
:10A5780084F8E32384F8D625494684F8D53584F849
:10A58800D33584F8D4356C2204F58A600FF036FB95
:10A598006C22494604F2BC4003B0BDEC028BBDE816
:10A5A800F04F0FF02BBB00BF0301080000000000B4
:10A5B8009A99193F00002041F6287C3F3D0A773FD1
:10A5C8001DF70108D6CA01080ECB010832CB0108D5
:10A5D80010B50B4C2046FFF707FE0A4B04F57972BD
:10A5E8001A60094A94F8283413700C2202FB0343BA
:10A5F800064A03F22A43BDE8104013600BF0F0BD91
:10A60800B04500200C2500208E240020F43C0020BA
:10A6180030B50278202A034600F10100F9D0092A52
:10A62800F7D02D2A03D10346BFEE000A04E02B2AF7
:10A6380008BF0346B7EE000A9FED377A1A46F2EED6
:10A64800046A134612F8010BA0F13001CCB2092CB0
:10A6580008D807EE901AF8EEE77AE7EE267AB0EE19
:10A66800677AEEE72E2816D1F2EE046A1146B0EEAC
:10A67800666A0B4611F8012B303AD0B209280AD87D
:10A6880007EE902AF8EEE77AC7EEA65A66EE866AD3
:10A6980037EE257AEDE71A7802F0DF02452A33D142
:10A6A8005A782D2A02D10233012004E02B2A14BF44
:10A6B800013302330020013B00220A2513F8011F51
:10A6C8003039CCB2092C02D805FB0212F6E7B2F5F4
:10A6D8009A7F28BF4FF49A72DFED106A1346F7EE9F
:10A6E800007A072B03D967EEA67A083BF9E702F050
:10A6F8000703F2EE046A1BB167EEA67A013BFAE79C
:10A7080020B1C7EE276A03E0F7EE007A67EE276A02
:10A7180020EE260A30BD00BF0000000020BCBE4C61
:10A72800B5EEC00ADFED2D7AF1EE10FACCBF30EEAF
:10A73800270A30EE670ADFED2A7A20EE270A30B5BD
:10A74800FDEEC07A87B017EE904A054684EAE470B9
:10A75800002303A9A0EBE47000930193029307F090
:10A7680087FD002CACBF20232D2303A88DF80030D3
:10A778000EF018FA012807D130238DF801308DF832
:10A7880002308DF803300CE0022805D130238DF813
:10A7980001308DF8023004E0032804BF30238DF81F
:10A7A800013003A9684611F07BFD68460EF0FAF9FE
:10A7B8000338C4B222466946284611F0CCFD00236E
:10A7C8002B550849284611F06BFD0DEB040128466E
:10A7D80011F066FD284607B030BD00BF6F12033A7E
:10A7E80000007A446218020870B506461546084605
:10A7F800B6FBF2F414B12046FFF7F6FF05FB14642C
:10A80800024B1B5D00F8013B70BD00BF26F7010835
:10A818002DE9F04F814689B08A4616461C46002528
:10A828003178002900F0DA80252901D001368EE040
:10A838007278302A08BFB278A2F1300319BFB71C6A
:10A848004FF0000BF71C4FF0010B092B4FF00008DD
:10A8580019D8A2F13003D9B2092905D80A2202FB76
:10A86800083817F8012BF4E7A2F16103052B02D889
:10A87800A2F1570305E0A2F14103052B03D8A2F189
:10A8880037030A2BEADD6C2A4BD13A78642A07F1A0
:10A89800010600F093800BD8252A57D003D8002A48
:10A8A80000F09C80BCE7582A0CD0632A33D0B7E765
:10A8B800732A3CD002D86E2A51D0B1E7752A5BD0F2
:10A8C800782AADD1A2F15800424204F1040705AB41
:10A8D800424110212068FFF7A9F93C460EE042D911
:10A8E800582A15D1A2F158014A424A41206805ABBD
:10A8F8001021FFF79BF9261D34463E4605AB009311
:10A9080042465B4651464846FFF7BBF9054487E790
:10A91800632A2AD13E4621784846271DD04701356B
:10A928000FE0642A38D00ED9732A14D13E46236822
:10A9380000934246002351464846FFF7A2F9271DD7
:10A9480005443C466CE7252AC9D13E4625214846A0
:10A95800D047013564E70AD86E2A06D13E462368F7
:10A9680004341D605CE7002A38D03E4658E7752A53
:10A9780007D0782AB6D0F8E7271D05AB00220A21B0
:10A98800A8E7231D0393002205AB0A212068FFF7DF
:10A998004DF93E46039CB1E72068231D0028039328
:10A9A8000ADA2D238DF8143040420DF115030022E8
:10A9B8000A21FFF73BF9ECE705ABF8E72068002828
:10A9C80004F1040708DA2D238DF8143040420DF104
:10A9D800150300220A217EE705ABFAE7284609B0ED
:10A9E800BDE8F08F0EB40FB505AB019053F8042BFA
:10A9F8000649039301A8FFF70BFF019B00221A7079
:10AA080004B05DF804EB03B0704700BF819C0008F8
:10AA18000FB437B50B4C06ABD4F8901053F8042B91
:10AA2800D4F894000193FFF7F3FE0546206801F07F
:10AA38003CFB0028FAD0284603B0BDE8304004B0FB
:10AA4800704700BF1C17002080EAE073A3EBE07397
:10AA58008B4206DB002801DD401A704702D008440B
:10AA6800704700207047DFED037A30EE270A0DF0BB
:10AA7800FFBE00BFDB0FC93F2DE9F341037823B9BF
:10AA880002B0BDE8F04106F0F5BA41490FF0C2F84E
:10AA9800002605463446B0464FF0FF376DB3012E09
:10AAA80007D0022E0AD00EBB28460FF077F80746CB
:10AAB8001CE028460FF072F8804617E03549284612
:10AAC80011F05CFC20B93449284611F057FC08B154
:10AAD80044F001043149284611F050FC20B93049AE
:10AAE800284611F04BFC08B144F002042849002024
:10AAF8000FF090F801360546D0E72A4B78B20C26BD
:10AB080006FB05F2D118D256824223D00135052D15
:10AB1800F6D1B8F1000F02D1394623480FE0002CD6
:10AB280008BF03240022E4B20192009443464FF484
:10AB3800807105F0E7FE054630B91C48394602B079
:10AB4800BDE8F041FFF764BF424639461848FFF7B1
:10AB58005FFF07E04D68002DDBD039461548FFF749
:10AB680057FF44B91448FFF753FF144B00222946F6
:10AB7800186806F01FFF69798C42F3D02246104806
:10AB8800FFF746FFE1B2284601F08CFAEAE700BF7A
:10AB9800AE0C02084BF70108390B02084EF7010802
:10ABA800310B0208AC4B002051F701087EF7010871
:10ABB8009CF70108B6F70108FDF70108144C0020BE
:10ABC800CDF701082DE9F04F8FB0554E0D91824613
:10ABD8000D46002796F8E4300A9396F8E530099375
:10ABE80096F8E730089396F9E68096F9E8300B93E3
:10ABF80096F8EA300C9396F9E9B095F8E43095F8B0
:10AC0800E52095F9E61095F8E70095F9E8E095F95B
:10AC1800E9C095F8EA90B8F1000F07D1DFF8008194
:10AC280040480DF005F90024C34642E00A9C9C42C6
:10AC380012D1099C94420FD188450DD1089C8442B9
:10AC48000AD10B9C744507D1E34505D10C9C4C45B2
:10AC580014BF0024012400E00024CDF814C0CDF86E
:10AC680010E003900291019200932F4ACDF81890BA
:10AC78003B46214650460DF0A1F80C9B06930B9BD2
:10AC88000493089B0393099B01930A9B0093CDF8B7
:10AC980014B03B46CDF80880234A21465046013778
:10ACA8000DF0ACF8102F06F1070605F1070591D154
:10ACB800B4E70E2666430BEB0603002508930D9BAD
:10ACC80033440127D3F85E2108EB0603AF40D3F8DD
:10ACD8005E31534037EA030314BF4FF001094FF0C8
:10ACE80000093A4206D000952346104A4946504684
:10ACF8000DF064F8089BD3F85E313B4206D000950E
:10AD080023460A4A494650460DF078F801350E2D7B
:10AD1800D5D10134082CCCD10FB0BDE8F08F00BFDD
:10AD2800B04500205D0D020855F8010874F80108C7
:10AD38002DE9F041334C88B080460D460027B4F920
:10AD48005421B5F954319A4295F95D211DD1B4F9D0
:10AD58005601B5F95611884217D1B4F95801B5F919
:10AD68005811884211D194F85B0195F85C1188421A
:10AD78000BD194F95A0195F95A11884205D194F9E1
:10AD88005D11881A4142414100E00021069295F97F
:10AD98005A21059295F85C21049295F85B2103925B
:10ADA800B5F958210292B5F9562101920093164A35
:10ADB8003B4640460E460DF001F894F95D31069386
:10ADC80094F95A31059394F85C31049394F85B3103
:10ADD8000393B4F958310293B4F956310193B4F995
:10ADE80054310093084A3B463146404601370DF03E
:10ADF80005F8082F04F10E0405F10E059FD108B0DF
:10AE0800BDE8F081B04500208BF80108F0B5017865
:10AE180085B0054609B1002417E0012005B0BDE85A
:10AE2800F04085E72D2B14D1072C19DC28460EF0AD
:10AE3800B5FE04AB661C03EB440424F8100C15F8AB
:10AE4800013F303B092BFAD934462B78002BE9D146
:10AE580004E0A3F13002092A07D8E5E7082C09D055
:10AE680005B0BDE8F04006F005B9202BF8D1013552
:10AE78002646E9E7BDF9002093B2072BF0D8BDF9C3
:10AE88000200A0F2EE239BB240F2DC54A342E7D8C2
:10AE9800BDF90410A1F2EE239BB2A342E0D8BDF99C
:10AEA8000640A042DCDCA142DADB8842D8DCBDF9EE
:10AEB8000C6006F164039BB2C82BD1D8BDF90E50C3
:10AEC800112DCDDCBDF908E01FFA8EF3B42BC7D8DD
:10AED800BDF90A70BBB2B42BC2D80A4B4FF00E0CA6
:10AEE8000CFB0233A3F85401A3F85611A3F85841F8
:10AEF80083F85BE183F85C7183F85A6183F85D51EC
:10AF080005B0F0BDB04500202DE9F74FDFF8A8A047
:10AF180007460E4600254FF0060808FB05F80024F2
:10AF280004EB080303EB0A02334492F8B49393F852
:10AF3800B4330193C3EB0901D1F1000B4BEB010BC7
:10AF480000942B461B4A594638460CF037FF8DE8CB
:10AF580010022B46174ADFF86090594638460134EC
:10AF68000CF04CFF062CDBD10135062DD3D106F2AF
:10AF7800D735002409EB0403384693F8D88315F82D
:10AF8800013F0193C3EB0802564256410094062341
:10AF9800084A31460CF012FF8DE810010623054AD5
:10AFA8003146384601340CF029FF0B2CE2D103B0AE
:10AFB800BDE8F08FABF80108B045002030B5017846
:10AFC80085B021B9012005B0BDE830409CE71C4997
:10AFD8000EF020FE002460B1032C0FD00EF0DEFD31
:10AFE80001AB174943F8240000200EF013FE01348A
:10AFF800F1E7032C02D1039B0F2B04D905B0BDE860
:10B00800304006F037B80199029AC8B2052809D825
:10B01800052AF3D80B4C062505FB0040104480F8A0
:10B02800B43307E00628E9D10A2AE7D805481044CE
:10B0380080F8D833044805B0BDE830400CF062BD54
:10B04800AE0C0208B0450020ABF801082DE9FF4717
:10B058001F4C804689460F460026A246B7F874134F
:10B06800B4F874338B420BD106F1DC039B000AEB76
:10B0780003024B44D288DD88531B5D425D4100E0EA
:10B08800002597F87733029397F87633114A8DE8BD
:10B098000A004046334629460CF090FE94F8773370
:10B0A800029394F876330193B4F874330093094A01
:10B0B80033462946404601360CF0A0FE102E04F116
:10B0C800040407F10407C9D104B0BDE8F08700BF44
:10B0D800B0450020C1F801082DE9F0410178054686
:10B0E80019B90120BDE8F041B0E70EF057FD0F286F
:10B0F80004462CDC284605F029FFDFF87C801C4F2D
:10B1080006460025DC3430460EF048FD38F8153088
:10B11800984223DC012D07EB840303D0022D03D0D2
:10B12800988002E0987100E0D87130462C2111F027
:10B13800C6F8064610B10136012302E0AA1E5342A2
:10B148005341013553B1032DDDD1BDE8F0810F2204
:10B1580000210848BDE8F04105F034BF044B03EB7B
:10B16800840400236360BDE8F04105F083BF00BF9D
:10B17800B0450020D5F8010840CB01082DE9F0477B
:10B18800DFF860A08EB0064601F53C79002409AFCF
:10B1980059F8045F5AF8043F03935B1B029539463C
:10B1A8005D4203A80DF110085D4106F039FC4146E7
:10B1B80002A806F035FC2346094ACDF80080294646
:10B1C80030460CF0FBFD23460097054A29463046D9
:10B1D80001340CF013FE202CDAD10EB0BDE8F08754
:10B1E800DBF80108A04800202DE9F04F017887B06E
:10B1F800054619B90120FFF7C1FFA8E00EF0CEFC03
:10B208001F28044600F39E80284605F09FFE04F19F
:10B21800BC030093009A4F4B019303EB8202002476
:10B2280007465460A046A246A146A34625462646A0
:10B23800494BE2B2E05C0023BE4617F8011B49B156
:10B24800884207D00A2B05D00DF10C0E03F80E101A
:10B258000133F1E706AF3B4488424FF0000703F89B
:10B268000C7C02D005F006FF71E0013A0EF10107EF
:10B27800032A0FD8DFE802F0130902450DF10B008D
:10B28800DFF8E4C04FF0010E2DE00DF10B014FF097
:10B29800010C15E003A80EF081FC064639E003A86E
:10B2A8000EF07CFC054634E00133062B08D02B4811
:10B2B80013F800E09645F7D10CFA03F349EA0309BD
:10B2C80011F8012F2AB30023F1E7254AD25C8A42FC
:10B2D8000ED1002212F80CA08A450ED10EFA02F205
:10B2E80048EA02089A4610F8011F91B10023ECE7DA
:10B2F8000133072BE9D15346EBE70132062AE9D19E
:10B30800F0E703A80EF04AFC0F28D4BF83464FF09D
:10B31800000B0134052C8BD105F00F059DE80C00BE
:10B3280045EA8B4545EA895949EA0A2A360103EB79
:10B3380082034AEA0838F6B248EA06065E600AF06E
:10B348004FFF04E01F220021064805F03BFE07B02E
:10B35800BDE8F08FB045002046CB010839E601086A
:10B368003FE60108D5F8010846E601082DE9F34152
:10B37800184D80460F460026B5F88822B7F888325F
:10B388009A42B7F88A2205D1B5F88A42A11A4C42E6
:10B398004C4100E00024019200930F4A33462146B5
:10B3A80040460CF00BFDB5F88A320193B5F88832A7
:10B3B8000093094A33462146404601360CF01EFDEB
:10B3C800042E05F1040507F10407D5D102B0BDE844
:10B3D800F08100BFB0450020E7F80108F8B5017812
:10B3E800054619B90120BDE8F840BFE7274910F024
:10B3F80037FFA8B9264B4FF47A714FF4FA62A3F8D5
:10B408008812A3F88A22A3F88C12A3F88E22A3F834
:10B418009012A3F89222A3F89412A3F89622F8BDEA
:10B4280028460EF0BBFB0328044627D8284605F01B
:10B438008DFD074620B10EF0B1FB0125064600E060
:10B448000546384605F082FD18B9BDE8F84005F014
:10B4580011BE0EF0A3FB012DF7D1A6F2EE2240F2A9
:10B46800DC539A42F1D8A0F2EE229A42EDD8084B6A
:10B47800A03403EB84031E815881F8BD0322002108
:10B488000448BDE8F84005F09DBD00BFAEFE0108C8
:10B49800B0450020B7FB01082DE9F04F2DED088BD2
:10B4A8003E4E8DB080460D46002796ED038AB5EED8
:10B4B800408AF1EE10FA6BD095ED030AD6ED049AA6
:10B4C80096ED059AD6ED068A95ED04BAD5ED05AA4E
:10B4D80095ED06AAB4EE408AF1EE10FA11D1F4EE19
:10B4E8004B9AF1EE10FA0CD1B4EE6A9AF1EE10FA1A
:10B4F80007D1F4EE4A8AF1EE10FA0CBF01210021BF
:10B5080000E000210AA80C46FFF70AF9B0EE4B0A42
:10B51800814608A8FFF704F9B0EE6A0A824606A831
:10B52800FFF7FEF8B0EE4A0A834604A8FFF7F8F8DA
:10B538003B461B4A039021468DE8000E40460CF01E
:10B548003DFCB0EE480A0AA8FFF7EAF8B0EE690A2F
:10B55800814608A8FFF7E4F8B0EE490A824606A833
:10B56800FFF7DEF8B0EE680A834604A8FFF7D8F8BC
:10B578003B4603908DE8000E094A214640460137B4
:10B588000CF03CFC0C2F06F1100605F110058CD1CF
:10B598000DB0BDEC088BBDE8F08F00BFB0450020B2
:10B5A800FAF801082DE9F041554E05462B7823B9E4
:10B5B80000210120BDE8F0416EE7052251492846E7
:10B5C80010F08BFE48B9504B002103F1C002D9603E
:10B5D80010339A42FBD1BDE8F08104224B4928463A
:10B5E80010F07BFE04462846002C40D105F0AEFC46
:10B5F8000746002800F082800DF0D4FA5FFA80F840
:10B6080056F8245025B94248BDE8F0410CF010BC6A
:10B6180042462946384610F060FE01340028EFD132
:10B62800394B002103F1C0029E46D96010339A427B
:10B63800FBD1384B03EBC404D4F810C0BCF1000FA5
:10B6480003D0002794F80C8005E029463248334D92
:10B658000CF058FAAAE74745F7DA3B010EEB03046A
:10B6680063440FCB0C3484E80F000137F3E70EF086
:10B6780095FA0B2806463AD8284605F067FC054691
:10B6880040B1FEF7C5FF204B03EB061383ED030A19
:10B69800012400E00446284605F058FC054638B168
:10B6A800FEF7B6FF184B03EB061383ED040A0134CB
:10B6B800284605F04BFC054638B1FEF7A9FF124BAA
:10B6C80003EB061383ED050A0134284605F03EFC1A
:10B6D80018B9BDE8F04105F0CDBCFEF799FF0A4B5B
:10B6E800032C03EB061686ED060AF2D160E70B225F
:10B6F80000210B48BDE8F04105F064BCBDE8F081CD
:10B7080094EB0108AEFE0108B045002010F90108CD
:10B7180015F9010840CB010824F901087FF5010853
:10B72800D5F801082DE9F047354C86B081460E461C
:10B7380000274FF0190896F879E594F8793596F8C6
:10B748007A2596F87B0596F87DC5734519D194F846
:10B758007A35934215D194F87B35834211D194F808
:10B768007C1596F87C3599420BD194F87D35634564
:10B7780007D196F87E1594F87E355B1A59425941DF
:10B7880000E00021CDF814C04FF4617A96F87C35BA
:10B79800049318FB00A018FB02A203900292CDF8B4
:10B7A80004E096F87E350093164A3B4648460D4617
:10B7B8000CF004FB94F87A3594F87B2594F87D1501
:10B7C800059118FB03A3029394F8793594F87C1536
:10B7D800019318FB02A294F87E350491039200931A
:10B7E800084A3B462946484601370CF007FB0F2F0D
:10B7F80004F1060406F106069DD106B0BDE8F087FF
:10B80800B045002030F90108F7B50178054619B9A7
:10B818000120FFF787FF6FE00EF0C0F90E280446FD
:10B8280065DC0023681C8DF8073005F08FFB334E6C
:10B83800054668B10EF0B2F9032809D8062303FBC0
:10B84800046383F87E059DF8073001338DF80730CF
:10B85800284605F07BFB074668B10EF09FF90D28D6
:10B8680009D8062303FB046383F879059DF807309C
:10B8780001338DF807300625654371190DF107026C
:10B8880001F27A51384605F06EFB05F05FFB07467A
:10B8980060B10EF083F9142808D8184B1D449DF8A0
:10B8A800073085F87C0501338DF80730384605F0F8
:10B8B8004DFB68B10EF072F90D2809D8062303FB79
:10B8C800046383F87D059DF8073001338DF8073050
:10B8D8009DF80730062B0FD0062303FB04640023D2
:10B8E800C4F87935A4F87D3505F0C4FB04E00E22D0
:10B8F8000021034805F066FB03B0F0BDB045002009
:10B90800D5F80108026BC168034610B5406942B119
:10B918001A6C8C1A013A005D08BF0A46C0B21A6454
:10B9280010BD1A6A805C01328A4228BF0022C0B268
:10B938001A6210BD436B13B190F844007047836AD4
:10B94800406A1B1A584258417047426A816A036923
:10B958008A4238BFD218521A416B21B149680A4449
:10B96800591E8A4203D2013B981AC0B27047002080
:10B978007047036B13B15968036C01E0C169036A2E
:10B98800994237BFC268C81A8818C01A704710F899
:10B998000A3C0133DBB20A2B00F80A3C07D910F83D
:10B9A800131C034A002322F8113000F80A3C7047A0
:10B9B800FC22002070B5524B1A78DD68013214243D
:10B9C800B2FBF4F004FB102298681A705A6C81429A
:10B9D8000A4404D293F84C0008B102F58032494871
:10B9E8000078B2FBF0F295420AD293F84C401CB1B1
:10B9F8004FF4803494FBF0F4501B041B1C6106E0E8
:10BA08004FF4803494FBF0F0401B104418619960A7
:10BA180093F85010DA6000241422013183F84C4066
:10BA280091FBF2F402FB141183F8501093F85110B3
:10BA38001C693348013191FBF2F502FB151283F8BA
:10BA4800512040F68C2294423DD9027990F9491050
:10BA58008A4214460CD1111F082909D890F84A10B7
:10BA680018299ABF013180F84A1080F8482002E06E
:10BA7800002183F84A1093F94800214982421AD1DB
:10BA880091F84B00B8B1204D10310020904205DAF2
:10BA980051F8046F25F810600130F7E71A490020C3
:10BAA8000C2C03D021F814000134F9E793F8521054
:10BAB800013183F8521083F84920002201211A71BC
:10BAC80083F84B1070BD90F84B20C2B1A4F2EF215F
:10BAD80040F2DA52914208D802790B2A05D800EBD5
:10BAE8008203013202715C6170BD002283F84B2031
:10BAF800064B03F1300143F8042F8B42FBD170BD94
:10BB0800B4170020A4000020FC220020C417002045
:10BB180010B50A4B1A7814240132B2FBF4F004FB76
:10BB280010221A705A6C01320A445A644FF6FF7296
:10BB3800914204BF012283F84C2010BDB4170020A5
:10BB4800024B53F820301B68196070474C400020A6
:10BB5800064B53F820301A681B89A1F57A715943AE
:10BB68004FF47A7391FBF3F1116070474C40002059
:10BB7800F0B5046D8668236823F001032360054649
:10BB880083796A7913F0020F0CBF00274FF400572E
:10BB980013F0040F14BF4FF48060002012F0010F5F
:10BBA80014BF042300239207226822F001022260B6
:10BBB800616821F4405141EA07016160226822F47A
:10BBC800B05222F00C0248BF43F00803024313436B
:10BBD8002360A36895B023F44073A360684602F01D
:10BBE8009FF8284B9C4201D10C9B0EE0264B9C42AF
:10BBF80001D10D9B09E0254B9C4201D10E9B04E02D
:10BC0800234B9C420CBF0F9B109B2268A8791704FA
:10BC180048BF5B00B3FBF6F206FB1233B3EB560FDB
:10BC2800236828BF01321E0441BF4FF6F073C2F3E8
:10BC38004201134041EA03026B7992B213F0020FFA
:10BC4800A28100F0010114BF4FF400320022DC078A
:10BC580048BF42F480322B6D11B159680A4302E0A3
:10BC6800596821EA02025A609A6801074CBF42F0FB
:10BC7800080222F008029A601A6842F001021A606B
:10BC880015B0F0BD003801400044004000480040B5
:10BC9800004C004041716BE7816069E7A1F57A715A
:10BCA80007EE901A084B9FED097A9FED090A53F8A1
:10BCB8002030F8EEE77A10B5A7EE870A1C680EF078
:10BCC8008DF9206010BD00BF4C400020EC51B83FFA
:10BCD8000000B443094B53F8203010B51C681823F2
:10BCE800594307EE901AB8EEE70AF3EE087A80EEA9
:10BCF800270A0EF073F9206010BD00BF4C400020E9
:10BD0800064B53F8203010B51C68CB0000EE103AF3
:10BD1800BAEEEE0A0EF062F9206010BD4C40002029
:10BD2800044B0146586D93F858300BB981F0010166
:10BD380006F036BBB4170020836A8169426B194448
:10BD4800D160416A8B4223BF0169CB1A5360CB1A79
:10BD58002ABF0023536083624FF0000380F8443009
:10BD6800136838BF816243F0010313607047436A68
:10BD78008269D154436A02690133934228BF002380
:10BD88004362436B1BB11B68DB0705D4D4E7026D24
:10BD9800136843F08003136070472DE9F0471D4690
:10BDA800B24B8EB09842884617469DF8586057D1D6
:10BDB800AF4CB04BE36504F5AC73236704F5167319
:10BDC80063674FF48073A366E366AB4BC4F89030A7
:10BDD800A3F54843203BC4F8AC00C4F8A8304E2073
:10BDE80004336266C4F8A4300AF0E8FD20200AF0A3
:10BDF800E5FD192006F0A6FA82461A2006F0A2FAF6
:10BE08004FF0010933462A460146CDF800905046C6
:10BE18000AF0F8FE99499A4B4869DA6D02434A617B
:10BE28005C34984A5A651C664FF0000A93F85930FA
:10BE38008DF80C3003A88DF80D908DF80EA08DF8B4
:10BE48000F900AF0BFFE252303A88DF80C308DF85B
:10BE58000D908DF80EA08DF80F900AF0B3FE76E0E5
:10BE6800894B984237D1824C824BC4F8B0304FF49A
:10BE78008073C4F8BC30C4F8C03004F55673C4F8F5
:10BE8800C430C4F8000104F58B637120C4F8B820ED
:10BE9800C4F8C8300AF092FD1E2006F053FA814615
:10BEA8001F2006F04FFA0223014600932A46334624
:10BEB80048460AF0A7FE26238DF80C3000220123FD
:10BEC80003A88DF80D308DF80E208DF80F30B034A2
:10BED8000AF078FE3BE06D4B984240F0C280644C1B
:10BEE800644BC4F804314FF48073C4F81031C4F8BB
:10BEF800143104F5AB63C4F81831C4F8540104F5DF
:10BF0800CB637220C4F80C21C4F81C310AF056FD2A
:10BF18002A2006F017FA81462B2006F013FA03238D
:10BF2800014600932A46334648460AF06BFE27230B
:10BF38008DF80C300022012303A88DF80D308DF800
:10BF48000E208DF80F300AF03DFE04F582744FF094
:10BF58000009012384F84430C4F82090C4F81C90E8
:10BF6800C4F82890C4F82490C4F82C806571A760A0
:10BF7800A6712046FFF7FCFDEA0739D5236B002B95
:10BF88002FD003A801F050FDE36C03934FF48053C6
:10BF98000C9380230893E368ADF8183020230B93A3
:10BFA800206B63690493CDF83490CDF81C90CDF8DC
:10BFB8002490CDF82890CDF8149001F060FD03A9E5
:10BFC800206B01F03EFD236B216D1A6842F00102DF
:10BFD8001A608A6842F040028A605B689BB22364F8
:10BFE80006E0236D20221A621A6842F020021A60C5
:10BFF800AB072FD5636B43B303A801F015FDA36C02
:10C0080003934FF480530C93802308932369ADF86E
:10C01800183000251023606B05930D950795099539
:10C028000A950B9501F02BFD03A9606B01F009FD42
:10C03800636B1A6842F002021A60226D5D605D60EF
:10C04800936843F08003936004E0226D136843F023
:10C0580080031360226D136843F0010313602046C8
:10C0680000E000200EB0BDE8F08700BF00380140B6
:10C07800B417002024D101084400024000100240F7
:10C08800A4000020D9740008004400400048004083
:10C0980003685B6A03B11847704703681B6A03B1FA
:10C0A8001847704703689B69184703685B69184716
:10C0B80003681B6918470368DB68184703685B68EF
:10C0C800184703681B6818470368DB692DE9F041C6
:10C0D80004460E46174693B90D467B1B3344002B86
:10C0E8000BDD236820469B6898470028F9D015F88F
:10C0F800011B2046FFF7E5FFEFE7BDE8F081BDE84B
:10C10800F04118471FB50123ADF808300023ADF8FA
:10C118000C30ADF80A30094BADF8041093F85837D5
:10C12800ADF80620012B08BF032301A908BFADF80D
:10C138000C3001F031FD05B05DF804FBB4170020A8
:10C1480038B510F80E2C50F8043C044652B90122B8
:10C1580000F80E2C20F80C1C597918680222BDE84A
:10C168003840CFE730F80C2C20F80A1C891A89B21D
:10C1780020F8081C074A10F80F0C002522F81010A8
:10C1880004F80E5C2A4659791868FFF7BBFF04F8D3
:10C19800065C38BDFC220020054B03EB8003D3F876
:10C1A8005C371BB107289CBF1B681960704700BF2C
:10C1B800B417002070B547200CF0F6F8174B184C50
:10C1C8001B6813F4002F06D06368164A1B681068B2
:10C1D800C01A0CF0A3F9144E144D30780CF09EF9E7
:10C1E800E3682868C01A0CF0A8F923696868C01ABF
:10C1F8000CF0A3F90E4B18880CF090F90D4B188829
:10C208000CF08CF90C4B18880CF088F933782377EC
:10C218002B6863616B68A36170BD00BF580C002078
:10C22800301F0020E03D00204A1600204C16002058
:10C238004816002046160020080F002038B5354B58
:10C2480035481C68354B1B682360354B1A6862609B
:10C258005A689B68E360334BA2601A6822615A6887
:10C268009B68A361304B62611A68E2615A689B68F7
:10C2780063622E4B22621A8822855A8862859A88C0
:10C28800DB88E3852A4BA2851A6822865A689B6850
:10C29800A386284B62861A68E2865A689B68638779
:10C2A800254B22871A88A2875A88E2879A88A4F899
:10C2B80040202246DB8822F8423F204B1978002391
:10C2C8008B4205DA30F9135022F8025F0133F7E7A1
:10C2D8001B4B1B88A4F86C301A4B1B88A4F86E30D3
:10C2E800194B1A68A4F874205A689B68A4F8783027
:10C2F800164BA4F876201B6823670BF07DFB144BC4
:10C30800E0671B88A4F88030124B5B89A4F866307C
:10C3180038BD00BF301F00207C400020E03D0020D9
:10C32800BC2B0020C82B0020D42B00201C2500206B
:10C338003025002020160020CC2100203F25002099
:10C34800C821002030400020543E00203016002034
:10C35800C44D0020F80E00202DE9F04FC34BC44F08
:10C368001888C44C8BB00093002840F0C18097F81F
:10C37800D335012B05D197F8D405A0F120025042FE
:10C38800504100F001000AF093FEFFF757FF2568BF
:10C39800DFF8E8B249200CF007F8B74B2E461868CA
:10C3A8000CF0BCF856F8040B0CF0B8F830460AF05C
:10C3B800CBFC05F110000AF0C7FC05F11C094FF091
:10C3C80010084FF0010ADBF80020AC4E0AFA08F317
:10C3D800134203D0D9F800000CF0AFF808F10108B7
:10C3E800B8F1130F09F10409EDD1032105F1280073
:10C3F8000CF0A7F8B7F8CC30B5F92E00C01A0CF03D
:10C408008DF83368DB0408D59D4BB5F86C001B88A4
:10C41800181AC0F30D000CF081F83368980403D59E
:10C42800B5F86E000CF07AF83368590504D5032185
:10C4380005F174000CF085F833681A0502D5286FE9
:10C448000CF07BF833685B0402D5E86F0CF075F8E4
:10C458003368180403D5B5F880000CF05FF80321A1
:10C4680005F130000CF06DF8A846032105F13600FF
:10C478000CF067F8042105F13C000CF062F838F97B
:10C48800440FB7F8CC30DFF814A2C01A0CF046F805
:10C498004FF001099AF80030994509DA38F9020F86
:10C4A800B5F94430C01A0CF048F809F10109F1E770
:10C4B8003368990505D5B5F96600A0F2DC500CF093
:10C4C8003CF822686F486260A260121A91106E4AA6
:10C4D8004A43531C032293FBF2F202EB42029A1ADC
:10C4E800842303FB02032360684B01221A7021E2B4
:10C4F800674B1D68D4F8AC319D420FD0654BC4F82A
:10C50800AC511B78093B012B08D845200BF04CFF98
:10C5180000200BF049FF28460CF000F85E4BD4F8D9
:10C52800B0611D68B54213D0524BC3F8B051594B96
:10C538001B78093B012B0BD845200BF035FF1E203B
:10C548000BF032FF28460BF0E9FF30460BF0E6FF10
:10C55800009B97F8D3151B8897F8D4050B44013B2B
:10C56800B3FBF0F200FB1233994240F2AE81012096
:10C578000AF09EFDFFF762FE5020266865680BF002
:10C5880013FF2268A36810681B6862680344106878
:10C59800A3EB40000BF0D1FF06F1040E281D002389
:10C5A80050F823105EF82320521A02A941F82320DC
:10C5B8000133032BF4D108460AF0C6FB06F1100E2E
:10C5C80005F11000002350F823105EF82320521ABA
:10C5D80002A941F823200133032BF4D108460BF0BC
:10C5E8000DFF264A06F11C0B05F11C094FF0100837
:10C5F8004FF0010A13680AFA08F0184208D0DBF86D
:10C608000000D9F800300192C01A0BF096FF019A89
:10C6180008F10108B8F1130F0BF1040B09F1040933
:10C62800E8D106F1260005F12601002331F902EFD1
:10C6380030F9022FCEEB02020DF1080E4EF823203E
:10C648000133042BF2D103214FF0000A4FEA8A0389
:10C658005FFA83FA02AB53F8212042B302F10800D3
:10C668000F281DD84AF0010A21E000BF600C002005
:10C67800B0450020301F0020640C0020580C00201A
:10C688005C0C0020501F0020E1830F3ED90E0020D3
:10C6980040400020EA2C0020D42400203F25002020
:10C6A8008032FF2A94BF4AF0020A4AF0030A11F1C5
:10C6B800FF31CBD250460BF077FE4FF0000B0DF157
:10C6C8000809D8460AF00301022916D003291ED00A
:10C6D80001293BD1D9F80000B8F1000F04D10001BD
:10C6E8005FFA80FB884631E000F00F0040EA0B005B
:10C6F8000BF05AFE4FF0000828E0B8F1000F0DD0FB
:10C70800D9F80000C0F3031040EA0B0017E0B8F1B5
:10C71800000F08D199F801000BF046FE99F80000C7
:10C728000BF042FE12E0D9F80000C0F3033040EAF3
:10C738000B000BF039FED9F80000C0F307100BF01E
:10C7480033FED9F8001009015FFA81FB09F10409E9
:10C7580006AB4B454FEA9A0AB4D1B8F1010F02D1A2
:10C7680058460BF021FE784B1B6813F4805807D00D
:10C77800B6F86C20B5F86C10521A02924FF0010806
:10C788009A040BD50AAA02EB8801B5F86E00B6F830
:10C798006E20121A41F8202C08F10108580514D50A
:10C7A80002AA02EB880C06F1720E05F17200002253
:10C7B8003EF9021F30F9029FC9EB01014CF8221023
:10C7C8000132032AF4D108F10308190509D50AAA88
:10C7D80002EB8800296F326F521A40F8202C08F1BA
:10C7E80001085A0409D50AAA02EB8800E96FF26F1A
:10C7F800521A40F8202C08F1010818040CD50AAB8D
:10C8080003EB8802B5F88010B6F880305B1A42F85E
:10C81800203C08F1010802E0B8F1000F22D0B8F17D
:10C82800010F03D102980BF088FE1BE008F1FF33DB
:10C83800002002AA400052F82320C0B20AB140F0FA
:10C84800010013F1FF33F4D20BF0AEFD4FF00009F5
:10C8580002AB53F8290008B10BF06FFE09F101098A
:10C86800C145F5DB032130200AF07CFC032136208A
:10C878000AF078FC04213C200AF074FC334B442075
:10C8880019780AF06FFC304B1B68990506D5B6F984
:10C898006600B5F96630C01A0BF04FFE22682C48C6
:10C8A80063686260121A91102A4AA3604A43531CB3
:10C8B800032293FBF2F202EB42029A1A842303FB4F
:10C8C80002032360244B01221A70244B1B681A06AA
:10C8D80030D5234DE2682968224B91420BD1696813
:10C8E8001A69914207D1009A1288102A11D1B3F817
:10C8F800B4315B060DD148200BF056FD28680BF0CB
:10C908001CFE68680BF019FE2B68E3606B682361F6
:10C918000EE0154A217F1278124B914208D1134A32
:10C9280059691068884203D152689B699A4201D0BC
:10C93800FFF740FC97F8D535012B01D10AF07AFDB5
:10C948000BB0BDE8F08F00BF580C00203F25002039
:10C95800501F0020E1830F3ED90E002098240020AC
:10C9680008170020301F00204A1600204C1600200F
:10C978000C4A1388013313800B4A13680133136080
:10C988000A4A138801339BB2202B03BF002313806C
:10C99800074A138002BFB2F8B4310133A2F8B431A8
:10C9A800704700BF5E0C0020640C0020600C002063
:10C9B800301F00202DE9F74FC2EB030817460E9BE6
:10C9C8000D9A4C4C9B1A00936368002914BF0626E5
:10C9D8000426013305468A4624D123689E4240F244
:10C9E8008580DFF82CB15BF823000CF0DBF80B3006
:10C9F8000BF000FC814608B1012078E021683E4830
:10CA08005BF82120032994BF294651460BF0BAFC54
:10CA18003A4A1368181A6368106001336360384B28
:10CA280083F8B691DFF8D490DFF8D4A063680C9A45
:10CA3800304D934242DA0D9A4AB1009A0D995A4301
:10CA4800895C01228A402F4909680A4232D003FBD7
:10CA580008F5236807EB050B23B978590CF0A2F801
:10CA6800431D00E00323184601930BF0C3FB002885
:10CA7800C2D1D9F80000019BC01A9AF8B631C9F89A
:10CA880000001BB12C200BF08FFC02E001238AF878
:10CA9800B631236843B978590BF004FC9BF90410AC
:10CAA8004B1C07D0184803E09B4418489BF8041017
:10CAB8000BF068FC636801336360B7E710D10120AD
:10CAC8000BF098FB60B90D4A13680A20013B13600C
:10CAD8000BF06AFC2B6801332B604FF0FF336B605F
:10CAE8002068864294BF0020012000E0002003B0A7
:10CAF800BDE8F08F500C002050F90108480C0020C8
:10CB0800301F0020580C00205FF901089FFA010827
:10CB18004CD10108124A38B513780B2B144617D894
:10CB280001229A4040F603051540BDB912F4C06FC2
:10CB38000ED0093B012B0BD845200BF035FCFF200C
:10CB48000BF032FC07480BF0ADFB28460BF02CFC31
:10CB5800054B1A68054B5A600B23237038BD00BF7C
:10CB6800EA2C002064F9010884240020500C0020DD
:10CB7800F0B51A4A58B113885B08012B98BF48F2E0
:10CB8800050313800B6803F5C333A0330B601388C8
:10CB980013F0010320D1124C124D134E1349144FB8
:10CBA8002278934218DA2A6852F82320C2F307320F
:10CBB80050074FEA830E05D412070BD53A680B3A93
:10CBC8002B2A07D891F8DC2301EB8202D2F87403F0
:10CBD8004EF806000133E3E7F0BD00BFE82000206F
:10CBE800C04D0020C40800201A4D0020B045002088
:10CBF800BC4D00202DE9F043264B274CC8B11A78CC
:10CC0800F02A0FDD7F221A70A07893F90120824262
:10CC180001DA002A02DA987840429870987802443B
:10CC28005A7001E00F321A700A6802F582421A320D
:10CC38000A601A4A18781568247893F9016093F9FC
:10CC48000270DFF85C800022A0F17F0EC0F1FF0CBB
:10CC58001146A2421CD255F822309B0416D5CBB2FD
:10CC68009B1B83EAE379A9EBE379B9F1010F05DCB2
:10CC780033B1BB4214BF6346734602E0082300E0A9
:10CC8800034608EB8209013189F803300132E0E7F5
:10CC9800BDE8F083C8010020C04D0020C408002072
:10CCA8001A4D00202DE9F047244E70B1244A93789C
:10CCB80003B9F378013BDBB29370224B1A68224B1D
:10CCC80093FBF2F30A6813440B60204D1B4FDFF807
:10CCD80080E0DFF880C0DFF8689000210C46A5F5F9
:10CCE8003C783378994227DA55F8040FC0F30323C8
:10CCF800062B1FD19EF800305B070DD599F802303E
:10CD080097F803A0234493FBFAF20AFB1233012B92
:10CD1800CCBF0023012303E004F0010383F00103E7
:10CD28003BB1C0F3834008EB8000D0F874034CF8A3
:10CD3800210001340131D4E7BDE8F087C04D00205F
:10CD4800E8200020BC4D002080841E00A048002060
:10CD5800D82400201A4D002008B509480BF022FFFE
:10CD6800084AC0B220210928034604DC13440130D4
:10CD7800C0B2D970F7E7034B18440023C37008BD4D
:10CD8800EB200020E820002008B509480BF00AFF36
:10CD9800084BC0B22022142804D8411C1844C27081
:10CDA800C8B2F8E7034B18440023C37008BD00BF9E
:10CDB800EB200020E82000202DE9F8432C4C20B37C
:10CDC8002C4B08681B78DBB12B4AB2F90230B2F958
:10CDD8000020002BB8BF5B42002AB8BF52429342E2
:10CDE800B8BF13461933322BB8BF3223234A92FBFC
:10CDF800F3F303440B60637E83F00103637604E07E
:10CE080000F5433303F5A0730B60637E73B31A4BCD
:10CE1800B3F90020192A04DC1A32CCBF0024C0243C
:10CE280000E03024B3F90230192B02DD44F050043D
:10CE380003E01933B8BF44F0A004114E114FDFF8D6
:10CE48004880DFF8489000253B789D420EDA56F876
:10CE5800043FDB0308D5284609F082F920421CBFAD
:10CE6800D9F8003048F825300135EDE7BDE8F883FA
:10CE7800E8200020C41400201C250020809698007B
:10CE8800A0480020C04D00201A4D0020E2CA010829
:10CE980030B41E4CA8B11E4B9A7E0AB1013A09E083
:10CEA800D87E257885428BBF0130DA76D876042281
:10CEB80088BF01229A760B6803F5C32303F5207314
:10CEC8000B602278134B1AB1134A1268900602D4E9
:10CED80093F8DD1310E011490D4A0978927E89070D
:10CEE80006D512B993F8DF1306E093F8DB1303E0D5
:10CEF800002AEDD193F8DE1303EB810303F55D718E
:10CF08004FF4A06030BC09F0B3B800BF4A16002047
:10CF1800E8200020B0450020542E002044160020B0
:10CF2800154AA8B1154B18886423434340F2FF30D3
:10CF380093FBF0F3322B03DD00231377012003E08A
:10CF4800142BCCBF02200820137F83F00103137732
:10CF58000B4B93FBF0F00B681844137F086053B930
:10CF6800084B93F8DB1303EB810101F55D714FF476
:10CF7800806009F07DB87047E8200020C44D00208B
:10CF880040420F00B0450020124A70B1124B1B7886
:10CF980023B1012B0CBF0220082001E053770120A8
:10CFA800537F83F00103537700E001200B4B93FB81
:10CFB800F0F3086803440B60537F53B9084B93F8A8
:10CFC800DB1303EB810101F55D714FF4407009F04B
:10CFD8004FB87047E82000208824002040420F0006
:10CFE800B0450020642928BF6421F8B510FB01F57D
:10CFF8006424064695FBF4F40027E4B2FBB29C4295
:10D0080004D99F2006F0FDFE0137F7E7A6420BD9A9
:10D01800C4EB84101421C4EB800095FBF1F5663D48
:10D028002844C0B206F0EDFE0134E4B2B44201D2A5
:10D038009A20F7E7F8BD2DE9F0432DED028B9A4CC5
:10D048008FB007F035FF236AC31A002BC0F2AB83F9
:10D0580000F5433303F5A0732362944B94F824201E
:10D068001D7805F00405EDB2002D14BF012300233F
:10D0780084F8243009D0934200F095838C4B5A7879
:10D088009A7001225A701A702CE09342884A05D08F
:10D09800D37843F00203D37093785370D67806F0B0
:10D0A800020101F0FF0339B981498968411A002951
:10D0B80003DB06F0010300E0012303F001077C49CC
:10D0C80017707BB1F2070DD50A790132D2B2072366
:10D0D800B2FBF3F3C3EBC303D31ADBB2754A0B718C
:10D0E800D35C4B70724EDFF81882337883B3F378D1
:10D0F80023F00203F370704B0344AE20B3600BF0CF
:10D1080074F808B106F00EFE88F80000002800F058
:10D118004A83B0200BF069F840200BF066F8002035
:10D128000BF063F810200BF060F84FF48067013FB4
:10D138000020BFB20BF054F8002FF8D1384606F0A3
:10D1480080FE72785B4B03EB8203986806F070FEF2
:10D1580098F80030002B00F026837378082B00F233
:10D16800EF82DFE813F00C00ED021D0082000900D9
:10D1780037019E011102D9020026504F26E1504B7B
:10D18800504A51495148FDF72DFC012006F059FE3F
:10D198004E4806F04DFE022006F053FE4C48B3E21E
:10D1A8004C4F3B689B073AD5DFF85881DFF8589118
:10D1B800B8F8001045480A23B1FBF3F203FB121339
:10D1C80099F8001000919BB292B24349FDF70AFC0E
:10D1D800FFF7DAFD012006F034FE3C4806F028FE91
:10D1E8003E4B99F800201968B8F800300E79C978D4
:10D1F80006FB1230891B642343435143B3FBF1F10F
:10D208006429A8BF642121EAE171CEB2022006F0A8
:10D2180018FE31461520FFF7E5FE032600E001263B
:10D228003B681F0540F18C822D4B2E481968006819
:10D2380000906423254891FBF3F203FB12132A495B
:10D24800FDF7D0FBFFF7A0FD304606F0FAFD1F48BA
:10D2580006F0EEFD00F0AEFF0746701C06F0F1FD8B
:10D2680039461520FFF7BEFE6AE201201F4F06F07F
:10D27800E8FD1F4806F0DCFD3B68980746D51D4BC6
:10D288001D499A6801925A6800921B681B4A0F4808
:10D29800FDF7A8FBFFF778FD022006F0D2FD0B484A
:10D2A80006F0C6FD032632E0E8200020D82400203E
:10D2B8001C4C002064D10108404B4C00342E002047
:10D2C80024EF01082CEF01088EF90108EB2000205B
:10D2D80019EF01089824002097F90108A4210020DB
:10D2E80040160020A8210020AFF90108542E002084
:10D2F800C4F9010820160020DEF90108DAF901084E
:10D3080080080020F42100204005002002263B6808
:10D31800D90717D5884B89499A6801925A680092AB
:10D328001B68874A8748FDF75DFBFFF72DFD3046F0
:10D3380006F087FD834806F1010806F079FD5FFADB
:10D3480088F846463B681A0715D57F4B7B499A688B
:10D3580001925A6800921B687C4A7A48FDF742FBA2
:10D36800FFF712FD304606F06CFD7648771C06F094
:10D378005FFDFFB23E46764A0A20B2F90030B2F9A4
:10D38800041091FBF0F10191B2F9022000926B496F
:10D39800704A6C48FDF726FBFFF7F6FC3046B0E113
:10D3A8000E2E00F0CD817008013006F04AFD30469F
:10D3B80004F0D8FA3B78B34206D9202006F021FDC4
:10D3C800701CC0B204F0CEFA0236F6B23B78B34213
:10D3D800E6D8B5E1604E614996F828255948FDF729
:10D3E80001FB012006F02DFD564806F021FD5C4B9F
:10D3F8003746D3F800905B4E4FF0000899F8152097
:10D4080099F80130019299F80B20574900924D483C
:10D4180056F82820FDF7E6FAFFF7B6FC08F10200F7
:10D42800C0B206F00EFD08F10108464806F000FDFE
:10D43800B8F1030F09F10109E0D14C4B4C491E78B2
:10D4480040483246FDF7CEFA052006F0FAFC3D4882
:10D4580006F0EEFC6C227243BB180C2693F82814D5
:10D46800384806FB0123FE18424996F82A3496F8F4
:10D478002C24FDF7B7FAFFF787FC062006F0E1FC3D
:10D48800304806F0D5FC96F8311496F8303496F802
:10D498002F242C4800913849FDF7A4FAFFF774FCB3
:10D4A8002EE1012006F0CDFC34489FED358A06F0C8
:10D4B800BFFC0026022705A9F0B200F0F5FE9DF892
:10D4C8001C30ABB3052E33D0DDED0D7A0A9B0C98DA
:10D4D800B8EE677A42F2107EC8EE077A07F10108C3
:10D4E8005FFA88F8FDEEE77A17EE902A00FB02F162
:10D4F8005A4301F59C5102F59C5208310832B1FBA0
:10D50800FEF1B2FBFEF202918DE805001D490D48BF
:10D518003246FDF767FAFFF737FC384606F091FC0C
:10D52800084806F085FCB8F1080F00F20981474663
:10D538000136102EBFD103E130250020DEF90108A5
:10D54800EDF90108EB200020543E0020160B0208DC
:10D5580028250020F1F90108B0450020F5F9010857
:10D568000C25002090D1010801FA01088E24002022
:10D5780016FA010827FA010838FA01084AFA0108D8
:10D588000024744960FA0108894B1B681B0640F1A6
:10D59800BE80A36AE16A874A8B4207D0D36292F8B9
:10D5A8003030013303F0030382F8303001210020CA
:10D5B80006F054FC94F830307F4ADFF85C82D05C87
:10D5C80006F01FFC0121022006F048FC0026362741
:10D5D80018F80630C3EBC30090FBF7F0C0B206287A
:10D5E80028BF06206038C0B2013606F00AFC102EAB
:10D5F800EED1724B724A1B78127872497248734E98
:10D6080013F0020F14BF59234E23FDF7EBF9FFF770
:10D61800BBFB022006F015FC6B4806F009FC6C49C0
:10D628006C4A4B68684893FBF2F3096891FBF2F285
:10D638006949FDF7D7F9FFF7A7FB032006F001FCBE
:10D64800614806F0F5FB654B65491A885E48FDF7A9
:10D65800C9F9FFF781FB042006F0F3FB5A4806F0EE
:10D66800E7FB604B60491A885748FDF7BBF9FFF79D
:10D6780073FB04210A2006F0F1FB534806F0D8FB9F
:10D68800626B5A495048FDF7ADF9FFF765FB052075
:10D6980006F0D7FB4C4806F0CBFBB36872685449D8
:10D6A8004948FDF79FF9FFF757FB05210A2006F0C7
:10D6B800D5FB454806F0BCFB3369F2684D49424842
:10D6C800D21AFDF78FF9FFF747FB062006F0B9FBE2
:10D6D8003D4806F0ADFBB26847493B48FDF782F983
:10D6E800FFF73AFB06210A2006F0B8FB364806F099
:10D6F8009FFB1522414934480EF02DFEFFF72CFB05
:10D70800072006F09EFB304806F092FB18E0F378FD
:10D7180043F00203F37013E0394F002637F916304F
:10D728003849294832460136FDF75CF9FFF72CFBEA
:10D73800F0B206F086FB244806F07AFB042EEDD101
:10D74800002D30D1304B93F82030052B9BBF2F4A4A
:10D758009B183F2593F838500021122006F07EFBD5
:10D76800284606F04EFB1320002106F077FB284BD5
:10D778001B78002B274B1B7814BF72202120002B0D
:10D7880018BF522006F03DFB0021142006F066FB6E
:10D7980094F83850084B585D013505F0030506F03C
:10D7A80030FB84F838500FB0BDEC028BBDE8F08335
:10D7B80098240020E820002070FA01084416002070
:10D7C8004A16002075FA0108EB200020743E00205C
:10D7D8004C1600208096980086FA0108461600200C
:10D7E80093FA0108080F00209BFA0108A2FA010821
:10D7F800A9FA0108B2FA0108B9FA0108A00800203C
:10D80800CC210020C1FA0108A424002064D1010819
:10D81800C4140020721500203C0F0020064B186825
:10D8280040B19A6864214A43B2FBF0F29A80002220
:10D838001A609A60704700BF2421002003788B4249
:10D8480083BF034B03EB410188890020704700BF69
:10D858002421002070B5324C054607F029FB636A85
:10D868006062C31AB3F5FA5F82BF002384F82830D8
:10D8780084F8293094F828302BB9A12D02BF284A02
:10D88800012182F8291094F82910254A31B1D118BC
:10D89800EDB2013381F82A5082F8283094F82850E4
:10D8A80094F84B30AB4239D11D4B93F84C30052BD3
:10D8B80002D0062B03D02CE0002001F075FA94F872
:10D8C8002B301E2B25D100210B46013DCAB2AA429E
:10D8D80017DA2244184692F82A201346082283EAC7
:10D8E80000065B0816F0010FDBB202F1FF3218BF29
:10D8F80083F08C0312F0FF02C0F34700EFD101312F
:10D90800E4E7254495F82A20934202D1032001F048
:10D918004BFA002384F8293084F8283070BD00BF02
:10D92800242100202DE9F8431E4B1F4E81460F4647
:10D938000025F61ADFF87C8008EB0504237903F04C
:10D9480030034B4527D1204604F0A4FC55F8088045
:10D95800164A0146434638460AF030FA50B1204686
:10D9680002F082FA0022811920460AF0DFF81048F6
:10D978000AF05EFA204604F08DFC434601460B4A45
:10D9880038460AF03BFA30B1204600210AF030F957
:10D9980007480AF04DFA1435B5F5666FCAD1BDE8E7
:10D9A800F88300BFB0450020F435002010FB0108C3
:10D9B8005D0D0208A4D10108022810B50C4613D841
:10D9C80005F038F809480AF033FA09480AF034F93A
:10D9D80008480AF02DFA21461020FFF7A3FF044853
:10D9E800BDE810400AF00FB910BD00BF1AFB0108CE
:10D9F8007FF501085D0D020810B50C4604F05EFFC6
:10DA080006480AF015FA06480AF0FDF805480AF033
:10DA18000FFA21462020BDE8104083E728FB0108C3
:10DA28007FF501085D0D02080023036043608360F1
:10DA38008381036143618361C361036243628362DB
:10DA480070470A6A036810B58C6814430A6914435E
:10DA58004A6914438A691443CA6914434A6A1443D5
:10DA68008A6A23F4FF4323F07003224313430360BD
:10DA78008B8943600B6883604B68C36010BD026884
:10DA88004FF6FE7313400360002303604360836016
:10DA9800C360294B984201D1284A27E0284B984275
:10DAA80001D1264A2AE0274B984201D1234A2DE08A
:10DAB800254B984201D1214A30E0244B984201D1AC
:10DAC8001E4A33E0224B984204D11C4A536843F45F
:10DAD80070032EE01F4B984204D1184A536843F054
:10DAE800706326E01C4B984204D11C4A536843F0EB
:10DAF8000F031EE01A4B984204D1184A536843F0AA
:10DB0800F00316E0174B984204D1144A536843F4C3
:10DB180070630EE0144B984204D1104A536843F4E2
:10DB2800704306E0114B984204D10C4A536843F401
:10DB380070235360704700BF080002400000024095
:10DB48001C000240300002404400024058000240DD
:10DB58006C000240800002400804024000040240B9
:10DB68001C040240300402404404024058040240AD
:10DB7800084BDA68D10709D4DA68D20608D4DB681A
:10DB880013F0040F14BF03200420704701207047CE
:10DB98000220704700200240F0B50C884A888B8824
:10DBA8000E89CD88C4B9016A21F001010162846936
:10DBB800016A24F0F3041C4321F00A0142F0010237
:10DBC80044EA06130A4383610262836923F00C0363
:10DBD800836183691D431FE0042C1FD1046A4FF63B
:10DBE800EF71214001628469016A1B0224F47344C5
:10DBF80043EA06331201234342F010024FF65F74E2
:10DC08000C4092B2144383610462836923F4406335
:10DC18008361836943EA05258561F0BD082C046AA0
:10DC28001DD14FF6FF6121400162C469076A4FF6B2
:10DC38000C7121404FF2FF543C4043EA061344EA7A
:10DC480002220B4342F480729BB292B2C361026219
:10DC5800C2694FF6F3731340C361C3691FE04EF600
:10DC6800FF7121400162C469016A40F6FF472740FD
:10DC780045F6FF740C40310341EA032344EA0232BB
:10DC88003B4342F480529BB292B2C3610262C269C2
:10DC98004FF2FF331340C3612D02C369ADB21D4378
:10DCA800C561F0BD036A23F001030362036A426899
:10DCB80030B584690D6824F4803424F073042C434F
:10DCC8008D8923F002032B438D882B43134DA842E3
:10DCD8000FD005F50065A8420BD005F54065A842B0
:10DCE80007D005F58065A84203D005F58065A842F0
:10DCF8000DD1CD8923F008032B43CD8823F00403ED
:10DD08002B430D8A22F440722A434D8A2A434260EB
:10DD18008A6884614263036230BD00BF002C014001
:10DD28009A4A536803F00C03042B2DE9F04105D0FF
:10DD3800082B06D096490160B3B916E0944B0360EE
:10DD480012E053685468C3F38343991CE30349BF43
:10DD5800D36A904B8E4C03F00F0344BF0133B4FBDE
:10DD6800F3F34B43036000E0002351688A4FC1F38B
:10DD780003117E5C0168F6B221FA06F44460556826
:10DD8800C5F3022517F805E024FA0EFEC0F808E0EE
:10DD98005568C5F3C2257D5DEDB2EC40C460D2F88C
:10DDA8002C804FEA181808F00F0C07EB4C0C18F0F1
:10DDB800100FBCF810C01FFA8CFC07D0BCF1000F84
:10DDC80004D0B3FBFCFCC0F810C000E00161D2F83D
:10DDD8002CC04FEA5C2C0CF00F0807EB48071CF02E
:10DDE800100F3F8ABFB204D01FB1B3FBF7F74761EA
:10DDF80000E04161176BFF065ABF654F876181617B
:10DE0800176BBF065ABF624FC761C161176B7F06A8
:10DE18005ABF5F4F07620162176BFF0506D58B4239
:10DE280004D1AE4202D15F00476200E04462176B42
:10DE3800FF0406D58B4204D1AE4202D15F0087624F
:10DE480000E08462176BBF0506D58B4204D1AE4251
:10DE580002D15F00C76200E0C462176B7F0506D578
:10DE68008B4204D1AE4202D15F00476400E04464B3
:10DE7800176B3F0506D58B4204D1AE4202D15F0035
:10DE8800876400E08464176BBF0406D58B4204D115
:10DE9800AE4202D14B00C36400E08464156B3B4B77
:10DEA800AD0701D1046315E01C6B04F00304012CD9
:10DEB80001D101630EE01C6B04F00304022C02D1B3
:10DEC8004FF4004305E01B6B03F00303032B01D160
:10DED8002F4B0363146B2D4B14F4403F02D1C0F851
:10DEE80034E018E01C6B04F44034B4F5803F01D1F1
:10DEF800416310E01C6B04F44034B4F5003F02D1D8
:10DF08004FF4004306E01B6B03F44033B3F5403F86
:10DF180001D11F4B4363146B1C4B14F4402F02D1E7
:10DF2800C0F838E018E01C6B04F44024B4F5802FE6
:10DF380001D1816310E01C6B04F44024B4F5002F78
:10DF480002D14FF4004306E01B6B03F44023B3F502
:10DF5800402F01D10E4B8363146B0C4B14F4401FFC
:10DF680002D1C0F83CE021E01C6B04F44014B4F585
:10DF7800801F01D1C16319E01C6B04F44014B4F58F
:10DF8800001F0BD14FF400430FE000BF0010024008
:10DF980000127A0000093D00CC0100201B6B03F43D
:10DFA8004013B3F5401F01D1134BC363126B134BDE
:10DFB80012F4400F03D1C0F840E0BDE8F0811A6BBD
:10DFC80002F44002B2F5800F02D10164BDE8F0818D
:10DFD8001A6B02F44002B2F5000F02D14FF400436D
:10DFE80006E01B6B03F44003B3F5400F01D1024B6D
:10DFF8000364BDE8F08100BF00127A0000100240FF
:10E008002DE9F04300230F681A464FF0010E03264E
:10E018000EFA02F939EA070430D191F804C00CF17C
:10E02800FF34012C18D8846891F8058006FA03F5A6
:10E0380024EA05048460856808FA03F848EA0505B7
:10E0480085608488A4B224EA090484808C79858850
:10E0580094402C43A4B28480056806FA03F4E44390
:10E068002540056005680CFA03FC4CEA05050560C7
:10E07800C5682540CC799C402C43C4600132102AE5
:10E0880003F10203C4D1BDE8F083074B5A694FF48A
:10E098007A73B3FBF2F3C3EB431203EB8203034A35
:10E0A800DB00A2F84E307047CC2E0020242100203F
:10E0B80038B52DED048B13460D4607C83B4C84E854
:10E0C80007009A1E503C062A05D8DFE802F0080C23
:10E0D80012191E222600236D2B60636D0DE0636DFF
:10E0E8002B60236D03E0236D5B422B60636D5B4205
:10E0F80003E0636D5B422B60236D6B60A36D14E0DE
:10E10800236D5B422B60636D0CE0636D2B60236DA8
:10E1180008E0236D2B60636D03E0636D5B422B6049
:10E12800236D5B426B60A36D5B42AB60204B93F841
:10E138003030C3BBD5ED007A94ED1A0AB8EEE79AF1
:10E14800D5ED017AB8EEE78AD5ED027A28EE000A15
:10E15800F8EEE78AD4ED177AA7EE890AD4ED1D7A8E
:10E16800A7EEA80A0BF03AFF94ED1B0AD4ED187A33
:10E17800286028EE000AA9EE270AD4ED1E7AA8EE38
:10E18800A70A0BF02BFF94ED1C0AD4ED197A6860EE
:10E1980028EE000AA9EE270AD4ED1F7AA8EEA70AEE
:10E1A8000BF01CFFA860BDEC048B38BD7421002067
:10E1B800CC010020104B9FED117AD3F88020D3F8C2
:10E1C8008430D28983F31003D31A07EE903AF8EE1D
:10E1D800E77A67EE877A07EE102AF8EEC76A87EEC5
:10E1E800A67AFDEEC77A17EE900A6428A8BF6420C5
:10E1F80020EAE070C0B27047242100200000C84225
:10E20800094BD3F88020137844F6FB7103EB4313D2
:10E2180000FB03135078C0EB0030B3FBF0F39078A9
:10E22800B3FBF0F080B2704724210020F7B51C4BF7
:10E238001B4E93F88A2093F8A67003EB4202022F34
:10E24800B2F89C50ADB2A3F8A4501C4608BFA3F87E
:10E25800A85093F8B03053B94CF250319FED110AE1
:10E2680006F1B4000AF042FC012386F8B03007EE4C
:10E27800905A0B4EB8EE670A06F1B4000AF0ACFBF0
:10E28800FCEEC07ACDED017ABDF80400FFF7B8FFC7
:10E29800022FA4F8D00008BFA6F8AA0003B0F0BD6A
:10E2A80024210020CDCCCC3E164A34234343F0B57C
:10E2B800D418656B0D60A46B134D4C6002F13404E7
:10E2C8002344D5F8D4600024D835B44205DA55F88B
:10E2D8002470BB4203D00134F7E7002300E0012398
:10E2E8000B72342303FB0020436CCB6090F848305A
:10E2F8000B74036E4B61436E8B61836DCB61C36D91
:10E308000B62F0BDCC01002024210020F8B51A4D85
:10E31800D5F8D4400F2C07462BDC002305F1D80292
:10E328009C4205DD52F823108F4222D00133F7E7D3
:10E33800DFF848E00022A2421BDC5EF822100F48FA
:10E348009600531C71B98119A21A2E44920000EB51
:10E35800830001340DF061FFC6F8D870C5F8D440C9
:10E368000120F8BD91F814C0397D8C45EBD31A46CD
:10E37800E1E70020F8BD00BF24210020FC21002097
:10E38800112870B506D00F282AD8164B342202FB64
:10E39800003002E0144BD3F81C0109B1C36823B95B
:10E3A800114B0022D3F8D44003E0BDE87040ADE73C
:10E3B8000A46A24214DA0C4D05F1D803960053F828
:10E3C8002210884202F10101F2D1A21A920003EB55
:10E3D80081019819013C0DF020FFC5F8D44070BDAB
:10E3E80070BD00BF000200202421002007299ABF29
:10E3F800024B33F821000020704700BF4422002060
:10E40800024B03EB4101088CC008704744220020EE
:10E4180003788B420BD9074B1A78074B89001944AC
:10E42800086C02B1400800F5777080B27047002090
:10E43800704700BF382E0020442200200A4BDFED31
:10E448000B7A03EB810191ED1C7AB8EE477AF6EE70
:10E45800046AE7EE267A82B0FCEEE77ACDED017A1F
:10E46800BDF8040002B070474422002000005C445C
:10E4780000207047024B03EB4101B1F8B800704728
:10E4880044220020024B03EB4101B1F8B800704769
:10E4980044220020024B03EB4101B1F8D000704741
:10E4A8004422002003788B4283BF034B03EB4101D6
:10E4B800B1F8F4000020704744220020024B03EB1F
:10E4C8008101B1F8140170474422002010B50446B8
:10E4D80006F0EEFC0E4BD3F84C21C3F84C01821A1F
:10E4E80041F288318A4284BF002283F8502193F890
:10E4F800502107491344142A18BF013283F85141A7
:10E5080012BF81F85021012381F8663110BD00BF88
:10E518004422002038B5044606F0CAFC274A274999
:10E52800D2F86831C2F86801C31AB3F57A6F84BFAC
:10E53800002382F86C3192F86C3133B9A82C3BD1A6
:10E5480081F86D31A1F86E3106E0022B02D181F815
:10E55800704101E0242B02D8D11881F8714192F85A
:10E568007011164D01330231DBB249008B4282F83B
:10E578006C3118DAB5F86E31E0B283EA002008236E
:10E5880010F4004F4FEA400018BF80F4815003F1A7
:10E59800FF3318BF80F0010013F0FF0380B2EFD102
:10E5A800A2F86E0138BD01318B4201BF002385F806
:10E5B8006C31012385F86D3138BD00BF442200203D
:10E5C80010B5044606F074FC104BD3F89821C3F834
:10E5D8009801821A41F288318A4284BF002283F866
:10E5E8009C2193F89C31094A0F2B0DD8591CC9B2AC
:10E5F80013441029E4B283F89D4114BF002301237A
:10E6080082F89C1182F8AD3110BD00BF4422002071
:10E6180010B5044606F04CFC124BD3F8B02140F676
:10E62800AC51821A8A42C4BF002283F8B42193F8FD
:10E63800B4212AB90F2C13D10A49C1F8B00101E05D
:10E64800182A0DD8511CC9B283F8B41113441929DA
:10E65800044883F8B54114BF0023012380F8CE3164
:10E6680010BD00BF4422002038B5384C054606F0DE
:10E678001FFCD4F8D031C4F8D001C31AB3F57A7F9F
:10E6880009DD0023282284F8D43184F8D52184F8C0
:10E69800D63184F8D73194F8D4312C4A83B93D2D3A
:10E6A80007D03E2D50D1012182F8D61102F5EE7126
:10E6B80004E0012182F8D71102F50171C2F8D811DE
:10E6C800D4F8D811214ACD540133DBB2062B84F893
:10E6D800D4311CD192F8D631012B02D18B78282B5A
:10E6E80007D994F8D731012B06D18B78092B03D899
:10E6F800164A82F8D53138BD0023282284F8D4314F
:10E7080084F8D52184F8D63184F8D73138BD92F809
:10E71800D511994218D192F8D6310C4D012B04BF6E
:10E72800022382F8D63194F8D731012B06D102237F
:10E7380085F8D73106F0BCFBC5F81002002384F831
:10E74800D431282384F8D53138BD00BF44220020B5
:10E7580038B5044606F0ACFB2249D1F81432C1F8AA
:10E768001402C31AB3F5FA7F84BF002381F8183264
:10E7780091F818221B4B1ABB93F81902F0B9552CC3
:10E788000CD101201F2583F81A0283F8194283F857
:10E798001B52A3F81C2283F81E0211E0202C1FD163
:10E7A800022083F81E024FF6FF7083F81A2283F8BE
:10E7B800194283F81B42A3F81C0201E084420FD1DE
:10E7C8008B18084883F81F4291F81B32013B9A4284
:10E7D80003D1012380F83F3238BD013280F8182276
:10E7E80038BD00BF4422002008B5044809F020FBCA
:10E7F8000120BDE8084009F0D7BB00BF4B0602085E
:10E8080007B5064B0193064B0093064A064B07498A
:10E81800074809F077F903B05DF804FB24EF010815
:10E828005AEF01082CEF010863EF010819EF0108FE
:10E83800640602082DE9F74329492A4C08882A4F1B
:10E8480094F84412294B2A4A57F821101B78128849
:10E85800D4F8405200916428A8BF642001904FF476
:10E868007A712448B5FBF1F109F04CF948212248A6
:10E87800DFF8A49009F046F9204BD3F80080002572
:10E888001F4B53F82510D9B10126AE4016EA080FE0
:10E8980014D0330712D015F809201A480C2303FBAB
:10E8A800052307EB83031A6B09F02CF9022E05D117
:10E8B800154B997A11B1154809F024F90135DFE7AC
:10E8C800134809F0B5FAB4F84622B4F848121148CA
:10E8D80040F2F45392B203B0BDE8F04309F012B924
:10E8E800282100204422002004E0010840050020DF
:10E8F800F421002086060208D3060208542E0020C0
:10E9080014E00108E3060208442E0020EB06020882
:10E918005D0D0208EF0602085C0500202DE9F347AB
:10E928001E481F4C1F4D09F0EDF804F5EA77A3794E
:10E9380094F8089005EB83032046D3F8F060E37958
:10E9480005EB8303D3F85881B9F1000F11D003F018
:10E9580044FD8246204603F036FDCDF80480024689
:10E96800CDF8009033460AF141010F4809F0CAF882
:10E978000EE003F032FD8146204603F024FDCDF879
:10E9880000800246334609F14101084809F0BAF807
:10E998000C34A742CBD102B0BDE8F08721070208AA
:10E9A800DC43002004E001083F0702085107020881
:10E9B8002DE9F0472DED028B48489FED498A90B02C
:10E9C80009F0A0F800244FF47A792646A046CA46F2
:10E9D80007A9E0B2FFF768FC9DF82430002B67D048
:10E9E800012C1CD13F4BB3F8483207EE903AF8EEB1
:10E9F800677A3D4B88EE277A93F8EA51012DFDEEB0
:10EA0800C77A17EE907A02D997FBF5F511E0079BC4
:10EA1800089A3648214609F075F83D460EE0DDEDC6
:10EA28000F7AF8EE677A88EE277AFDEEC77A17EE46
:10EA3800905A079A2E48214609F064F80C9A0E9BC2
:10EA480005FB02F003FB05F100F59C50052C00F1D5
:10EA5800080001F59C51B0FBF9FE0D98B0FBFAF0E7
:10EA680004904FF00A0001F10801B1FBF9F191FBA4
:10EA7800F0FC18BF761800FB1C1103919EFBF0F107
:10EA880000FB11E001900091CDF808C02946194813
:10EA980018BFF04409F036F8012C09D1124B93F84D
:10EAA800EA31012B04D93A460899134809F02AF8A3
:10EAB8000134102C8CD10A2296FBF2F302FB136668
:10EAC80098FBF2F1009602FB11820C4809F01AF843
:10EAD80010B0BDEC028BBDE8F08700BF61070208EB
:10EAE8000024744944220020B0450020BA070208D7
:10EAF800AB070208CC070208F2070208040802085C
:10EB08002DE9F8430024144E8146254654F8068022
:10EB180049464046A7190DF031FC88B141460F48D7
:10EB280008F0F0FF0021384609F062F80C4809F0B7
:10EB38007FF9384609F08AF9094809F079F9013569
:10EB48001434B4F5666FE1D125B90648BDE8F84339
:10EB580009F06EB9BDE8F883A4D1010814FB0108D7
:10EB68005D0D020815F901082DE9F04F2DED028B16
:10EB780083B007460AF016F8054620B1012818D1D7
:10EB88003B782A2B15D17D487D4E09F051F9002498
:10EB9800A1597C48A71908F0B5FF2946384609F05D
:10EBA80027F81434784809F043F9B4F5666FEFD1C3
:10EBB800DFE03D2138460DF082FB002800F0D280CE
:10EBC800054615F8013C202B05F1FF3201D1154609
:10EBD800F7E7ED1B0130824601309AF80030202B10
:10EBE800F9D0674C4FF000081423EDB203FB08F28C
:10EBF800019352F804904846161909F0D3FF494684
:10EC08000246834638460DF068FB019B002840F019
:10EC18009B80AB4540F09880357915F0C0030FD044
:10EC2800402B40F08680594A337B9FED598A02EB8E
:10EC3800C303044693F8A8B1014602461F4634E0D0
:10EC480050460AF0ABFF04465046FBF7E1FCD6ED10
:10EC5800037AF8EEE77AB0EE408AB4EEE70AF1EE0E
:10EC680010FA66DBD6ED047AF8EEE77AB4EEE70A36
:10EC7800F1EE10FA5DD805F00F03052B18BF08EE6A
:10EC8800104A16E099B9D7F8A4310192514653F8C1
:10EC980024000DF0E5FA002808BF08EE104A019A92
:10ECA8000ABF01210021012201345C45EAD3002A70
:10ECB8003FD0334A142303FB082805F03002102AFA
:10ECC80018EE101AD8F8083006D1324A92F82805FA
:10ECD8006C2200FB02330EE0202A0CD12D4A92F858
:10ECE80028452D4A92F84A2202EB420292006C20F3
:10ECF80010FB0422134405F00F02052A0CD8DFE8A4
:10ED080002F0030305050709197005E0198003E0FF
:10ED1800196001E083ED008A4946204808F0F2FEB8
:10ED28000021304603B0BDEC028BBDE8F04F08F07F
:10ED38005FBF1B4809F07CF8304603B0BDEC028B7E
:10ED4800BDE8F04F09F082B808F10108B8F1B80F32
:10ED58007FF44CAF134803B0BDEC028BBDE8F04F15
:10ED680009F066B8384603B0BDEC028BBDE8F04F39
:10ED7800C6E603B0BDEC028BBDE8F08F340802088C
:10ED8800A4D1010814FB01085D0D020804E0010884
:10ED980000000000B0450020442200204908020875
:10EDA8005408020815F90108F0B50021244D0B4656
:10EDB8004218234CAA5C082683EA022313F4004F66
:10EDC8004FEA430218BF82F4815206F1FF3618BF9A
:10EDD80082F0010216F0FF0693B2EFD10131192932
:10EDE800E6D100F11902A15C00F11A02A25C02EB63
:10EDF800012292B29A4222D11249334691F84B52DB
:10EE0800114E01304FF4AF67DAB2954214D900EBD6
:10EE180042025FFA82FE14F80EC00EF1010E14F8D9
:10EE28000E2002EB0C2292B27A43121302F54872BA
:10EE380026F813200133E7E7012381F84C32F0BDAF
:10EE48004E21002044220020302100202DE9F041ED
:10EE58000A4E05460F46441E06F1080814F8011F1D
:10EE680051B106480DF02BFA0028F7D040453EBFB7
:10EE7800801B631B3B54F1E7BDE8F08124E60108E1
:10EE8800094B93F84D225AB9D3F850220749527EBC
:10EE980009780432D2B28A4228BF0A4683F84D2242
:10EEA80093F84D02704700BF44220020342E002002
:10EEB800124910B5D1F8503203EB400292F82040C5
:10EEC80014B1022C10D00BE0022805D9032807D171
:10EED800D1F85422D20401D5188A10BD988B10BDE0
:10EEE800074B33F8100010BD92F8210000EB8000AA
:10EEF80000EB800000F2EE2080B210BD442200201A
:10EF0800E42D002008B505F0D3FF074B022283F853
:10EF18005C22D3F84022C3F868220122C3F85802C1
:10EF280083F8812208BD00BF4422002008B505F0FF
:10EF3800BFFF084B022283F85C22D3F8682200F551
:10EF4800B71000F5587002F2DC52C3F85802C3F843
:10EF5800682208BD4422002030B50C4D0446002329
:10EF6800221AD2B291420ED914F8012B53409A00BA
:10EF780082EA43025A40DB0803F0180345FA03F318
:10EF88005340DBB2ECE7184630BD00BF0007090E5E
:10EF980070B5064604460020A31BDBB299420ED981
:10EFA80014F8013B434083EA0313DBB2020ADD0095
:10EFB80042EA032285EA131382EA0300ECE770BDF4
:10EFC8000C4B93F88402012810B51C4606D004D3D4
:10EFD800022805D107F053FE02E0002007F05CFE8E
:10EFE80005F066FF00F5F42000F59070C4F888027B
:10EFF80010BD00BF442200204849B1F88C22D1F846
:10F0080090322DE9F04F02F0080003F4475404430E
:10F0180003F4804012F0010F44EA000403F40040B6
:10F0280014BF4FF0020A4FF0000A044312F0020F17
:10F0380003F4803014BF4FF004094FF00009044373
:10F0480012F0040F03F4003003F4802514BF4FF0CE
:10F0580010084FF00008044312F0400F44EA05047A
:10F0680014BF4FF0200C4FF0000C03F4002012F0F6
:10F07800100F40EA040014BF4FF4007E4FF0000E5A
:10F0880003F4801412F0200F14BF4FF48067002798
:10F09800044312F4807F91F8940214BF4FF4006681
:10F0A800002603F0285312F4007F14BF4FF4001514
:10F0B8000025C0F3800012F4806F43EA040242EA9C
:10F0C800000242EA0A0242EA090242EA080242EA65
:10F0D8000C0242EA0E0242EA070242EA060242EA49
:10F0E800050214BF4FF0806B4FF0000B002091F821
:10F0F800956242EA0B02034601F296210125B342CA
:10F1080009D25C5C05FA04F414421CBF05FA03F446
:10F1180020430133F3E7BDE8F08F00BF442200200D
:10F1280038B50D4C23689842054606D101F0D5FB49
:10F138004C22002120460DF08BF8E36CAB4209D13C
:10F14800284601F0CAFB4C2200210448BDE838409B
:10F158000DF07EB838BD00BF3C2D0020882D002062
:10F16800044BD3F8B422D379591C1344D171187ABB
:10F17800704700BF4422002010B5FFF7F1FF84B2AA
:10F18800FFF7EEFF04EB002080B210BD10B5FFF7CB
:10F19800F3FF0446FFF7F0FF04EB004010BD38B55D
:10F1A800064D04460146D5F8B80203F04FFBD5F8E2
:10F1B800B43298796040987138BD00BF442200206D
:10F1C80010B5064CD4F8B4329879FFF7E8FFD4F8B4
:10F1D800BC02BDE81040FCF75BBF00BF4422002022
:10F1E80070B5104C0646D4F8BC020D46FCF755FF26
:10F1F8002420FFF7D4FF4D20FFF7D1FF002E14BFC6
:10F2080021203E20FFF7CBFFD4F8B4320022284655
:10F218009A71FFF7C4FFD4F8B432BDE8704093F890
:10F228004900BCE74422002001460020D8E710B579
:10F238000446C0B2FFF7B3FF200ABDE81040AEE7AE
:10F2480010B5044680B2FFF7F2FF200CBDE810406D
:10F25800EDE700BF064B93F8E225002A054A03F2C2
:10F26800E25306BF012113460021034A08F0C6BD38
:10F27800B0450020C80B0208CA0B02082DE9F74F59
:10F28800824609F08FFC474D0446D5F8D875B8B9C1
:10F298004548464E08F036FC012505FA04F33B4282
:10F2A80006D00C2303FB04634148996808F02AFC44
:10F2B8000134122CF1D1CFB93E4808F0B9FD15E060
:10F2C80002463D49DFF8E49050460DF006F8064640
:10F2D80070B93A4808F0ACFD344609EB04033448E9
:10F2E80099680C3408F00EFCF02CF6D134481FE075
:10F2F8009AF800302D2B03BF0AF1010A04F1FF34FC
:10F308004FF0010B4FF0000B4FF000080C2303FBEC
:10F318000892504696680193224631460CF0DDFF6C
:10F32800019B50B108F10108B8F1140FEFD125483D
:10F3380003B0BDE8F04F08F07BBDBBF1000F14D05F
:10F34800B8F1120F01D1204B04E0B8F1130F04D12A
:10F35800D5F8DC35C5F8D83505E0012202FA08F3FE
:10F368001F43C5F8D875194812E0B8F1120F02D139
:10F37800C5F8D8B50BE0B8F1130F1DBF012303FA88
:10F3880008F39F43C5F8DC7518BFC5F8D875104851
:10F3980008F04EFD0F48314603B0BDE8F04F08F0C5
:10F3A800B1BB00BFB0450020D40B0208A4EA010895
:10F3B800E50B0208DE0B0208EA0B0208EF0B020855
:10F3C8005D0D020815F90108FFFF0300FA0B02089A
:10F3D800030C020859110208F0B585B0054609F07A
:10F3E800E1FB082827D16E1EEF1D16F8014F0AF021
:10F3F800E9FB2044437803F00303022B08BF203CB9
:10F40800B7423470F1D12C4605F1080714F8016BA6
:10F41800164831460CF053FF20B1314620460CF017
:10F428004EFF10B101F026FE1DE0A742EED11049B3
:10F438002846FFF70BFD0F480F4C08F0F9FC0B4866
:10F4480000231A1904A992F844220A44195C02F804
:10F458000C1C0133082BF4D1002301A907488DF8AF
:10F468000C3008F04FFB05B0F0BD00BF24E60108E2
:10F47800F44700200B0C0208B04500205A1102087E
:10F488002DE9F84F814609F08DFB2F4E0446D6F83A
:10F49800088098B92D482E4D08F0CAFC012655F869
:10F4A800241049B106FA04F313EA080F02D02948D8
:10F4B80008F028FB0134F2E7274824E002462749F0
:10F4C80048460CF00AFF58B92548264C08F0B0FC0D
:10F4D80054F8041F0029EFD01E4808F013FBF7E783
:10F4E80099F80030DFF868B02D2B03BF09F1010946
:10F4F80004F1FF344FF0010A4FF0000A00255BF8D1
:10F50800257027B91848BDE8F84F08F091BC224685
:10F51800394648460CF0E1FEA0B90120A840BAF1EE
:10F52800000F03D003F0C2F9104803E040EA0800D6
:10F53800B0600F4808F07CFC39460E48BDE8F84F2B
:10F5480008F0E0BA0135DAE7B0450020110C0208EE
:10F5580004E401081B0C02085D0D0208EA0B02080E
:10F568001F0C020800E4010815F90108FA0B02084B
:10F57800030C02085911020838B5054609F012FBB8
:10F58800044690B1112200210A480CF061FE22467F
:10F59800094928460CF0CAFE38B1102C22462946E3
:10F5A80028BF102203480CF0D6FE0120BDE83840E1
:10F5B80050E600BF924B0020C80B020808B50B4864
:10F5C80008F0A0FA07F082FF094B00221A705A705F
:10F5D8005A6007F03BFE18B9642005F0A7FCF8E76D
:10F5E8000448BDE8084008F08DBA00BF2B0C02089B
:10F5F80004250020380C02082DE9FF410A48048838
:10F60800856846888788D0F80C8007F0FFFD8DE86C
:10F618008001029033462A462146044808F072FACF
:10F6280004B0BDE8F08100BF44050020400C02088A
:10F638002DE9F041A14C88B00546284609F0B2FAF8
:10F64800C1B229B9012008B0BDE8F041FBF7BABA48
:10F6580005229B4928460CF040FE064690B9014613
:10F66800702298480CF0F4FD974930460E24324633
:10F6780004FB001301300828A3F85E21A3F86021D9
:10F68800F6D118E10422914928460CF026FE0646D8
:10F69800002849D1284601F059FC0746002800F007
:10F6A8000A8109F07FFA35465FFA80F854F8256038
:10F6B8002EB9874808B0BDE8F04108F023BA4246A1
:10F6C800314638460CF009FE01350028EED17E4B54
:10F6D80003F170021F4683F8EA0083F8E60083F816
:10F6E800E50083F8E40007339A42F4D1794B03EB41
:10F6F800C505002295F860C0624510DA686EC2EB55
:10F70800C20307EB030E034401321868CEF8E40085
:10F718009888AEF8E8009B798EF8EA30ECE7314635
:10F728006D4808F0EFF9BFE007226C4928460CF055
:10F73800D4FD0646002872D1202128460CF0BFFDD2
:10F74800074609F02FFAC5B275BB654808F0DAF923
:10F758002C4621466348013408F0D4F90E2CF8D120
:10F768006148594F08F0CEF9002421465F48DFF878
:10F77800908108F0C7F90E26002506FB0476D6F816
:10F788005E215B495B480123AB401A4218BF4146E2
:10F79800013508F0B7F90E2DF1D15348013408F0BE
:10F7A800B1F9082CE1D186E0534938460AF032FA1B
:10F7B800354600287AD0022D09D00AF0EFF94E49D3
:10F7C8004DF8250000200AF025FA0135F1E7009BE5
:10F7D800072B20D8019A0D2A1DD8017872290DD03F
:10F7E8006E2918D138490E2000FB0313012101FAB4
:10F7F80002F2D3F85E1121EA020209E032490E2032
:10F8080000FB03130121D3F85E0101FA02F202435F
:10F81800C3F85E2101E001F02DFC304D0DE72846CC
:10F8280035490AF0F7F9002558B1082D3ED00AF0FD
:10F83800B5F931494DF8250000200AF0EBF90135FA
:10F84800F2E7082D32D1009B0F2B2FD8DDF804E00A
:10F85800BEF1070F2AD8029F0D2F27D8039E06F165
:10F868006402C82A22D8049DFF2D1FD8059964294F
:10F878001CD8069A642A19D8914217DA07980328DF
:10F8880014D8DFF844C0C3EBC303634483F8E4E04F
:10F8980083F8E57083F8E66083F8E75083F8E810AA
:10F8A80083F8E92083F8EA00144DC6E608B0BDE8FD
:10F8B800F04101F0DFBB08B0BDE8F08194EB01082E
:10F8C800AEFE010894460020B045002010F901085A
:10F8D80015F9010804E4010824F901089D0C02083F
:10F8E800C2110208A50C02085D0D02089FFA010862
:10F8F800CE040208AA0C0208AE0C02087FF5010823
:10F908008DFD010870B5044608460D4609F04AF910
:10F918002946024620460CF0E0FC08B1002070BDE4
:10F928000AF050F90646284609F03CF9235C3344AE
:10F938005B785B07F2D10130204470BD2DE9F04FB0
:10F948000E4691B05F490446FFF7DCFF0546B0B9A3
:10F958005D492046FFF7D6FF054690B95B4920462A
:10F96800FFF7D0FF054670B920465949FFF7CAFF8F
:10F978000028054612BF08242546012404E0012476
:10F9880002E0022400E004240EB144F010045148BF
:10F99800FAF72AFC50492846FFF7B4FF08B144F0AB
:10F9A800200414F0090F00F010824C4808F040FAC7
:10F9B8000020FEF725FF04F01803182B02D1484851
:10F9C80008F036FA4748434F474EDFF8448108F0BD
:10F9D8002FFA2046FFF73EFC444808F029FA7B79C5
:10F9E8007579434AC3EB050EDEF1000503F1FF33D9
:10F9F80045EB0E05294658F82330204608F0DEF975
:10FA080073793B4A013B294658F82330204608F0D1
:10FA1800F5F9D6ED037A374AF5EE407AF1EE10FAA9
:10FA28000CBF01210021204608F0E8F9394620469C
:10FA3800FBF732FD304808F0FBF939462046FBF762
:10FA480077F92E4808F0F4F996F9E6102C4AB1FA3D
:10FA580081F14909204608F0D1F939462046FBF7DB
:10FA6800B1F8284808F0E4F9D7F808A00597D6F8BF
:10FA78000890254F0396002557F82560DFF8888001
:10FA880016B969EA0A0B63E04FF0010808FA05F8AD
:10FA98006AEA090313EA080F14BF0121002133465B
:10FAA8001A4A204608F08AF969EA0A0313EA080F95
:10FAB800164A334614BF01210021204608F09EF95A
:10FAC8000135D9E7C90C020892140208D00C0208C3
:10FAD800D60C0208F4350020DA0C0208E70C0208FC
:10FAE800F50C02082D0D0208B0450020380D02085B
:10FAF800440D02084F0D0208600D02086C0D020843
:10FB08007C0D02088B0D020804E40108990D020817
:10FB180094EB01080127B7401AEA070F09D01BEA3E
:10FB2800070F2B46B44A14BF01210021204608F0D4
:10FB380045F919EA070F0AD06AEA09033B42AE4AB7
:10FB48002B4614BF01210021204608F057F9013641
:10FB580058F82650002DDDD1A848DFF8FCB2DFF8B0
:10FB6800FCA208F065F9039BD3F8D865059BD3F888
:10FB7800D8357340DB4307934FF00109079A09FA18
:10FB880005F31A4218BF4F469D4A08BF0027334065
:10FB980006934FF00C0303FB0523394614BF5A465E
:10FBA80052469B680493204608F008F9069A049B7D
:10FBB800002A14BF52465A46394620464D4408F09A
:10FBC8001DF9122DD8D18F488F4D08F031F94E46C6
:10FBD8000023039A595D1A4410A892F8442210444D
:10FBE80010AF00F8201C0598184490F84402074408
:10FBF80007F8101C16B1171A7E427E410133082BF4
:10FC080006F00106E5D10CAB804A814FDFF8089277
:10FC18003146002520468DF8285008F0CFF808AB6B
:10FC28007A4A3146204608F0E9F87A4808F000F99F
:10FC38007949204601F0ACF8784808F0F9F8764997
:10FC48002046FBF79BFA764808F0F2F872492046FE
:10FC5800FBF7FCF9734808F0EBF86F492046FBF70F
:10FC680053F9714808F0E4F86B49204601F014F99B
:10FC78006E4808F0DDF868492046FBF753FD6C48EC
:10FC880008F0D6F864492046FBF770FB694808F08D
:10FC9800CFF897F8641299F86432994207D199F825
:10FCA800656297F86522901B4642464100E00026AF
:10FCB800022924D199F8652243444FF0190A40F2E9
:10FCC800EE2B1AFB02B293F83831019200933146B9
:10FCD8002B46594A204608F071F897F86532564A7B
:10FCE8001AFB03B3019397F864324344314693F8FF
:10FCF8003831009320462B4608F080F815E043443D
:10FD08004E4A93F83831009331462B46204608F086
:10FD180055F897F86432494A4344314693F83831E4
:10FD2800009320462B4608F069F80135122D07F19B
:10FD3800020709F10209ACD14148424E08F078F8AF
:10FD480021460020FDF7EEFD14F0080F2FD0039B8D
:10FD580093F828750025E8B22146FDF72DFEB36813
:10FD68002146002093F84480FDF746FE21460120F5
:10FD7800FDF742FE21460220FDF73EFE404602F016
:10FD88009DFD314808F054F80135304807F03BFF35
:10FD9800032DE0D1384602F04DFE2D4808F048F812
:10FDA8002A4807F049FF2B4808F042F80DE0039B6A
:10FDB800214693F82805FDF7FFFDB36893F8440042
:10FDC800022802D82146FDF717FEA20705D5104BD9
:10FDD800214693F82805FDF7EFFD630708D5194B71
:10FDE8009B6893F84400022802D82146FDF704FED8
:10FDF80011B0BDE8F08F00BFA70D0208B40D0208CE
:10FE0800A4EA0108C10D020824E60108CB0D020886
:10FE1800B0450020D40D0208F4350020E10D020899
:10FE2800EB0D0208F70D0208080E0208120E020870
:10FE3800210E02082F0E02083C0E02084E0E020880
:10FE48005D0E0208042500206A0E02087FF50108ED
:10FE5800970E0208C00E0208B00C0208BC0C02087B
:10FE680001216BE5002169E50379826803F030031D
:10FE7800102B06D10B4B93F828156C2301FB03229A
:10FE88000DE0202B0BD1074B93F82805064B1B7868
:10FE980003EB43039B006C2111FB00331A4410460B
:10FEA800704700BFB04500208E24002070472DE920
:10FEB800F04F2DED028B87B01C4607460391049244
:10FEC80004F01EFDB44B1B889E0709D53B7F97F8AD
:10FED800412097F84010208A04F094FC019001E03A
:10FEE80064230193DFF8B492B8460024AB4B4FEA81
:10FEF800840A5344D3ED007AA74B1888FDEEE77ABD
:10FF0800850717EE902A28D0022C26D0A44B33F967
:10FF180014100833650033F9143003EB4101039BD7
:10FF28005B42994203DB039B8B42A8BF0B469D496A
:10FF3800695E5B1A049931F914100B44C10703D5A3
:10FF48003A7A53431A1108E0B97C4B4301994B4361
:10FF5800642193FBF1F302EB2312934D5AF8053019
:10FF68000C35042193FBF1F12B5D029398F80130D5
:10FF7800029D501A43436B43642593FBF5F599F8AA
:10FF88002F30032B4FEAE51510D9B7F82EE0BEF154
:10FF9800000F0BD0022C0DD1CEF10006B542C0F2F5
:10FFA800F8807545A8BF75462E46F2E0022C01D1AF
:10FFB800BE8D00E07E8D98F80BC0002AB8BF524273
:10FFC800920192FBF6F2B2F5807FA8BF4FF48072DF
:10FFD80022EAE272C2F5807292B20CFB02FC6F4A0E
:10FFE800B2F830E002F1340B00FB0EF65AF80B20A1
:08FFF8004FEA2C2CF61206FB67
:020000040801F1
:100000000C26B6F5001F6B4AA8BF4FF400169642A7
:10001000B8BF1646022C4AF80B604FEA66366CD021
:1000200097F828300BF10C0B2BB95BF80A304BF822
:100030000A00C31A04E05BF80A304BF80A105B1A96
:100040004FF6FF704FEA1E1EB0FBFEFE03FB0EF3E1
:100050005811594B1B780B2B0CD198F81530029A7C
:1000600043435A431346642293FBF2F3534A1B1251
:1000700022F81430B7F820B0BBF1000F2CD0FB7F72
:1000800007EE900A012BB8EEE78A08D14C4B1C20F2
:10009000B0EE480A00FB043008F0A2FC18E073B987
:1000A00004F09AFC474B0C20F0EE400A5FFA8BF10B
:1000B000B0EE480A00FB043008F04CFD08E0424B6B
:1000C0004FF4F870B0EE480A00FB043008F034FC3E
:1000D000B0EE480A09F086FF98F815303B4A5843BD
:1000E000135D02F5CD625843642390FBF3F0AB1926
:1000F0000012034422F8143034E0798CA1B1029349
:10010000059104F069FC07EE905A0599F0EE400A5B
:10011000C9B2B8EEE70A0BF5CD6008F01BFDFDEEA5
:10012000C07A029B17EE905AA91909B2032BA9F8BD
:10013000981616D9FB7DB9F91020DB00C3F5C873FA
:10014000502BB8BF502382EAE270A0EBE2705A4213
:10015000121A914203DB1A188A42A8BF0A46A9F86C
:100160009826002099F8A83613B9194A22F81430B5
:10017000184B01344AF8035003F10C021833032CD6
:100180004AF802604AF8030008F101087FF4B2AEB1
:1001900007B0BDEC028BBDE8F08F35460CE700BF21
:1001A000D0240020102500201C2500202825002018
:1001B000302500200000E0FFCA210020CC210020D3
:1001C0005C250020B0250020D42500203C250020FF
:1001D000A42B0020BC2B00202DE9F04F2DED0C8B23
:1001E000BC4DDFEDBD9A1E4695F82C3007EE903AD7
:1001F00085B0F8EEE77A04460BEE101A019287EE0E
:10020000A9AA04F081FBB54B1B8813F0020FA84686
:10021000B7EE009A0ED0237F94F8412094F8401056
:10022000308A04F0F3FA07EE900AF8EEE77AC7EEA8
:10023000A9AA01E0F0EE49AA94F83530002B41D08C
:10024000B8F8D026D8F83000A24944F62065B5FBAE
:10025000F0F0904233D8B1F9D226B1F91200811AE8
:100260000029D6BF121A07EE901A07EE902AF8EE70
:10027000E76A07EE903AB8EE677ADFED997A27EEF3
:10028000277A67EE267AF5EEC07AF1EE10FA09D4F5
:10029000B1EE047AF4EE477AF1EE10FAC8BFF0EE50
:1002A000477A01E0DFED8F7A8F4BA8F8D20677EE20
:1002B000897AC3ED007A0023A8F8D03602E0013233
:1002C000A1F8D026834E002506F2EC63274606F2FD
:1002D000D46B06F5DC6A0093A946844B7A7819F84A
:1002E000031091420CD1D91C97F80BE019F80100CA
:1002F000864505D1991D787D19F80110884266D090
:1003000007EE902A9FED7A7A7A4B208FF8EEE77A03
:10031000591967EE877A03F10C02C1ED007AFB7A76
:100320009FED757A029207EE903AF8EEE77A51194E
:1003300067EE877A9FED717AC1ED007A7B7D07EEDB
:10034000903AF8EEE77A67EE877ACBED007A94F888
:10035000373007EE903AF8EEE77A87EEA97A81ED2A
:10036000037A94F8363007EE103AB8EEC77A4FF4B5
:100370007A71C7EE297A4843039179EE677ACAED1C
:10038000007A07EE900AB8EEE78A04F025FB608F4A
:100390000399029A414328EE000A07EE901A82ED73
:1003A000060AB8EEE78A04F017FB504B7978029AF8
:1003B00003F80910A2F11501F87A01F8090028EEF6
:1003C000000A797D82ED070A123A02F80910B9F1A4
:1003D000020F0CBF4A4A4B4A92ED007AB5EE407AC2
:1003E000F1EE10FA22D0484AD6ED007A2A44D2ED36
:1003F000006A77EEE67AF5EEC07AF1EE10FA00F3D5
:10040000F281B1EE676AB4EEC67AF1EE10FA0BD55E
:10041000F5EEC07AF1EE10FA02DD37EE267A01E051
:1004200036EEC77A86ED007A316811602B4A128861
:10043000910700F08080B9F1020F7CD03348D4EDF1
:100440000F6A30F91930083807EE103A30F91930D0
:1004500007EE903A1BEE103AF8EEE77AB8EEC77A5C
:100460005B42A6EEA77A4FEA490107EE903AF8EE12
:10047000E77AB4EEE77AF1EE10FA08D4F8EECB7A28
:10048000B4EEE77AF1EE10FAD8BFF0EE477A2048E2
:100490000B5E07EE103A019BB8EEC77A33F91930BC
:1004A00037EEC77A07EE903AF8EEE77AF2EE046A92
:1004B00077EE277AD30787EEA66A2BD5237A07EE45
:1004C000103AB8EEC77A67EE067A87EEA67A86ED1E
:1004D000007A30E0102500200000C842D02400201F
:1004E0006F12833A0000000054050020082C002001
:1004F000D730033D142C0020033F7A3E97AC0A3AD4
:10050000382C00203C2C0020402C002024250020EA
:1005100028250020A37C07EE903AF8EEE77A67EEF4
:10052000867A67EEAA7A87EEA67AD6ED007A77EE1B
:10053000877AC6ED007AB9F1020F0CBFA38D638DE7
:1005400096ED00CAAB4ADFEDAC7A06EE903A51194F
:10055000B5EEC0CAF1EE10FA91ED007A51ED0EBA87
:10056000F8EEE66AD4BFB1EE4C6AB0EE4C6A87EEA4
:1005700027DAC6EE267A3CEE4D7A79EE677A67EE98
:100580002BBAF5EEC07AF1EE10FA6BEE8ABAF7EEFE
:10059000006A07D4F4EE667AF1EE10FAC8BFF0EE06
:1005A000667A01E0DFED957A954A92ED008A954AE8
:1005B000511951ED0ECAD1ED008A029127EE888AB9
:1005C00067EE2CCA04F008FA2CEE800ADFED8E7A72
:1005D0000299E8EE008AF4EEE78AF1EE10FA09D407
:1005E000DFED8A7AF4EE678AF1EE10FAC8BFF0EE1A
:1005F000678A01E0F0EE678AB9F1020FC1ED008A67
:1006000000F0A580824A5119D1ED007A94F8361095
:10061000632929D8B5EEC0CAF1EE10FA0ADD009BB5
:1006200093ED007A7CEE476AB4EEE67AF1EE10FACA
:100630001ADD0AE018D5009B93ED007A7CEE476A3C
:10064000B4EEE67AF1EE10FA0ED52A44DAED006A3D
:1006500092ED0E7A39EE666A27EE077A27EE277A50
:1006600066EE277AE7EE267A6A4A009B97EE8CDAE6
:100670002A4492ED008A83ED00CA82ED00DA04F08C
:10068000ABF989EE000A644A12780B2A3DEE488ADB
:1006900020EE088A0CD1DBED007A604968EE277AFB
:1006A00067EE8A7AFDEEE77A17EE902A21F8192094
:1006B00098F868274AB15A4A1C20B0EE480A00FB55
:1006C000092008F08DF9B0EE408A218C39B3E27F21
:1006D000012A08D1534A1C20B0EE480A00FB092029
:1006E00008F07EF919E0029172B904F075F90299E7
:1006F0004D4A0C20F0EE400AC9B2B0EE480A00FBA9
:10070000092008F027FA08E0484A4FF4F870B0EEE4
:10071000480A00FB092008F00FF9B0EE408A9BED73
:10072000000A28EE008A3BEEA80A28EE0A8A30EE7C
:10073000080A09F057FC218E4A42904203DB8842A6
:100740000246A8BF0A463A4921F8192017E0618CF1
:1007500069B1029104F040F902993648F0EE400A7E
:10076000C9B2B0EE6B0A08F0F5F9F0EE40BA3BEE14
:10077000A80A09F037FC9FED218AA8F8980698F896
:10078000A82612B92A4921F81920FDEEEBBA2A4A07
:100790001BEE903AFDEEE88A42F8293002F10C0196
:1007A00018EE903ABDEEC88A41F82930183218EE9A
:1007B000103A42F82930009B09F101090433B9F1DC
:1007C000030F07F1010705F1040506F104060BF11B
:1007D000040B0AF1040A00937FF47FAD05B0BDEC71
:1007E0000C8BBDE8F08FB4EEE77AF1EE10FA3FF52E
:1007F00014AE19E64C2C0020333383410000000076
:1008000054050020582C002000007AC300007A43D1
:100810002C2C0020702C0020CA210020CC2100208C
:100820007C2C00205C250020B0250020D425002051
:10083000A42B0020AC2B0020BC2B00200C4B10B5AF
:10084000014604461868FBF740FC0A4B188808224A
:1008500080EA042010F4004F4FEA40001CBF80F4EF
:10086000815080F00100013A80B2F3D1188010BDB0
:10087000744200207C42002010B5064C2068FBF733
:1008800021FC0028FAD0034BBDE810401868FBF7A4
:1008900016BC00BF7442002008B5FFF7EDFF0A4AFE
:1008A000138883EA00239BB2082113F4004F4FEA18
:1008B00043031CBF83F4815383F0010301399BB2CE
:1008C000F3D1138008BD00BF7842002010B5044664
:1008D0002046FBF7EEFB18B90A2004F02BFBF7E7E4
:1008E00010BD30B5084C00230C2101FB03425568B4
:1008F000A84203D00133052BF7D130BD0023C362DA
:100900001381536030BD00BFAC4B00202DE9F34193
:10091000054688469DF82070234811461A469DF8E2
:10092000243000264FF00C0C0CFB06F404EB000EF8
:100930002456AC4203D00136052EF5D102E0BEF8B4
:10094000080008B100202BE0022D11D006DC5DB1BB
:10095000012DF7D1009315483B460CE01E2D0ED01B
:100960001F2DEFD101200AE0009311483B4602E021
:10097000104800933B46FBF714FA044605E0F6F7EF
:10098000FBFD39460446FBF791FB002CDAD0064A02
:1009900025710C2303FB06262046A6F80880746008
:1009A00002B0BDE8F08100BFAC4B00200044004025
:1009B000003801400048004010B5084B196800227B
:1009C00001EBC20393F90240844201D1981C10BD8F
:1009D0000132052AF4D1002010BD00BFA84B002031
:1009E00038B1438813EA010003D08B420CBF0120C9
:1009F0000220704770B50D4B0D491D6891F8C02756
:100A00000024042A0DD8134605EBC303541C9E880A
:100A10003042E2B24FF00104F3D081F8C027981CB5
:100A200070BD0CB181F8C027002070BDA84B00201C
:100A300010250020024B002283F8C027DAE700BF10
:100A4000102500202DE9F74F274B284A1B68126814
:100A500090F803E090F80480254DC3F3007313422F
:100A60001FFA8EF303EB8307C3F10002C3F178038F
:100A7000CEF1640C9BB208BF0E88019318BF4FF4EF
:100A80007A765FFA8CFC7F00C8F1640B92B24FF06B
:100A90000A0A4FF47A7913B2002B02DC03D1012445
:100AA00002E0644600E0744603FB03F008FB00F03C
:100AB00014FB04F490FBF4F45C44634393FBFAF3FB
:100AC0003B441BB225F8023F4888801B434393FBFD
:100AD000F9F333442B800A32019B92B29342DAD16C
:100AE00003B0BDE8F08F00BFD4240020982400207C
:100AF000D02C002030B50C784D78AC421CD2011DB2
:100B00000E4B33F91130B3F5617F05DB40F633024C
:100B10009342A8BF134601E04FF46173192240F2DB
:100B2000833112FB0414A34206DD12FB051083423D
:100B3000CCBF0020012030BD002030BDE42D0020BE
:100B40000C4B1B6813F4805F0B4BB3F9063009D0D4
:100B50000A4A1268D20005D4008A421A934207DD7D
:100B6000084400E0408A8342B4BF0020012070475F
:100B70000120704798240020E42D0020D424002078
:100B800038B50D4B1B681B0305460C4613D50B4BA4
:100B900093F8DA37093B012B0DD8452007F008FC04
:100BA0000D2007F005FC284607F002FC2046BDE8B2
:100BB000384007F0C6BC38BD98240020102500201E
:100BC000044B1B681B015DBF034B1868C0F38050CA
:100BD00001207047D42400209824002010B5002064
:100BE000FBF7A2F8074B00241C70FEF7EDF9064B4B
:100BF00083F8DB47C3F8DC47A3F8E047C3F8E447D2
:100C000010BD00BFC82400201025002030B470B1F2
:100C1000194BD3F8D83513F400330BD0174B1B689E
:100C200013F0020306D0164B1B78012B01D830BC01
:100C3000D4E70023134A0C2505FB03F18C18895CCB
:100C4000814203D00133142BF6D112E00E4AD2F8C0
:100C5000E41719B16078497888420AD209490C2012
:100C600000FB0313C2F8E4370023A2F8E037C2F810
:100C7000DC3730BC704700BFB0450020982400200E
:100C800040050020A4EA0108102500204000142897
:100C9000094A30B4A8BF14200023022514249D540F
:100CA00002339918984201F8014CF8DC024AFF21FE
:100CB000D1540F2030BCA9E7794C00202DE9F8432E
:100CC00004F0FAF8DFF88C80054600F1FA0998F88C
:100CD0000040204FA40008EB0406706801F06EFB92
:100CE00058B104F0E9F88145F1D24FF0FF30BDE88A
:100CF000F88304F0E1F88145F7D37068DFF8548099
:100D000001F05CFB0028F4D004F0D6F8D8F83830B5
:100D1000401B9842C8F8340018D805F5FA753E19FA
:100D2000706801F04BFB20B104F0C6F88542F7D2A1
:100D3000DBE73C44606801F041FB20B904F0BCF8FB
:100D40008542F7D2D1E70020BDE8F8830120BDE855
:100D5000F88300BFF82C002038B500240546047045
:100D6000FFF7ACFF431C13D0012802BF2B78A04033
:100D7000184304F1010408BF2870082CF0D1054A7B
:100D8000297892F83C304B4082F83C30012038BD45
:100D9000002038BDF82C00202DE9F0473C4CDFF84E
:100DA000FCA03C4F86B080460D4604F1280994F91A
:100DB000B622002313F90A10914203D00C333C2BC6
:100DC000F8D15AE095F9B6329A4295F8BC225CD136
:100DD000B4F8B802B5F8B812884256D194F8BA02FD
:100DE00095F8BA12884250D194F8BB0295F8BB121C
:100DF00088424AD194F8BD0295F8BD12884244D188
:100E000094F8BC12881A4142414157F822200492BA
:100E100095F8BD2257F82220039295F8BB2257F887
:100E20002220029295F8BA2257F822200192B5F8B2
:100E3000B82200924046184A0E4606F0C3FF94F8C6
:100E4000BC2294F9B63257F82220049294F8BD22BD
:100E500057F82220039294F8BB2257F822200292DE
:100E600094F8BA2257F822200192B4F8B8220092DE
:100E70003146094A404606F0C5FF08344C4505F1A5
:100E8000080594D106B0BDE8F0870021BDE700BF9A
:100E9000B045002004E60108880F0208AC4B002092
:100EA0002DE9FF47294C81460E4600274FF01908CF
:100EB00094F8293596F8290596F82C25834296F85A
:100EC0002B350FD194F82A5596F82A158D4209D161
:100ED00094F82B15994205D194F82C158D1A694276
:100EE000694100E000214FF4617A18FB02A218FB6F
:100EF00003A30392029396F82A35154A8DE8090058
:100F00003B4648460D4606F05DFF94F82B3594F8B5
:100F10002C2518FB03A3029394F82A35019318FBA0
:100F200002A294F8293503920093094A3B462946C8
:100F30004846013706F066FF142F04F1040406F159
:100F40000406B5D104B0BDE8F08700BFB04500206D
:100F5000A70F020808B520210BF0B5F90346184683
:100F600023B10278202A03F10103F8D008BD2DE94E
:100F7000F84380460C4615464FF00009192640F606
:100F800034074046FFF7E6FF8046B8B108F00AFE96
:100F9000B0F5617F03DBB842A8BF384601E04FF4EB
:100FA0006170A0F5617090FBF6F0B9F1000F01D10E
:100FB000207000E060702B7801332B7009F101097B
:100FC000B9F1020FDDD14046BDE8F88313460A4669
:100FD0000146014806F09ABDBC0F020873B50178BE
:100FE000044619B90120FFF75BFF41E008F0DAFD84
:100FF0001328054637DC0023601C8DF80730FFF707
:10100000A9FF1C4C064605F5A57558B108F0CAFDA8
:101010001D2807D804EB850358709DF8073001336D
:101020008DF807303046FFF795FF064658B108F0B7
:10103000B9FD0D2807D804EB850398709DF807309B
:1010400001338DF8073004EB85040DF10702E11C34
:101050003046FFF78CFF9DF80730042B08D00023A3
:10106000C4F8013004E0132200210348FFF7AEFF6B
:1010700002B070BDB0450020D5F80108014806F067
:10108000DBBE00BFDB0F02082DE9F743017821B971
:10109000012003B0BDE8F0437EE6002200920192F9
:1010A000451C08F07FFD44B22046FFF785FC06464C
:1010B00018B18DF80040012400E004462846FFF7EF
:1010C00049FF074628B108F06DFD0134ADF8020074
:1010D000E4B2DFF88C900025C8463846FFF73AFFA7
:1010E000074680B308F05EFD002159F821209042A8
:1010F000CBB203D001310829F7D1002358F82320BF
:10110000904220D1022D0FD0032D12D05A1E012D56
:10111000D2B204D0042A13D88DF804300EE0042A89
:101120000ED88DF8053009E0052B09D88DF8073069
:1011300004E09A1E052A03D88DF806300134E4B283
:101140000135042DC9D1052C03D803B0BDE8F04307
:1011500094E76B4603CB3060716003B0BDE8F08369
:1011600004E60108F7B5047805464CB901A9204604
:1011700001F082F80134FFF7F5FF122CF6D16DE093
:1011800008F010FDC4B2112C63D8681CFFF7E2FE12
:10119000334D074640B9334B03EB440393F86412D5
:1011A0008A1E514251413CE0017828460BF08BF8F1
:1011B00050B12D4A401B032C8CBF0323002352FA4D
:1011C00080F0C65C032E02D1FFF758FF46E0384698
:1011D000FFF7C0FED8B1022EF6D108F0E3FC40F2D2
:1011E000ED2380B2984205DD40F6CA039842A8BFBD
:1011F000184601E040F2EE201A4B03EB4403A0F244
:10120000EE20192290FBF2F083F8650201E0022E35
:10121000DAD0B31E59425941124B03EB440383F811
:101220006462104A04F5987302EB43031A79AA5CCE
:1012300051B15B7940F2EE21192000FB03132146E6
:101240000A4806F063FC09E02146094806F05EFC06
:1012500004E0112200210748FFF7B8FE03B0F0BDFB
:101260003CE50108B0450020FDE501083C0E020800
:101270004E0E0208B7FB010808B5044806F0DCFD75
:10128000034B1868BDE8084001F0D8BAE90F02081E
:10129000284C0020F7B50023454C464E8DF803300E
:1012A0006023A3633378152B074606D0122B04D096
:1012B000012B0CBF02258C2501E044F62065FFF7C9
:1012C000FDFC002802DA013DF9D16EE00A25FFF7A6
:1012D000F5FC013069D0013D15F0FF05F7D1626BD7
:1012E000930803EB5203A363FFF7E8FC431C5CD0B5
:1012F0000028F9DC00230DF1030084F83C30FFF7EF
:101300002BFD002851D09DF803301B2B4DD10DF142
:101310000300FFF721FD002847D0254B9DF803204F
:1013200093F83D309A4240D10DF10500FFF714FDCE
:101330009DF80530012B38D801A8FFF70DFD9DF869
:10134000043093B30DF10300FFF706FD68B39DF879
:1013500003300E2B29D10DF10300FFF7FDFC20B364
:101360009DF8032033789A421FD10DF10300FFF757
:10137000F3FCD0B19DF80330BBB93D46BDF8043055
:10138000EA1B92B2023B9A4205DA2846FFF7E4FCD8
:1013900058B10135F2E70DF10300FFF7DDFC94F8D9
:1013A0003C00B0FA80F0400900E0002003B0F0BD3E
:1013B000F82C0020E0350020F8B51B4C94F83E30A6
:1013C0004340074684F83E300826257804EB85051F
:1013D000FB07686809D500F0E2FF402003F088FDB4
:1013E000686800F0D7FF402014E000F0D8FF20200C
:1013F00003F07EFD686800F0CDFF202003F078FD4B
:10140000686800F0CCFF202003F072FD686800F0EF
:10141000C1FF2020013E03F06BFD16F0FF064FEAEE
:101420005707D2D1F8BD00BFF82C002010B50A4CE8
:1014300094F83E00FFF7C0FF237804EB8304606854
:1014400000F0ADFF202003F053FD60682021BDE8CF
:10145000104001F00BB800BFF82C002010B5104C64
:10146000237804EB83030121586800F0FFFFFF207D
:10147000FFF7A2FFFF20FFF79FFF7F20FFF79CFFF2
:1014800000231B2084F83E30FFF796FF94F83D00C0
:101490000130C0B284F83D00BDE810408CE700BFC9
:1014A000F82C00200B4B10B501241C70FFF7D6FF61
:1014B0000020FFF781FF2046FFF77EFF0E20FFF799
:1014C0007BFF2046FFF778FFFFF7B0FF0248BDE83B
:1014D0001040DFE6E0350020E135002073B50478E8
:1014E00005462CB104F10A03ADF80430002604E0EF
:1014F0004FF48573ADF804300126FFF7AFFF9DF878
:101500000500FFF759FF9DF80400FFF755FF0E2077
:10151000FFF752FF184B1878FFF74EFF3046FFF7E2
:101520004BFF2046FFF748FF0020FFF745FF002054
:10153000FFF742FF0020FFF73FFF0020FFF73CFFCF
:101540000020FFF739FF0020FFF736FF0020FFF7EC
:1015500033FF6B681878FFF72FFF6B68013C01338E
:1015600014F0FF046B60F4D1FFF760FF034802B092
:10157000BDE870408EE600BFE0350020E135002078
:1015800038B505460478FFF769FF0020FFF714FF20
:101590000420FFF711FF0E20FFF70EFF0A4BB4FAED
:1015A00084F418786409FFF707FF2046FFF704FF6B
:1015B0002878FFF701FFA020FFF7FEFEFFF736FFB8
:1015C0006868BDE8384065E6E035002038B5036856
:1015D000164A23F07F4323F0FF039342044622D0B0
:1015E000134B06251D70FFF739FF0020FFF7E4FEBF
:1015F0000520FFF7E1FE0E20FFF7DEFE2846FFF78D
:10160000DBFE0020FFF7D8FE0020FFF7D5FE607854
:10161000FFF7D2FEA078FFF7CFFEFFF707FF0548E0
:10162000BDE8384036E6012038BD00BF00FFFF00AE
:10163000E0350020E135002070B5800040F4806482
:1016400003F03AFC0C4D44F0010406462B7805EB00
:1016500083035868E30702D500F0A1FE01E000F023
:1016600099FE640806F1340604D003F025FC864296
:10167000FBD8EBE770BD00BFF82C002010B50D497A
:10168000B1F83F30082280EA030414F0010F4FEA5A
:10169000530318BF83F4204302F1FF3214BF83F0D9
:1016A00001039BB212F0FF024FEA5000EBD1A1F808
:1016B0003F3010BDF82C002037B502ADFF2305F8F0
:1016C000013D0446284603F0B5FC10B90CB1013CBD
:1016D000F8E79DF8070003B030BD73B5FE238DF821
:1016E000043000238DF805308DF806300B788DF826
:1016F000073006460C46154613B901238DF806300F
:1017000004210DEB010003F05DFC0220FFF7D4FF84
:10171000FF281CD12178606803F054FC2820FFF7D3
:10172000CBFFA0F130025042504188B10123022189
:1017300001A88DF805308DF8046003F043FC2846BD
:10174000FFF7BAFFA0F130035842584100E00020F3
:1017500002B070BD07B50368114A23F07F4323F040
:10176000FF03934218D0FF238DF804300023042197
:101770008DF8053043788DF8063083788DF8073082
:101780000DEB010003F01EFC0220FFF795FFA0F116
:1017900030035842584100E0012003B05DF804FBDB
:1017A00000FFFF0037B5054608460C46FFF7D2FF9D
:1017B00060B123788DF80450022101A88DF805301E
:1017C00003F000FC2178606803F082FC03B030BDB8
:1017D000024B00221A7005F0DFBA00BFA44B0020B4
:1017E0002DE9F74F0120FFF725F9184EDFF860903B
:1017F00000244FF04C0828B3012C23D808FB04F731
:1018000006EB070AF55915B10134E4B2F3E70379A1
:1018100090F9000059F8233001950322009201212C
:101820002A46FFF773F8834640B14C2229465046BA
:101830000AF012FD013446F807B0E4B20120FFF7C8
:10184000D9F8D8E703B0BDE8F08F00BF3C2D0020E9
:1018500004E601082DE9F0412D4F07F1100408F0CE
:10186000B5F93B4613F801EB7044427802F00402EC
:1018700002F0FF052AB19C421F46F0D10020BDE8CE
:10188000F081234AB91A022909DD12F8011B05EB80
:101890008505303901EB450505F0FF05F2E7002627
:1018A000974209D912F8011B06EB8606303901EB85
:1018B000460606F0FF06F3E7BEF12E0F1AD1984652
:1018C0000427002408F082F998F80020104404EB63
:1018D0008404437864005B07A4B244BF303AA41880
:1018E00007F1FF3744BF08F10108A4B217F0FF0762
:1018F000E8D100E0002464204443064800FB06468B
:101900000620B6FBF0F6044800FB0560BDE8F08158
:10191000D42D002040420F008096980012490023E9
:10192000F0B51A460D461E460A278C1894F89840C2
:10193000B4B12E2C05D1013290B18C18044484F836
:101940009860AC187B4394F89840A4F1300EBEF137
:10195000090F9CBF303B1B190E2A03D80132E4E764
:101960001846F0BD0020F0BD3C2D0020114B034473
:1019700010B5044693F8200002F047FA0E4800EB39
:101980004400B0F9A810B1F57A7F05DBB1F5FA6F24
:10199000A8BF4FF4FA6101E04FF47A71A1F57A71B2
:1019A0000A23092091FBF3F1BDE81040C9B2FBF70F
:1019B0001DBB00BF04E601083C2D00200C4680B58D
:1019C00015460646FEF782FF2046FEF77FFF154BC1
:1019D000002D08BF1D46002005F062F93046FAF7D9
:1019E00071FB78B1012005F05BF93046FAF767FB2F
:1019F000014607462046FAF768FB3846A84700200C
:101A000005F04EF92046FAF75DFB0028E6D00120EC
:101A100005F046F92046FAF752FB01463046FAF740
:101A200054FBD8E7B5FE0008F0B505460C4689B072
:101A30001422002120460AF00FFC2A681F4E04A938
:101A4000C2F3855000230D4640FA03F7FF0744BF59
:101A50009F5D0F7003F1010348BF0131062BF3D1E5
:101A6000174800230B70C2F303210144C2F305366B
:101A700091F83B108DF8181042300DF1190146FA1B
:101A800003F7FF0744BF1F5C0F7003F1010348BF5A
:101A90000131062BF3D100230B70C2F38343029371
:101AA00006AB0193009502F00F030649C2F303123F
:101AB0002046F8F79BFF09B0F0BD00BF39E60108EA
:101AC00004E60108EE0F020838B50E4C94F8D31066
:101AD00084F8CF0001F03F018B1C01F10A0584F866
:101AE000D13084F8CE5004F1CC000831FDF754FA1F
:101AF000254485F8CA0094F8CE301C44000A84F8C6
:101B0000CB0038BD3C2D002073B5224C04F1F80306
:101B1000C4F8F430204B93F84C325BB1012B14D154
:101B2000032284F8FA20072284F8FC3084F8FB2092
:101B30000C2308E0022284F8FA20032284F8FC3007
:101B400084F8FB20072384F8F830144B144A1A60F9
:101B50004020FEF76FFF0546C8B105F049FE95F934
:101B60000060002814BF03230123002205460192D0
:101B700000930C4A4FF4E13340213046FEF7C6FE95
:101B80000DB1C4F80001003018BF0120FFE702B01A
:101B900070BD00BF3C2D0020B0450020580500203E
:101BA00019E40008C9E500082DE9F0472DED028B86
:101BB000D64C88B094F804519DF848809DF84C703C
:101BC0000E4699464FF0010E0B28034628BF00230E
:101BD0000EFA03F040F2B2710140F9B910F04D0F66
:101BE0001CD0022D1AD1CA4BC4F80831C94BC4F815
:101BF0000C3194F80531002B0CBF6F236E2384F851
